:020000040800F2
:100000000000012071400008BD270008BF2700083C
:10001000C1270008C3270008C5270008000000000A
:10002000000000000000000000000000C7270008DA
:10003000C927000800000000CB270008CD270008D2
:10004000C1400008C1400008D1270008C140000895
:10005000C1400008C1400008DD270008E327000870
:10006000C1400008C140000815280008C140000830
:10007000E9270008EB270008ED270008F92700080A
:100080000528000811280008C1400008C1400008E8
:1000900000000000C140000817280008C140000807
:1000A000C1400008C1400008C1400008C14000082C
:1000B000C1400008C1400008C1400008C14000081C
:1000C000C1400008C1400008C1400008C14000080C
:1000D000C140000821280008C1400008C1400008B4
:1000E000C14000081D2800082D280008C140000854
:1000F000C14000080000000000000000C1400008EE
:10010000C1400008C140000839280008C14000086B
:10011000C1400008C1400008C1400008C1400008BB
:10012000C1400008C1400008C1400008C1400008AB
:08013000C1400008C1400008B5
:1001380010B5054C237833B9044B13B10448AFF319
:1001480000800123237010BDCC08002000000000AF
:10015800E03B010808B5034B1BB103490348AFF363
:10016800008008BD00000000D0080020E03B010826
:1001780014214160704714207047406A704700009E
:10018800790100087F01000883010008990100082F
:1001980010B5044604F1100000F05CFCC4F8F80047
:1001A8000148C4F87C0110BD88010008F8B5E6B024
:1001B80004460D4616461F460A4906A800F0CAFE20
:1001C80070996F9A05910492009733466E996D9ACB
:1001D800039102922A466C990191214600F060F839
:1001E80067B0F0BD94010008F8B5E6B004460D46C6
:1001F80016461F46094906A800F0ACFE6F996E9A8C
:100208000491039200976D996C9A0291019233467A
:100218002A46214600F087F867B0F0BD940100082F
:1002280038B500281CBF01680029184A23D1184B8B
:100238001C684FF6F0710C404CF24025AC421FBFD1
:100248001B6819404CF27024A14212D1114D296843
:1002580079B911490B68C3F30B03B3F58A6F1FBF54
:100268000968C1F30B0140F28343994204BF01219D
:10027800117028B905E0094B994204BF012111709A
:100288004068BDE8324001F09FBE00BFE80800208A
:1002980000ED00E0002004E00010005C000037489A
:1002A8002DE9F04104460D46216816464A681F4666
:1002B80090478046B8F5403F2ED122680A99936846
:1002C800204698478046B8F5403F25D12368089ACC
:1002D8000799D3F80CC02046E0478046B8F5403F60
:1002E8001AD12368069A39461F692046B8478046BE
:1002F800B8F5403F10D1236829465D69324620464B
:10030800A8478046B8F5403F06D123680B9A09995B
:100318009D692046A847804621680A68204690477C
:100328004046BDE8F0812DE9F04104460D462168BC
:1003380016464A681F4690478046B8F5403F2ED17A
:1003480022680A999368204698478046B8F5403F46
:1003580025D12368089A0799D3F80CC02046E047AE
:100368008046B8F5403F1AD12368069A39461F6976
:100378002046B8478046B8F5403F10D12368294643
:100388005D6932462046A8478046B8F5403F06D109
:1003980023680999DD6900222046A847804621681C
:1003A8000A68204690474046BDE8F0814FF4403047
:1003B80070470000F0B50C4685B0114600281A4673
:1003C8001CBF0568002D0B4B11D082B104B971B95F
:1003D8000D9860B10F9E0E9F0A9B0290049603979A
:1003E8000B980C9E009001962046A8470346184695
:1003F80005B0F0BD020003002DE9F04F0646D0B06D
:100408000868F56DD6F860E0726EB76EF36E00BAE4
:1004180000906C46486800BA60600DF14008886832
:1004280000BAA060C86800BAE060086900BA206134
:10043800486900BA6061886900BAA061C86900BAF1
:10044800E061086A00BA2062486A00BA6062886A95
:1004580000BAA062C86A00BAE062086B00BA2063FA
:10046800486B00BA6063886B00BAA063C86B00BAB7
:10047800E063402058F80C1C58F820CC58F838ACE9
:100488008CEA010158F840CC8AEA01018CEA01099A
:100498004FEAF979401E48F8049BEBD187EA02003D
:1004A80000EA0E00784010EBF5610098DFF824C4EC
:1004B80041186144C81882EABE032B404FEAF06134
:1004C80053405918636859186144CF194FEAB50366
:1004D80083EABE01014081EABE0111EBF765A1681C
:1004E8004D196544A91883EAB0023A404FEAF1650C
:1004F8005A405519E26855194FEAB70282EAB0071F
:1005080065440F4005EBBE0E97EAB00717EBFE6592
:1005180027697D194FEAB10782EA0701654401EAB4
:100528000E01EB18514011EBF36561694D194FEA63
:10053800BE0187EA010E65440EEA030E15EBB00012
:100548008EEA070E0EEBF065D4F818E075446544A2
:10055800AA1881EAB30505404FEAF26E4D40AE4451
:10056800E569AE44E64477444FEAB00080EAB30E4A
:100578000EEA020E8EEAB30E0EEBF765D4F820E011
:1005880075446544691880EAB2053D404FEAF16E4A
:100598004540AE44656AAE44E6440EEBB3034FEA09
:1005A800B70787EAB20E0EEA010E8EEAB20E0EEB1C
:1005B800F365D4F828E075446544281887EAB1053E
:1005C8001D404FEAF06E7D40AE44E56AAE44E64415
:1005D8000EEBB2024FEAB30383EAB10E0EEA000E45
:1005E8008EEAB10E0EEBF265D4F830E0754465443E
:1005F800EF1983EAB00515404FEAF76E5D40AE4447
:10060800656BAE44E6440EEBB1014FEAB20282EAF2
:10061800B00E0EEA070E8EEAB00E0EEBF165D4F8B6
:1006280038E075446544EB1882EAB7050D404FEA97
:10063800F36E5540AE44E56BAE44E6440EEBB000B5
:100648004FEAB10181EAB70E0EEA030E8EEAB70E41
:100658000EEBF065D4F840E07544654481EAB30ECA
:10066800AA180EEA000E4FEAF2658EEA010E7544EA
:10067800DDF844E04FEAB000754480EAB30E654403
:100688000EEA020E15EBB7078EEAB30E0EEBF7650E
:10069800DDF848E04FEAB202754480EA020E65448C
:1006A8000EEA070E69188EEA000E0EEBF165DDF80A
:1006B8004CE07544654405EBB3034FEAB70E1427C5
:1006C8000DF1500CDFF810528EEA010B82EA0B0B89
:1006D8000BEBF36A5CF804BBDA44AA44504483EA9F
:1006E800B10B4FEAF06A8EEA0B0BDA445CF804BBF4
:1006F800DA44AA44524480EAB30B4FEAF26A8BEA1E
:10070800B10BDA445CF804BBDA444FEAB000AA44FF
:1007180080EA020BD6448BEAB30B0BEBFE6A5CF85B
:1007280004BBDA444FEAB202AA4482EA0E0B0AEB8F
:10073800B10180EA0B0B0BEBF16A5CF804BBDA44FD
:100748007F1DAA44282F0AEBB3034FEABE0EBBD382
:100758003C2F61D3502F4DD204EB870CC7F15407BF
:100768005E4CA7FB04A504465D4FA8088EEA010A63
:1007780082EA0A0A5CF804BB0AEBF3655D447D195A
:100788002C1983EAB10A4FEAF4658EEA0A0A55443D
:100798005CF804AB5CF804BB55447D19AA1884EADC
:1007A800B30A4FEAF2658AEAB10A55445D444FEA52
:1007B800B4047D1984EA020AAE448AEAB30A0AEB51
:1007C800FE655CF804AB55444FEAB2027D1982EA33
:1007D8000E0A15EBB10184EA0A0A5CF804BB0AEBBD
:1007E800F1655D447D1915EBB303401E4FEABE0E5B
:1007F800BCD12046F46D1B19F365336EC9183166F8
:10080800716E71447166B36ED218B266F16E40189B
:10081800F06650B0BDE8F08F4EEA010B0EEA010A0F
:100828000BEA020B4BEA0A0A0AEBF36554F827A015
:10083800DFF8B0C0554443EAB10B654403EAB10A96
:100848000BEA0E0B28184BEA0A0A7F1C0AEBF06524
:1008580054F827A0554440EAB30B654400EAB30AAC
:100868000BEAB10BAA184BEA0A0A7F1C0AEBF265DD
:1008780054F827A055444FEAB00040EA020B6544FB
:1008880000EA020A0BEAB30BAE444BEA0A0A7F1CE1
:100898000AEBFE6554F827A055444FEAB20242EA33
:1008A8000E0B654402EA0E0A0BEA000B15EBB101C8
:1008B8004BEA0A0A7F1C0AEBF16554F827A0554455
:1008C8007F1C65443C2F05EBB3034FEABE0EA3D350
:1008D80040E700BF9979825AA1EBD96ECDCCCCCC38
:1008E800D6C162CADCBC1B8F00B581B00168074A5B
:1008F800914200D110B9064801B000BD7C2113F027
:10090800D3F84FF4003001B000BD00BFFC09000867
:10091800030002002DE9F0410B4A92E8F85188B033
:10092800694681E8F8510268084B9A4200D118B923
:10093800074808B0BDE8F0811422083000F04FFBEA
:1009480008B0BDE8F08100BFDC090008FC09000818
:1009580003000200152904D20268044B9A4200D110
:1009680008B903487047083000F048BBFC09000884
:100978000300020010B481B013460268074CA2427B
:1009880000D118B901B010BC0548704701B000F19A
:10099800240210BC083000F035BB00BFFC09000879
:1009A8000300020010B481B013460268074CA2424B
:1009B80000D118B901B010BC054870470A4601B00B
:1009C80000F1240110BC083000F070BBFC090008DD
:1009D800030002000123456789ABCDEFFEDCBA981E
:1009E80076543210F0E1D2C300000000000000008D
:1009F80000000000F10800081D0900085D09000852
:100A08007D090008AD09000801040008790F0008F5
:100A1800C50F0008810F0008F0B5A3B004460B48C5
:100A280002900D4616461F46094B0822402104A88D
:100A380000F0D1FA28980190009733462A462146BB
:100A480002A800F01BF823B0F0BD00BFFC090008A5
:100A5800100A000810B5040008BF002408D0054893
:100A6800054B20600822402104F1080000F0B3FA89
:100A7800204610BDFC090008100A00082DE9F041C5
:100A880004460E46216817464A681D469047804628
:100A9800B8F5003F19D1226806999368204698470F
:100AA8008046B8F5003F10D123683146DE683A46E3
:100AB8002046B0478046B8F5003F06D12368079A1C
:100AC80029461D692046A847804621680A682046AD
:100AD80090474046BDE8F08110B500F033FA4FF476
:100AE800403400280EBF034C4FF4C07112F0DCFFF5
:100AF800204610BD0200030010B5044600F022FA9B
:100B080008B9054810BD0021A160D0F87C21116802
:100B180088474FF4403010BD0200030070B504460A
:100B28000D4600F00FFA064E40B1D0F87C0141683E
:100B38008847A84224BF65604FF44036304670BDF0
:100B4800020003002DE9FF4715000C4600D02CB128
:100B5800064600F0F7F95FEA000801D16448C3E0EF
:100B6800D8F8F80001684A689047B0F5003F17D1F7
:100B7800D8F87C118A68404690478146B9F1810FC0
:100B880080F09E80A94508F1FC0A17D2D8F8F80031
:100B98000368D3F80CC02A462146E047B0F5003F69
:100BA80040F08E80D8F8F8000368D3F810C06A4681
:100BB8005146E047B0F5003F76D10AE0002004E056
:100BC800215C0AF800100098401C00900098A84288
:100BD800F6D34FF0000C4749474A484B01AC009800
:100BE800844558D2D3E9007001ADC5E9007010788A
:100BF80000281ABF042086464FF0000E085854F803
:100C08000E5028443E4D05600127D0F800E087606B
:100C1800019D4F681AF80C007D408EEA050585F0A5
:100C2800040E65680F687D4085F0FC05754485F005
:100C3800A30568400AF80C000CF1010CCFE7D3E9D2
:100C4800004501A8C0E9004510782E4D002814BFC2
:100C58004FF0040E4FF0000E01A8744651F80EE054
:100C68000459A6440127CEF80050DEF80040CEF81B
:100C780008704D68019F40687D406C400D68684071
:100C880084F0040480F0FC00041984F057040AF886
:100C98000C400CF1010CCC45D1D3D8F8F800016810
:100CA8004A689047B0F5003F0AD1D8F8F8000368C1
:100CB800D3F80C804A465146C047B0F5003F01D0F2
:100CC800114811E0002006E05AF8201081F06A313E
:100CD8004AF82010401CB0EB990FF5D3B06840F0EB
:100CE8000100B0604FF4403004B0BDE8F08700BFA9
:100CF800020003004C3C0108E8080020240F00080B
:100D0800ADBE4ED70DBE75A10100030038B50C4627
:100D1800017A1546CA0702D500F014F908B908483F
:100D280032BDD0F8F80003682146DC682A46A0479F
:100D3800B0F5003F01D0034832BD4FF4403032BD1A
:100D480002000300010003002DE9F84191B00546B7
:100D58000E461746402101A812F0A6FE297AC807B8
:100D680004D5284600F0EEF8040002D1DFF8A4808C
:100D78004BE0D4F8F800DFF8A0800368D3F810C07F
:100D88006A4601A9E047B0F5003F3ED1D4F8F80023
:100D980001684A689047B0F5003F36D1D4F87C1115
:100DA8008A6820469047D4F8F830024618461B68EF
:100DB800D3F80CC004F1FC01E047B0F5003F24D1A2
:100DC800D4F87C0141688847D4F8F83002461846C0
:100DD8001B68D3F80CC001A9E047B0F5003F14D157
:100DE800D4F8F8000268696893689847B0F5003F3E
:100DF8000BD1D4F8F80003681C693A463146A0477D
:100E0800B0F5003F08BF4FF44038404612B0BDE887
:100E1800F08100BF02000300010003002DE9F84142
:100E2800A5B0074688461646402115A812F03CFE94
:100E380000220492402105A812F036FE387AC10734
:100E48005ED5384600F07EF8050059D0D5F8F80090
:100E58002D4C0368D3F810C06A4605A9E047B0F5E1
:100E6800003F3CD1D5F8F80001684A689047B0F5D2
:100E7800003F34D1D5F87C118A6828469047D5F8C8
:100E8800F830024618461B68D3F80CC005F1FC017F
:100E9800E047B0F5003F22D1D5F87C01416888478A
:100EA800D5F8F830024618461B68D3F80CC005A9D7
:100EB800E047B0F5003F12D1D5F8F800026879682C
:100EC80093689847B0F5003F09D1D5F8F800036852
:100ED8001D6904AA15A9A847B0F5003F01D020460E
:100EE8000FE00A4B0A490B4A0396029101924046C9
:100EF8001C68049B009415AA796800F0E5F900E0E5
:100F0800054826B0BDE8F08101000300543C010803
:100F1800936E030026C703000200030004B001011A
:100F280000170145E10A0008010B0008250B00081D
:100F3800B50300084D0B0008150D0008510D0008F9
:100F4800250E00080168024A914218BF0020704728
:100F58002C0F000810B5040008BF002404D0034873
:100F68002060204609688847204610BD2C0F0008DD
:100F780020225C3012F096BDF0B58468A3080022E8
:100F880004F0030407E000F15C0555F8226035BA67
:100F980041F82250521C9A42F5D300220BE000F18E
:100FA8005C0502EB830755F82360D500C5F11805E9
:100FB800EE40CE55521CA242F1D3F0BD30B5C46804
:100FC80003690022E31AD5188C5C0544521C082AD0
:100FD8002C77F8D330BD0360C1600261704738B523
:100FE800044615460022626023685A68904700202C
:100FF8006061A061A5604FF4003032BD81604FF49C
:10100800003070472DE9F84304462079D4F80C8065
:10101800450748BF244845D466691D46A8F1010024
:1010280000EAD60306EBC506B6EBC50F666102D229
:10103800A669761CA6611746A66906EB5576A661D1
:101048000E46E918884225D2A8EB03094A463146DC
:10105800F81812F027FD2268136839460FE0424657
:10106800384612F01FFD23681A6839462046904713
:1010780007E0311811F00300F1D122681368204607
:101088009847484600EB0809A9F10101A942F0D3A5
:10109800002300E000202A1A3118F81812F002FD87
:1010A8004FF40030BDE8F283040002002DE9FC4F44
:1010B800024685B0D0681369DFF86CC1DFF86C812F
:1010C800A0EB030A506840F004005060002703A812
:1010D80002900DF10C0ED8E9003403A8544DC0E974
:1010E80000342878534D00280CBF00230423994668
:1010F8005CF803305EF80940234401261D601C6833
:101108009E60DCF80430039DDCF80090DEF8046093
:101118005D406540484C654089EA0606474C664094
:101128007519474C6540D8E9006B03AC0028C4E941
:10113800006B0EBF002404200424029E5CF800000B
:10114800345920183F4C04600126046886600398CF
:10115800029E43406340384C7068634089EA00004F
:10116800364C6040034438484340280018BF0120EB
:101178005B1E9B41042F2CBFC0B2D80F02F1140391
:1011880053F8200007F00303C3F10303DB00D84042
:101198000DF807007F1C082F9DD315460C466A6979
:1011A800AB69E868D20842EA4372401E00EA0207C7
:1011B800002302409B420AD8524508D28020E055BD
:1011C8007F1C574516D2AAEB0701E01910E08020D2
:1011D800E05500E0E355E8687F1C8742FAD32A68A7
:1011E800136828469847BAF1000F03D051462046A5
:1011F80012F05AFC2A68069E059F9368694628469D
:1012080098472A68D2F8009021462846C8472B6894
:10121800DA683946284690470EB1A86830604FF41E
:10122800003007B0BDE8F08F4C3C010854120008AC
:10123800E80800205FC5109304850012FC68017A55
:10124800C0F524FF24AF33D426AF698B04B0010165
:1012580000170145F8B501240094002300240DE08F
:10126800009D065D0F5D7E40F643761CF60F86F006
:10127800010635400095641C009DEB189442EFD39D
:101288001846F2BDF8B5002301240094002A11E0A5
:10129800009C85188F1815F8016C17F8015C6E40D2
:1012A800F643761CF60F86F0010634400094009C45
:1012B800E318521EECD11846F2BD00005D1200087A
:1012C8008D120008010000002DE9F84F1D46DDF8D9
:1012D80028900B9F0D9C4FF0FF3300930E469246CB
:1012E800D9F800B0804632465146D847834664B3A1
:1012F800D9F8043032465146404698476FEA0B0207
:10130800521C42EA0B0200996FEAD2735B1C194027
:10131800C2430091521C024300996FEAD2735B1CCE
:101328001940009186F05531484087EA000181F064
:101338005531216080F05531C943491C0843009A52
:101348006FEAD070401C82430092D9F80800012847
:1013580009D17540E943491C0D4300986FEAD572DD
:10136800521C90430AE0F11C85EA9102D243521CB8
:10137800154300986FEAD5735B1C984386F0AA362C
:10138800009086EA0B0686F0AA33F243DB430C98FA
:10139800C2F3C0725B1C42EAD3720099D243521C5A
:1013A80091430091774000998843009987F0AA37C4
:1013B8000F403843BDE8F28F034613F8012B002A8B
:1013C800FBD1181A0138704781F0004102E000BFD4
:1013D80083F0004330B54FEA41044FEA430594EAED
:1013E800050F08BF90EA020F1FBF54EA000C55EA28
:1013F800020C7FEA645C7FEA655C00F0E2804FEAF9
:101408005454D4EB5555B8BF6D420CDD2C4480EADA
:10141800020281EA030382EA000083EA010180EA0A
:10142800020281EA0303362D88BF30BD11F0004F58
:101438004FEA01314FF4801C4CEA113102D040428E
:1014480061EB410113F0004F4FEA03334CEA1333C9
:1014580002D0524263EB430394EA050F00F0A780E1
:10146800A4F10104D5F1200E0DDB02FA0EFC22FADC
:1014780005F2801841F1000103FA0EF2801843FAD0
:1014880005F359410EE0A5F120050EF1200E012AC1
:1014980003FA0EFC28BF4CF0020C43FA05F3C018FF
:1014A80051EBE37101F0004507D54FF0000EDCF178
:1014B800000C7EEB00006EEB0101B1F5801F1BD321
:1014C800B1F5001F0CD349085FEA30004FEA3C0C25
:1014D80004F101044FEA445212F5800F80F09A801B
:1014E800BCF1004F08BF5FEA500C50F1000041EB1F
:1014F800045141EA050130BD5FEA4C0C404141EB23
:101508000101013C28BFB1F5801FE9D291F0000F1D
:1015180004BF01460020B1FA81F308BF2033A3F1CC
:101528000B03B3F120020CDA0C3208DD02F1140CC3
:10153800C2F10C0201FA0CF021FA02F10CE002F1FE
:101548001402D8BFC2F1200C01FA02F120FA0CFCF7
:10155800DCBF41EA0C019040E41AA2BF01EB045140
:10156800294330BD6FEA04041F3C1CDA0C340EDC3E
:1015780004F11404C4F1200220FA04F001FA02F381
:1015880040EA030021FA04F345EA030130BDC4F13F
:101598000C04C4F1200220FA02F001FA04F340EA34
:1015A8000300294630BD21FA04F0294630BD94F0E5
:1015B800000F83F4801306BF81F480110134013DCC
:1015C8004EE77FEA645C18BF7FEA655C29D094EA3D
:1015D800050F08BF90EA020F05D054EA000C04BFBB
:1015E8001946104630BD91EA030F1EBF00210020A6
:1015F80030BD5FEA545C05D14000494128BF41F045
:10160800004130BD14F580043CBF01F5801130BDA8
:1016180001F0004545F0FE4141F470014FF0000033
:1016280030BD7FEA645C1ABF194610467FEA655CE4
:101638001CBF0B46024650EA013406BF52EA033586
:1016480091EA030F41F4002130BD00BF90F0000F74
:1016580004BF0021704730B54FF4806404F13204B0
:101668004FF000054FF0000150E700BF90F0000F69
:1016780004BF0021704730B54FF4806404F1320490
:1016880010F0004548BF40424FF000013EE700BF60
:1016980042004FEAE2014FEA31014FEA02701FBFF0
:1016A80012F07F4393F07F4F81F06051704732F022
:1016B8007F4208BF704793F07F4F04BF41F4002179
:1016C800704730B54FF4607401F0004521F00041D7
:1016D8001CE700BF50EA010208BF704730B54FF061
:1016E80000050AE050EA010208BF704730B511F062
:1016F800004502D5404261EB41014FF4806404F19A
:1017080032045FEA915C3FF4D8AE4FF003025FEA1F
:10171800DC0C18BF03325FEADC0C18BF033202EBA3
:10172800DC02C2F1200300FA03FC20FA02F001FAFD
:1017380003FE40EA0E0021FA02F11444BDE600BFA0
:101748004FF0FF3C06E000BF4FF0010C02E000BF85
:101758004FF0010C4DF804CD4FEA410C7FEA6C5C68
:101768004FEA430C18BF7FEA6C5C1BD001B050EA0B
:10177800410C0CBF52EA430C91EA030F02BF90EAF6
:10178800020F0020704710F1000F91EA030F58BFB5
:10179800994208BF90422CBFD8176FEAE37040F017
:1017A800010070474FEA410C7FEA6C5C02D150EAB5
:1017B800013C07D14FEA430C7FEA6C5CD6D152EA70
:1017C800033CD3D05DF8040B704700BF8446104635
:1017D80062468C461946634600E000BF01B5FFF734
:1017E800B7FF002848BF10F1000F01BD4DF808ED04
:1017F800FFF7F4FF0CBF012000205DF808FB00BFD5
:101808004DF808EDFFF7EAFF34BF012000205DF82E
:1018180008FB00BF4DF808EDFFF7E0FF94BF01207B
:1018280000205DF808FB00BF4DF808EDFFF7CEFF7C
:1018380094BF012000205DF808FB00BF4DF808EDBB
:10184800FFF7C4FF34BF012000205DF808FB00BF8C
:101858004FEA410212F5001215D211D56FF47873D0
:10186800B3EB625212D94FEAC12343F0004343EA73
:10187800505311F0004F23FA02F018BF404270474E
:101888004FF00000704750EA013005D111F00040D8
:1018980008BF6FF0004070474FF00000704700BF6E
:1018A80080F0004002E000BF81F0004142001FBF0D
:1018B8005FEA410392EA030F7FEA226C7FEA236C16
:1018C8006AD04FEA1262D2EB1363C1BFD21841400B
:1018D80048404140B8BF5B42192B88BF704710F0A1
:1018E800004F40F4000020F07F4018BF404211F044
:1018F800004F41F4000121F07F4118BF494292EAAC
:10190800030F3FD0A2F1010241FA03FC10EB0C00D7
:10191800C3F1200301FA03F100F0004302D5494264
:1019280060EB4000B0F5000F13D3B0F1807F06D311
:1019380040084FEA310102F10102FE2A51D2B1F109
:10194800004F40EBC25008BF20F0010040EA0300FE
:101958007047490040EB0000013A28BFB0F5000F7E
:10196800EDD2B0FA80FCACF1080CB2EB0C0200FA34
:101978000CF0AABF00EBC25052421843BCBFD04083
:101988001843704792F0000F81F4000106BF80F4FD
:1019980000000132013BB5E74FEA41037FEA226CC0
:1019A80018BF7FEA236C21D092EA030F04D092F08B
:1019B800000F08BF0846704790EA010F1CBF0020BF
:1019C800704712F07F4F04D1400028BF40F000401C
:1019D800704712F100723CBF00F50000704700F03C
:1019E800004343F0FE4040F4000070477FEA226263
:1019F80016BF08467FEA23630146420206BF5FEA34
:101A0800412390EA010F40F4800070474FF0000333
:101A180004E000BF10F0004348BF40425FEA000CFA
:101A280008BF704743F0964301464FF000001CE0A2
:101A380050EA010208BF70474FF000030AE000BFF8
:101A480050EA010208BF704711F0004302D5404236
:101A580061EB41015FEA010C02BF844601460020A8
:101A680043F0B64308BFA3F18053A3F50003BCFAC3
:101A78008CF2083AA3EBC25310DB01FA02FC634470
:101A880000FA02FCC2F12002BCF1004F20FA02F277
:101A980043EB020008BF20F00100704702F120026A
:101AA80001FA02FCC2F1200250EA4C0021FA02F2CB
:101AB80043EB020008BF20EADC7070474FEA40029F
:101AC800B2F1FE4F0FD34FF09E03B3EB12620DD964
:101AD8004FEA002343F0004310F0004F23FA02F0CE
:101AE80018BF404270474FF00000704712F1610F75
:101AF80001D1420205D110F0004008BF6FF000404C
:101B080070474FF00000704753B94AB9002908BF21
:101B180000281CBF4FF0FF314FF0FF3000F070B9C4
:101B2800ADF1080C6DE904CE00F006F8DDF804E02C
:101B3800DDE9022304B070472DE9F047089E0D4601
:101B480004460F46002B4AD18A42944665D9B2FA18
:101B580082F343B102FA03FCC3F120029F4020FA4A
:101B680002F217439C404FEA1C4E1FFA8CF5B7FB54
:101B7800FEF1220C0EFB117742EA074201FB05F049
:101B880090420AD91CEB020201F1FF3780F01B8159
:101B9800904240F2188102396244121AA4B2B2FB90
:101BA800FEF00EFB102244EA024400FB05F5A542B4
:101BB8000AD91CEB040400F1FF3280F00681A5422B
:101BC80040F203816444023840EA0140641B00216A
:101BD8001EB1DC400023C6E90043BDE8F0878B4214
:101BE80008D9002E00F0EC800021C6E9000508465F
:101BF800BDE8F087B3FA83F1002949D1AB4202D39B
:101C0800824200F2F780841A65EB0302012017462E
:101C1800002EE2D0C6E90047DFE702B9FFDEB2FADC
:101C280082F3002B40F08F808A1A4FEA1C471FFA74
:101C38008CFE0121B2FBF7F507FB1520220C42EAC6
:101C480000420EFB05F0904208D91CEB020205F198
:101C5800FF3802D2904200F2CA804546121AA4B256
:101C6800B2FBF7F007FB102244EA02440EFB00FE29
:101C7800A64508D91CEB040400F1FF3202D2A645A0
:101C880000F2BA801046A4EB0E0440EA05409FE734
:101C9800C1F120078B4022FA07FC4CEA030C05FA35
:101CA80001F420FA07F3FD40234300FA01F94FEA53
:101CB8001C401FFA8CFEB5FBF0F81C0C00FB1855F5
:101CC80044EA054408FB0EF5A54202FA01F20BD9D5
:101CD8001CEB040408F1FF3A80F08780A54240F22B
:101CE8008480A8F102086444641B9DB2B4FBF0F33D
:101CF80000FB134445EA044403FB0EFEA64508D93D
:101D08001CEB040403F1FF306BD2A64569D9023BF2
:101D1800644443EA0840A0FB0283A4EB0E049C42FF
:101D2800C6461D4655D352D056B1B9EB0E0364EBE7
:101D3800050404FA07F7CB40CC401F43C6E90074FA
:101D48000021BDE8F087C3F1200102FA03FC20FA64
:101D580001F225FA01F19D402A434FEA1C471FFA78
:101D68008CFEB1FBF7F007FB1015110C41EA054199
:101D780000FB0EF58D4204FA03F408D91CEB0101AF
:101D880000F1FF382FD28D422DD902386144491B0A
:101D980092B2B1FBF7F507FB151142EA014205FBC8
:101DA8000EF1914208D91CEB020205F1FF3816D258
:101DB800914214D9023D6244521A45EA004139E77A
:101DC8003146304609E73946E7E61046FCE6C145A4
:101DD800AAD2B8EB020E63EB0C050138A4E745461E
:101DE800EAE7034695E74046D1E7D0467CE7023D5F
:101DF800624433E708460BE76444023843E700BF10
:101E0800704700BF1348144A08B54FF00043C0E9B3
:101E180000230422002342610122C2614FF4805151
:101E280007220383C0E90233C0E90933C0E90C1271
:101E38000361837680F8203080F82C30826380F844
:101E48003C30C36404F014FF18B1BDE8084000F04A
:101E58000DBC08BDEC080020002401400268084BB6
:101E68009A4282B00AD14FF0B0431A6E42F400721F
:101E78001A661B6E03F400730193019B02B070474E
:101E8800002401400268054B9A4201BF4FF0B0425E
:101E9800136E23F400731366704700BF00240140DB
:101EA80030B585B000240546CDE901440394FFF719
:101EB800A9FF144805F074FA08B100F0D7FB1148DF
:101EC800039401A9CDE9015405F030F808B100F0F8
:101ED800CDFB0C4805F08EF908B100F0C7FB4FF0B8
:101EE800FF31084804F0C4FF064805F03BFA0548EE
:101EF80005F018F80446034805F0DEF9204605B059
:101F080030BD00BFEC080020014B024A1A60704740
:101F1800EC0800200024014008B50948FFF7C0FF7D
:101F280068B1084BB3F8AA304FF6FF72934216BF58
:101F380040F6E442044B5343B3FBF0F398B208BDB8
:101F4800002000B40075FF1FD8084C0013B500230B
:101F5800ADF80630FFF7E0FF04461948FFF7A0FF89
:101F6800184BB3F8C820B3F8A8108A4204FB00F055
:101F780018D040F6E443B0FBF3F364205B1A434304
:101F8800521A93FBF2F31E331BB2ADF80630BDF8BC
:101F980006305BB21B02ADF80630BDF8060000B291
:101FA80002B010BD4FF47A7240F6FF73B0FBF3F342
:101FB8005343A3F53923A3F50C6340F6C412E0E7B5
:101FC800001000B00075FF1F4FF0B04382B09A6A4E
:101FD80022F480529A629A6C42F480529A649B6C02
:101FE80003F480530193019B002002B070474FF027
:101FF800B04382B09A6C02439A649B6C034001938D
:10200800019B02B0704708B50420FFF7F0FF0120DC
:10201800FFF7EDFF0220FFF7EAFF002211460B2031
:1020280005F05CFA0B2005F08BFA002211460C2013
:1020380005F054FA0C2005F083FA002211460D2011
:1020480005F04CFA0D2005F07BFA002211460E200F
:1020580005F044FA0E2005F073FA002211460F200D
:1020680005F03CFA0F2005F06BFA0022114610200B
:1020780005F034FA102005F063FA00221146112009
:1020880005F02CFA112005F05BFA002236201146E3
:1020980005F024FABDE80840362005F051BA0000E2
:1020A80008B505F095FC10B16FF0040008BD064BAB
:1020B8009A6942F040429A614CF2FA321A6105F08C
:1020C80099FC0028F2D0EFE700400058F0B585B041
:1020D80000230C4600930646A8B3FFF7E1FF054628
:1020E80070BB05F075FC88BB1A481B4A0223019394
:1020F800D0F8E01506F1784302EA8121B3FBF1F745
:1021080001FB1733DB0A0293D0F8E00504F17841AC
:102118000139314402EA8022B1FBF2F002FB1011CE
:10212800C3EBD1230133694601A8039305F0E2FC10
:1021380020B102280CBF01256FF0010505F05AFCFB
:10214800284605B0F0BD6FF00505F9E76FF0040506
:10215800F6E700BF0070FF1F00FCFF03014B18608B
:1021680000207047500900202DE9F04F89B0B0F1E8
:10217800006F06460F460092C0F0C580DFF89881D0
:10218800664DD8F8E03505EA832303F10063013B87
:10219800984200F2B880002800F0B880002900F0CA
:1021A800B58040EA02035B0740F0B080FFF778FF94
:1021B8000446A0BB05F00CFC002840F0AA80D8F823
:1021C800E01506F1784205EA8121B2FBF1F301FB43
:1021D8001322009B03F17843013B3344B3FBF1F036
:1021E80001FB1033DB0A01334FEAD22AA3EBD222D8
:1021F800012A039388BFC6F30A050AF58038C6F199
:10220800080398BF009D069388BFC5F500654FEA8F
:10221800C828B346039B9A4505D305F0EBFB204637
:1022280009B0BDE8F08FA6F10803069A1A44954252
:1022380019D804950197CDF814B04FF00009059B03
:1022480009EB0301049B99453ED3009BAB442F4403
:102258005D1BB5F5006F28BF4FF400650AF1010A50
:1022680008F50068D6E753F8081F5A68B2F1FF3F2F
:1022780008BFB1F1FF3FD8D0294B186810B96FF0EB
:102288000504CAE7B8F1000F04D04FF400624146D4
:1022980010F09CFFDFF88890D9F80030CBF30A00E3
:1022A80039461844AAB210F091FF4FF40061404635
:1022B800FFF70CFF08BBD9F8003001934FF4006317
:1022C800CDF814800493B8E7019B07914B4402931F
:1022D8000120D3E9002305F0C7FB88B90799019BC2
:1022E800D1E9000259F80310029B5B689A4208BFC3
:1022F800884205D109F10809A1E76FF001048CE7CC
:102308006FF0030489E74FF0FF3488E76FF00504A6
:1023180085E76FF0040482E70070FF1F00FCFF03ED
:1023280050090020B1F1006F70B511D30B4BD3F8F1
:10233800E0650B4B03EA862303F10063013B9942F6
:1023480006D840B139B192B210F040FF002070BDFC
:102358004FF0FF30FBE76FF00500F8E70070FF1F54
:1023680000FCFF03B0F1006F10B40DD3084BD3F895
:10237800E045084B03EA842303F10063013B9842DC
:1023880002D810BCFFF7A2BE4FF0FF3010BC704758
:102398000070FF1F00FCFF034FF0B04382B0DA6CFF
:1023A8000243DA64DB6C03400193019B02B070477F
:1023B80070B5012086B00024CDE90444FFF7ECFF96
:1023C8000220FFF7E9FF0420FFF7E6FF01250DEBE8
:1023D800000102234FF404164FF09040CDE9013676
:1023E800039505F0D5FB4FF4441301A94FF0904035
:1023F800CDE90235019505F0CBFB2023CDE9013667
:10240800194E039401A9304605F0C2FB082301A91F
:102418003046CDE90135CDE9035405F0B9FB042375
:102428000DEB03013046CDE90135CDE9034405F054
:10243800AFFB22462146062005F050F8062005F09D
:102448007FF822462146072005F048F8072005F0C6
:1024580077F822462146162005F040F8162005F0A8
:102468006FF806B070BD00BF0004004808B51248F8
:10247800124A134BC0E9002300230122C0E90232AB
:10248800C0E90433C0E90633036205F01BFE08B156
:1024980000F0ECF80848002105F094FF08B100F0BE
:1024A800E5F80548002105F0B3FF18B1BDE808407C
:1024B80000F0DCB808BD00BF140A00200058004036
:1024C8005D3E302070B596B005461422002103A861
:1024D80011F0B4FA3822002108A811F0AFFA2A68DE
:1024E800304B9A425BD18023089308A84FF44023CD
:1024F8000E9306F0E9FC08B100F0B8F84FF0B044CC
:102508004FF4C050E36C43F00103E364E36C03F061
:1025180001030293029B12230026CDE90303032340
:10252800CDE905634FF09040042303A9079305F014
:102538002FFBA36DDFF870C043F48003A365A36D80
:102548001A4C03F480030193019B26620D23C4E90E
:1025580000C320468023C4E90266C4E90436C4E9FE
:10256800066605F04DF808B100F080F8104AEC63F3
:10257800A562104C0E23C4E90023102100238022F9
:102588002046C4E90213C4E90423C4E906332362DC
:1025980005F036F808B100F069F8AC63A56216B02A
:1025A80070BD00BF0058004044000240540900209C
:1025B80058000240B409002000B59BB04822002111
:1025C80008A811F03BFA1822002102A811F036FAE7
:1025D80005F044FF4FF0B0420120D2F8903023F0CC
:1025E8001803C2F89030D2F8003423F4C06343F4DF
:1025F8000073C2F80034D2F8003403F4C0630193C6
:10260800019B2423089381230B930023CDE9100316
:10261800B02208A8CDE9122306F098F808B172B6DE
:10262800FEE74F23CDE90230CDE90400CDE90600ED
:10263800022102A806F024FB08B172B6FEE71BB01F
:102648005DF804FB08B504F0C1FAFFF7B5FFFFF722
:10265800AFFEFFF7D8FCFFF709FF00F08CFD40F64E
:10266800B83000F03FFA00F08DFDFCE772B6FEE7E7
:1026780000B58DB02C22002101A811F0DFF9174810
:10268800174B03601F2383604FF080420023C0E98B
:102698000433C0E9072383614FF48073436206F073
:1026A80099FD08B1FFF7E2FF0C4806F0BFFE08B13C
:1026B800FFF7DCFF4FF0005300220793074808920A
:1026C8004FF4807301A9029206920B9306F0E2FD83
:1026D80008B1FFF7CBFF0DB05DF804FB680A0020D6
:1026E8000028004010B5044690B03822002102A806
:1026F80011F0A4F92268194B9A422CD14FF4803377
:10270800029302A84FF480730F9306F0DDFB08B123
:10271800FFF7ACFF4FF0B0430220D3F8902042F40B
:102728000042C3F890209A6D42F480629A659B6DCE
:10273800002203F4806311460193019B04F0CEFE4E
:10274800022004F0FDFE00222A20114604F0C6FEF5
:102758002A2004F0F5FE10B010BD00BF002800408C
:102768007047000008B504F047FA044B0120C3F88D
:102778008800BDE8084005F0C9BE00BF0004005845
:1027880004F041BA08B504F03EFA00F059FCFFF72E
:102798000FFEFFF738FCBDE80840FFF767BE08B535
:1027A80004F02AFABDE808400121002005F05EBEC9
:1027B80070477047FEE7FEE7FEE7FEE7FEE7704773
:1027C8007047704770470000014806F055BE00BFCB
:1027D800680A0020012005F007BB022005F004BBB1
:1027E80070477047014805F085B800BF54090020BC
:1027F800014805F07FB800BF400B0020014805F0F4
:1028080079B800BFE00A0020FFF7F2BF7047202028
:1028180005F0EABA70470000014807F0F1B900BFB7
:10282800A00B0020014806F059BC00BF680A002030
:10283800014807F04CB800BFCC0A00202DE9F0434E
:1028480089B080460020109E0790894615461F468D
:10285800FDF7E6FCF0B9104CCDE90090CDE9020493
:1028680007AB0E480593142304933A46434629467A
:102878000068FDF79FFD2346324604F1140153F822
:10288800044B42F8044B8B42F9D1079B337509B0CE
:10289800BDE8F0830120FAE7A00A0020483C0108BF
:1028A8001FB50E4C00233C2202A8CDE90233627505
:1028B800237500F0B9F8042303AA009412210848EC
:1028C800FFF7BCFF07491422204611F0A7F8B0FA19
:1028D80080F35B09637504B010BD00BFB40A002023
:1028E800703C01084E0E0020054808B50823036017
:1028F80006F008FE18B1BDE80840FFF7B7BE08BDEE
:10290800CC0A00204FF0B04307B55A6E42F00102DE
:102918005A665B6E002203F00103019311463220D0
:10292800019B04F0DBFD322003B05DF804EB04F0FA
:1029380007BE00000CB407B5054A05AB102101938A
:1029480010F04EFF03B05DF804EB02B0704700BF13
:10295800823C010830B585B0044602A80D4610F047
:102968006BFDBDF90C30064A00931021029B2046EE
:10297800FFF7E0FF2046FEF71FFD288005B030BDB9
:10298800823C01084FF0B04210B5936823F400432D
:10299800936010F0D9FD0E4B01241C7000F0B6F8BE
:1029A80010F0A2FA0B4810F0B9FA0B4B4FF40042A2
:1029B8001A61204610F0B8FAFFF7A6FA00F012F9EB
:1029C80010F0AEFB21462046BDE8104010F0C8BB11
:1029D800D80A00205D2900080040005810F0D6BB36
:1029E80008B5FFF799FA40F6B83398420CD8B0F515
:1029F800E16F0BD3FE23A0F5E16058434FF49663D3
:102A0800B0FBF3F0C0B208BDFE20FCE70020FAE7F7
:102A18007FB5684600F0CAF80198FFF74FF800B292
:102A280007B05DF804FB0000194A38B5D2F88035C4
:102A3800591C044619D104F0EDF8054604F0F6F8DF
:102A4800054404F0EDF82B0EE3712B0CA3712B0A4F
:102A58006371030EE370C0F30742C0F307232571C7
:102A6800C0B2A2706370207038BD190AC371817139
:102A7800190C1B0E41710371D2F88435C370D2F85A
:102A88008405C0F30722C0F30743000EE9E700BF3F
:102A98000070FF1F38B5094BD3F880350360013348
:102AA800054609D104F0B6F8044604F0B9F84440E4
:102AB80004F0BCF844402C6038BD00BF0070FF1F14
:102AC8000121022010F036BB0021022010F032BB99
:102AD80000207047024B187808B100F0BBB8704767
:102AE800D80A002082B00190019802B000F04EB9D7
:102AF8004FF0B04382B0DA6C42F00202DA64DB6C69
:102B080003F002030193019B02B070472DE9F043E3
:102B1800254C87B004F090F804F096F804F09CF87F
:102B28000123002502934FF48059032301A920466D
:102B380004934FF4005803950595FFF7D9FFFFF765
:102B4800D7FFFFF7D5FFFFF7D3FFCDF8049005F0C7
:102B58001FF801A920464FF40067CDF8048005F05E
:102B680017F801A920464FF40046019705F010F820
:102B780001A92046019605F00BF82A464946204649
:102B880005F02CF92A464146204605F027F92A4641
:102B98003946204605F022F92A463146204605F0F6
:102BA8001DF907B0BDE8F0830004004810B50446DD
:102BB800FFF7CCF9074BA36040F30F20FEF72AFF7D
:102BC800054B064A2360064B6060C4E903230020D6
:102BD80010BD00BF0000484200007A440D093E00C5
:102BE800AB03050000207047014B1868704700BF11
:102BF800DC0A00200320704708B501464FF47A72BA
:102C080000238002890DFEF77FFF08BD4FF47A7319
:102C1800A0FB0303800A40EA83507047034B98687F
:102C28009A689042FBD1C043704700BF002800401B
:102C380008B5FFF7F3FF014B186008BDDC0A002058
:102C480008B5FFF7EBFF024B1B68C01A08BD00BFB1
:102C5800DC0A0020024B187808B1FFF7DFBF704785
:102C6800D90A002010B5074B074C0122DA654FF44A
:102C78008071204606F0F8F94FF0FF3323630020F7
:102C880010BD00BF00280040680A0020024600214D
:102C9800014806F002BC00BF680A00200246012174
:102CA800014806F0FABB00BF680A002010B58CB0D6
:102CB8002C220021044601A810F0C0FEFFF7D2FF25
:102CC8000C4B0D481B681C440023089306934FF0D7
:102CD8000053E443079301224FF4807301A902943F
:102CE8000B9306F0D7FA08B1FFF7C0FC00200CB030
:102CF80010BD00BFDC0A0020680A002038B5054670
:102D0800FFF78CFF02210446074806F0CDFBC4F309
:102D180009024FF47A71A2FB0121920AA30A2A80C0
:102D280043EA805038BD00BF680A002001480021EE
:102D380006F0BABB680A00200148012106F0B4BBBE
:102D4800680A0020F8B50F4D2E78CEB90E4C4FF01A
:102D5800FF372763FFF78CFCFFF784FF4FF4807180
:102D6800204606F081F92046276306F041FB3246EB
:102D78002046022106F091FBFFF75AFF01232B7032
:102D88000020F8BDD90A0020680A0020014610B5C5
:102D98004FF47A7200238002890DFEF7B5FE0146D2
:102DA800FFF73CFF0446FFF739FF031B8B4200D3B4
:102DB80010BD00BFF7E710F0CFBC000010B5064CFF
:102DC8000221204606F070FB0221421C2046BDE885
:102DD800104006F062BB00BF680A00201648174A78
:102DE80008B54FF4E133C0E9002300230C22C0E901
:102DF8000233C0E90523C0E90733C0E90933036199
:102E080007F0DFFC08B1FFF731FC0B48002107F0A1
:102E180054FE08B1FFF72AFC0748002107F06DFEB1
:102E280008B1FFF723FC044807F027FE18B1BDE8F6
:102E38000840FFF71BBC08BDA00B00200044004061
:102E480070B596B005461422002103A810F0F6FDCF
:102E58003822002108A810F0F1FD2A68334B9A4265
:102E680061D10223089308A8314B0A9306F02CF885
:102E780008B1FFF7FBFB4FF0B0430C219A6D2D4CC6
:102E880042F400329A659A6D02F400320292029A74
:102E9800DA6C42F00102DA64DB6C03F0010301939F
:102EA800019B02230026CDE903130323CDE9056323
:102EB8004FF09040072303A9079304F069FE1E48CA
:102EC80026621423C4E900031023C4E9023620460D
:102ED8008023C4E90436C4E9066604F091FB08B10E
:102EE800FFF7C4FB154AEC67A562154C1323C4E928
:102EF8000023204600238022C4E90233C4E90423C6
:102F0800C4E90633236204F07BFB08B1FFF7AEFB8C
:102F18002520C5F8804000220221A56204F0DEFACF
:102F2800252004F00DFB16B070BD00BF0044004022
:102F380004000C00400B0020800002406C0002409E
:102F4800E00A002002680E4B9A4210B5044616D1DA
:102F58004FF0B0420C21936D23F4003393654FF08A
:102F6800904004F0C1FEE06F04F0BEFBD4F880008E
:102F780004F0BAFBBDE81040252004F0EFBA10BDFC
:102F88000044004008B50A460146024806F09CFD88
:102F9800002008BDA00B002013B5114B114C186080
:102FA8004FF40013009302AB13E90600204607F024
:102FB80008FD2368DA69D103FCD4DA695202FCD52A
:102FC8009A68084842F480029A6007F040FD064972
:102FD8000448012207F0AEFC002002B010BD00BF7B
:102FE800340C0020A00B00203C0C002008B5074B37
:102FF8001860FFF708F8FFF7F1FE054AD2F88030AD
:1030080043F00063C2F88030002008BD380C00206F
:103018000008005808B54FF0B04308489A6B42F4CE
:1030280000329A639A6B22F400329A63FFF78AFFA0
:103038000F2004F093FA002008BD00BFA00B002069
:1030480008B5074807F0BDFB08B1FFF70FFB0548B7
:1030580004F0D6FA18B1BDE80840FFF707BB08BD71
:10306800A00B0020400B00200268044B9A4203D1B9
:10307800034B00201B681847704700BF00440040FE
:10308800380C002002680B4B9A4210B504460FD149
:10309800094B1B682BB1D0F8902012B907480121C1
:1030A800984720460549BDE81040012207F042BC78
:1030B80010BD00BF00440040340C00203C0C002030
:1030C80010B5084C237863B1FFF7EAFB0038064BCC
:1030D80018BF0120400018701B78022B04BF002382
:1030E800237010BD4E0E0020440C002038B5104D42
:1030F8002B78DBB90F4C2368012B07D92368042BE5
:1031080004D80D4A0421012000F0ECF92368042BAF
:103118000CD9FFF7C5FB0038084B18BF0120400049
:1031280018701B78022B04BF00232B7038BD00BF1A
:103138004E0E0020400C0020DC3C0108440C00200E
:1031480001F0B2B970477047022808B50ED80122BD
:103158001021074804F042FE3220FFF7C3FCBDE807
:10316800084003480022102104F038BE08BD00BF03
:1031780000040048704708B5FFF704FCBDE80840A4
:1031880000F044BB4FF0FF3010F064B87047704750
:1031980070470000014BD870704700BF5C000020EA
:1031A800014B1874704700BF5C00002020B1037801
:1031B80013B1024810F07EBA704700BF840D00209A
:1031C80008B50220002110F00DF8BDE808400148BC
:1031D80010F070BA9C0D00200021012010F002B8F8
:1031E80010B5094C60B12060084810F015FA216844
:1031F800064810F099FABDE81040044810F05ABA91
:1032080042F210732360EFE7740000209C0D002049
:1032180010B5094C206023680BB9084B2360084897
:1032280010F0FAF92168064810F07EFABDE810405F
:10323800034810F03FBA00BF0C000020A086010030
:10324800B40D002038B504460D4607484FF4006118
:10325800FFF788F830B92A4621460348BDE83840C8
:10326800FEF782BF38BD00BF00F003080A460149D7
:10327800FFF758B800F0030838B50C4810F0CCF93F
:1032880008F094F860B90A4C0A480125257007F03F
:1032980031FF2078294607F05BFD044810F00AFA50
:1032A800BDE83840044810F005BA00BF9C0D002066
:1032B800000000205C0000206C0D002008F014B90C
:1032C80030B58BB0FFF78CFB0446FEF725FE0021D6
:1032D80005464FF480700FF085FF684600F0C6FF82
:1032E80020B200EB4000FE2300EB4010B0FBF3F0EF
:1032F8008DF80C0004A8ADF80250FFF757FC2B4BD3
:103308000B221A702A4A1178002937D0002111702F
:103318000C2228491A705A68097811705A689DF861
:103328000C10517002222449244C0978012988BFC5
:1033380000225A70637A33B107F0ACFC012802D13D
:10334800204610F069F91E4B1848D978002207F07A
:103358008DFD063027D107F097FC0446194810F078
:103368005BF9194B17481968A14238BF214610F07C
:10337800DBF9144810F09EF90BB030BD134914481E
:103388000A7822B9047804F0FF02002CCBD000227E
:1033980002700A70BDF808205968120A0A705A6843
:1033A800BDF80810BDE70024D8E700BF04000020DE
:1033B800CC0D0020370D0020440C0020380D0020D3
:1033C8005C0000209C0D002074000020630E00208B
:1033D8004D0E002008B50F4B0122002102201A7063
:1033E8000FF000FF0C4810F065F90C4B1B787BB10F
:1033F8000B4B1B7863B90B4B1A68042A9EBF1A68DB
:1034080001321A600021BDE8084010200FF0EABE22
:1034180008BD00BFCC0D0020B40D0020680D0020B1
:103428004E0E0020400C0020044B1B78022B03D1C9
:10343800002108200FF0D6BE704700BF0000002012
:1034480008B507F0BCFF80B907F024FC01280CD1AF
:10345800BFF34F8F0549064BCA6802F4E062134375
:10346800CB60BFF34F8F00BFFDE708BD00ED00E064
:103478000400FA0510B5044640B190F906302BB99E
:10348800034810F0C9F8034BE2791A7010BD00BF69
:10349800380D0020680D002070477047704770474E
:1034A800022808B5014611D0202812D0012813D1CE
:1034B8000A4B18704FF0904004F08AFC01280BD199
:1034C80000210220BDE808400FF08CBE0021082032
:1034D800F8E7034B01221A7008BD00BF4D0E00200B
:1034E800C80E002070B505460C46164607F0A0FC2D
:1034F8000346002834D000241A4810F08DF81A4BDF
:1035080018481968A14238BF214610F00DF9BDE8E6
:103518007040144810F0CEB84A68F05CD0540133BB
:10352800DAB29442F8D8114B0D701B78012B88BF82
:1035380000244C700E4C637A33B107F0ABFB0128C2
:1035480002D1204610F068F80A4B0B48D9780022BF
:1035580007F08CFC0630CED107F096FB0446CBE78B
:103568000549DDE79C0D002074000020440C002074
:10357800380D00205C00002004000020044B1B785C
:1035880023B9044A05210120FFF7ACBF704700BFEB
:10359800440C0020E13C010810B5002490B03C2206
:1035A800214601A8009410F049FA2C4B2022DA7227
:1035B80019788DF8001059788DF8011099788DF8E0
:1035C8000210D9788DF8031019798DF804105979FB
:1035D8008DF8051099798DF80610D9798DF80710AE
:1035E800197A8DF80810597A8DF80910997A8DF89A
:1035F8000A108DF80B2021460DF10B0258180131E5
:10360800007B02F8010F1C29F8D193F828208DF8C7
:10361800282093F829208DF8292093F82A208DF85E
:103628002A2093F82B208DF82B200DF12B01002256
:103638009818013290F82C0001F8010F142AF7D1DC
:1036480007484FF40061FEF78DFE20B90448402278
:103658006946FEF789FD10B010BD00BF7800002054
:1036680000F80308014940220FF0B0BD00F8030834
:1036780038B5254C207963794D2BC0B231D1C0EBD8
:10368800001080000A284FF47A7338BF0A20584384
:103698001E4D1F4B18602B785BB3FFF7A1FDA07977
:1036A800E3794D2BC0B227D1C0EB00108000012870
:1036B8004FF47A7338BF01205843FFF7A9FD237AE6
:1036C800144ADBB21370637A134ADBB21370002317
:1036D800E21892F82C20D2B2EA540133142BF7D115
:1036E80038BD6379482B0ABF4FF461636379584347
:1036F800C8E742F21070D0E7E379482B0ABF4FF4CD
:103708006163E3795843D2E7780000204E0E002029
:1037180074000020620E0020440C002010B590B008
:1037280000213C2201A8009110F088F94022344978
:1037380068460FF04BFD9DF800203AB99DF801004E
:10374800102803D19DF8021001290ED0FFF724FF9D
:103758002C48142200210FF043FD4FF47A70FFF734
:10376800C1F9FFF785FF10B010BD274B1A705870CC
:1037780099709DF80310D9709DF8041019719DF87F
:10378800051059719DF8061099719DF80710D971A7
:103798009DF8081019729DF8091059729DF80A10C1
:1037A80099729DF80B1001F03F01D972D87AD1B205
:1037B80088421BD89DF8282083F828209DF82920C6
:1037C80083F829209DF82A2083F82A209DF82B20A9
:1037D80083F82B200DF12B0100229818013211F8E3
:1037E800014F80F82C40142AF7D1BAE701F14000C4
:1037F8006844194410F8340C08730132D6E700BF46
:1038080000F803084E0E0020780000201FB50024A1
:1038180003A92046039407F0B5FD03A9012007F08A
:10382800B1FD384B3848009422464FF4FA710FF036
:1038380095FE364B3648009422464FF4FA710FF045
:103848008DFE344B3448009401224FF4FA710FF086
:1038580085FE2046FEF782FC08B1FEF707FF2F4BD6
:10386800009400224FF4FA612D480FF077FE2D4A9C
:10387800002101200FF072FD2B4A002102200FF0D9
:103888006DFD2A4A002104200FF068FD284A002116
:1038980008200FF063FD00F06BFB2649264807F06F
:1038A80033FD264807F026FC1B480FF003FF244B86
:1038B8000021187807F04CFA22490094224B096835
:1038C800224800220FF04AFE20480FF0F3FEFFF7CF
:1038D80025FF1F4A002110200FF040FD1D4A00213E
:1038E8004FF480700FF03AFD1B4B1C4819681C4BB5
:1038F800009400220FF032FE18480FF0DBFE04B0EF
:1039080010BD00BFA5340008840D0020A7340008AE
:10391800500D0020A1340008380D00203134000873
:103928006C0D002055AC0008C9320008C5320008EB
:103938008132000800000301100000205C00002014
:103948000000002074000020C93100089C0D0020F0
:10395800F5300008493100080C000020B40D0020A3
:10396800DD33000810B50024A2B07C22214603A84C
:10397800029410F063F853238DF808304FF48873DD
:10398800ADF80A3001238DF80C30ADF80440FFF78C
:1039980027F8FE23B0FBF3F000EB400000EB4010EB
:1039A8008DF80D0001A800F077FCA0B958238DF818
:1039B8000E30072430228021154810F03FF82246A7
:1039C80002A9134810F073F8114A21460120FFF7A5
:1039D80089FD22B010BD06238DF80E3000F034FCAE
:1039E8000C4B1A6812128DF80F201A688DF81020E7
:1039F8005A6812128DF811205A688DF812209A68A8
:103A08009B688DF8143012128DF813200D24D1E71D
:103A1800CD0D0020F40E002030B50378592B91B05D
:103A2800044640F0D881052959D84378443B162BE1
:103A380055D8DFE813F018015400080154001001AC
:103A480054005400540054007A005400F300540009
:103A5800540054007F015400540096005400540050
:103A6800540017008578482D11D1AA4A1421012045
:103A7800FFF738FD41F28830FFF734F840F6B830E8
:103A8800FFF730F811B0BDE83040FFF7D9BC532D2F
:103A98000ED130228021A0480FF0D0FFFFF762FF3F
:103AA80041F28830FFF71EF89B4A152101206DE08E
:103AB800432D16D1002468468DF8004007F07EFAA1
:103AC800954A4C231370102393709DF8003054705E
:103AD80001204133D07013710521FFF703FD11B0A8
:103AE80030BD442DFBD18C4C592323705A2363706D
:103AF800A57000F0A9FB2C228021201D0FF09EFF4D
:103B080000232570637001251023A370E5702571CB
:103B1800FEF766FFFE23B0FBF3F000EB400000EB7E
:103B28004010607122460621C0E78378303BDBB243
:103B3800092BD4D879497A4A0B700B78DBB25372C7
:103B4800754A592313704D2353700B783033937093
:103B580003210120FFF7C6FC11B0BDE83040FFF794
:103B68001BBD8578482D16D16B4A56231370002348
:103B780053701023937003231371172353710B236E
:103B8800012093710223D070D371082111B0BDE8D0
:103B98003040FFF7A7BC432DA1D15F4C00213C2248
:103BA80001A800910FF04AFF6846FFF75BFD242249
:103BB800802104F10C000FF041FF9DF80030637084
:103BC8009DF80130A3709DF80230E3709DF8033032
:103BD80023719DF8043063719DF80530A3719DF839
:103BE8000630E3719DF8073023729DF80830257080
:103BF80063729DF80B509DF80930A3729DF80A3046
:103C0800E3722A4603A9257304F10D000FF04FFF54
:103C180005F10D012246C9B201205EE780783928F6
:103C28000CD83038C0B2FFF78DFA3B4A23781370AE
:103C380063785370A3789370032137E711B0BDE818
:103C48003040FFF79BBC80783928F7D83038C0B2AD
:103C5800FFF779FAE9E780783928EFD83038C0B229
:103C6800FFF772FAE1E78378303BDAB2092AE5D840
:103C7800C0783038C2B2092AE0D82179A1F14802C7
:103C8800D2B20B2ADAD8274D45FA02F2D507D5D495
:103C98000A224D2902FB030036D13C2358434FF436
:103CA8007A735843204B1860204B1860FFF798FA36
:103CB800194A2378137063785370A3789370E37864
:103CC800D3702379137105210120FFF70BFC144BE6
:103CD80000221A7010225A7001229A70DA70A278A3
:103CE800303A02EB8201E278303A02EB4102D2B27A
:103CF8001A7122795A710E4A1278D2B21A72074A88
:103D08001278D2B25A7227E74829C8D14FF46163B2
:103D1800C4E700BFE73C0108CD0D0020440C00209B
:103D280078000020DEF7FFFF740000200C00002060
:103D3800620E00208278303AD3B2092B3FF67EAF6C
:103D4800C378303BD9B209293FF678AF0079A0F1A2
:103D58004801C9B20B293FF671AF624D45FA01F12E
:103D6800C9073FF56BAF0A214D2801FB02332DD15E
:103D78003C2253434FF47A7253435B4A13601068F2
:103D8800FFF746FA594A2378137063785370A3787B
:103D98009370E378D3702379137105210120FFF71D
:103DA800A1FB534B00221A7010225A7001229A70FC
:103DB800DA70A278303A02EB8201E278303A02EB0C
:103DC8004102D2B29A712279DA7194E74828D1D1A6
:103DD8004FF46162CDE7502B48D102297FF67FAEC0
:103DE8004378303B012B3FF67AAE8378312B7FF452
:103DF80076AE0B2904D8FFF7C1FB00213B4A55E6F4
:103E08003B4D0234002214F8013FA918303B01321F
:103E1800DBB20C2A0B73F6D1FFF7ACF9334B502207
:103E280010211A709970002201215A70D97003F874
:103E3800041FA9180132097B0C2A01F1300103F88B
:103E4800011FF6D100232B7010236B700123AB7078
:103E5800EB70284B1B78DBB22B72274B1B78DBB23D
:103E68006B72EA72FFF798FB1121C7E7412B7FF4C9
:103E780036AE4378432B7FF432AE16297FF42FAE4B
:103E88001E4D421C002312F8011FE9540133142B64
:103E9800F9D1FFF715F91A4B5B7D012B19D114499C
:103EA8000023EA5CC8180133D2B2142B80F82C2006
:103EB800F7D1114B00221A701B78DBB24B72FFF757
:103EC8006BFB0A4A631E1534A34206D1074A162122
:103ED800ECE5094B02221A70F3E713F8011F02F808
:103EE800011BF1E7DEF7FFFF0C000020CD0D0020DD
:103EF80078000020620E0020440C00204E0E0020A6
:103F0800B40A002038B504460D4661B316480FF0D0
:103F1800D1FB2B783BB334B36068237818B3032BF9
:103F28000CD00B2B17D0022B1DD1617801291AD088
:103F38000B0618D4BDE83840FFF76EBD6378012B37
:103F480011D10078012802D0022800D058B9BDE864
:103F5800384006F0B3BE6378012B04D10378034AD6
:103F680003F00103137038BD500D0020370D0020F9
:103F7800034B0022C3E902220122C3E90022704751
:103F8800640E002000487047640E00204FF0B043D4
:103F980082B0DA6C0243DA64DB6C03400193019B64
:103FA80002B070472DE9F04186B000240220154D7B
:103FB8000594FFF7EBFF0420FFF7E8FF124F039487
:103FC8004FF4807601230DEB0001CDE9016328460B
:103FD800032304934FF4005803F0DAFD01A938468F
:103FE800CDF8048003F0D4FD22464146384603F05C
:103FF800F5FE28462246314603F0F0FE204606B07C
:10400800BDE8F0810004004800080048032810B506
:104018000ED8012810D868B902460B484FF48071B1
:1040280003F0DCFE002209484FF4005103F0D6FEED
:10403800002010BD0122F0E7002203484FF48071F0
:1040480003F0CCFE0122EEE7000400480008004817
:1040580002207047002070470120704700280CBFDD
:104068000F201620704700000D48854602F0ACFD71
:104078000C480D490D4A002302E0D458C4500433BB
:10408800C4188C42F9D30A4A0A4C002301E0136091
:104098000432A242FBD30FF0D9FCFEF7D3FAFEE7B5
:1040A8000000012000000020CC0800209C470108E7
:1040B800CC080020382E0020FEE74FF0B04382B035
:1040C800DA6C42F00102DA64DB6C03F0010301935D
:1040D800019B02B07047000030B587B0FFF7EDFFD5
:1040E8004FF4805101224FF0904003F077FE0122F7
:1040F8004FF400614FF0904003F070FE4FF4C0554C
:104108001123CDE9015301A901234FF090400393F6
:1041180003F03EFD08240A2500224FF480514FF099
:10412800904003F05BFE0120FEF7DCFC01224FF417
:1041380080514FF0904003F051FE0120FEF7D2FC71
:10414800013DE9D14FF400614FF0904003F040FE8B
:1041580008B9013CDFD14FF400614FF0904003F003
:1041680037FE68BBFFF7A9FF04240123039001A9C8
:104178002A48CDE9014303F00BFD284C0122042114
:10418800204603F02BFE2120FEF7ACFC0022042180
:10419800204603F023FE2120FEF7A4FC012204217F
:1041A800204603F01BFE2120FEF79CFC204600223F
:1041B800042103F013FE4FF42570FEF793FCDDE7AE
:1041C800FFF77BFF4FF0B04300249A6D42F4800262
:1041D8009A659B6D03F4800300934FF4C052009BD3
:1041E8001223CDE901230323CDE9034304230DEB77
:1041F80003014FF09040059303F0CAFC08480949B1
:10420800094B8460C0E900130123C0E90334C0E905
:104218000744446103F056FF07B030BD000400486E
:10422800740E0020005800401A091020FFF754BFF0
:10423800012806D14B1E5A4202485A41082103F070
:10424800CDBD70470004004808B50120FEF77AFF8D
:104258006420FEF747FC00F027F96420FEF742FCD3
:10426800BDE808400120FEF76EBF0000084B1A6841
:1042780002805A689A68428110B51A685C68996821
:1042880013190B440381034B01221A7010BD00BFA0
:10429800F40E00204D0E002010B5044600F008F87A
:1042A80010F0FF001CBFEE232370AA23637010BD1B
:1042B8002DE9F34700242D4E2D4D3460214620462C
:1042C800FFF7B6FF21460120FFF7B2FF2146022083
:1042D800FFF7AEFF274F4FF05208A146012195F88E
:1042E800640185F86081C5F86891FFF7A1FF032094
:1042F800FEF7F8FB0DF10602C021284602F018FC73
:1043080078BBBDF806204EF6AA639A4229D14FEA37
:10431800440A0AF1540A5FFA8AFA5146284600F01C
:104328001FF9F0B90DF10602C021284685F860A1F1
:1043380002F0FEFB284600F0D7FA90B93268012354
:104348001A4432603A68C5F86831A34013433B60A9
:104358000134032C05F5C875C0D1306802B0BDE83A
:10436800F0870021E0B2FFF763FFF1E7EC0E0020D1
:10437800BC000020E80E00202DE9F74F354C83469D
:1043880004F5966A4FF00A094FF00E0848F2E8075C
:104398004FF490164FF48045D4F86821002A51D084
:1043A800204600F095FD0DF102020DF101012046B5
:1043B80000F048FB0DF1030201A9204600F08DFE34
:1043C8000021204600F0D0F801220021204600F00C
:1043D8008FF901221146204600F08AF9BBF1020F3D
:1043E8000ED81D4B1D4A33F81B501D4B12F80B807D
:1043F80053F82B601B4A1C4B12F80B9053F82B7088
:104408002A460121204600F0BEF932460021204606
:1044180000F0B9F93946204600F0C0F842460021BC
:10442800204600F0BDF84A460121204600F0B8F8C1
:104438000DF102020DF10101204600F003FB0122FB
:10444800C4F87C2104F5C8745445A5D103B0BDE86F
:10445800F08F00BFBC000020FC3C01081C3D010897
:10446800043D01081F3D0108103D010810B50B7EF1
:104478009BB9D0F87C21098912B1C0E95E1310BD3F
:10448800084BD0F878411A68C2F580734B4304FB97
:1044980002331B12C0F87831F1E70123C0F87C31F0
:1044A800EDE700BFB80000202DE9F047DFF898904D
:1044B800264EFFF7BBFED9F800300BB1336813B9AD
:1044C800FFF7F6FE30603368214D0024A3422C60CC
:1044D8006C60AC6036DDDFF87C801F4EDFF87CA0B6
:1044E8000220FFF749FF2C606C60AC6088F8004040
:1044F800D6F86871012F1BD11849304600F048FCE6
:10450800B0B951463046FFF7B1FF9AF818307BB979
:10451800D6F8783145F82430D9F80030A7401F4341
:1045280098F80030C9F8007043F0010388F80030AB
:104538001E200134FEF7D6FA032C06F5C876D7D12B
:1045480098F80030BDE8F087E80E0020F00E002053
:10455800F40E00204D0E0020BC000020CC0E0020E0
:104568004A088A2102F096BA152906D8044BCB408E
:10457800DB0702D50174002070476FF00700704711
:104588000B00300010B50A460C46092102F0A4FAC7
:1045980018B9237803F00103237010BD01F06BBE36
:1045A80001F053BD01F04DBEF7B500230C46174688
:1045B80001210DF1070206468DF8073002F08CFA4A
:1045C8000546D8B9012F9DF8073026D1042C3AD8D2
:1045D800DFE804F003171A1D200043F01004A3427B
:1045E8000CD022460121304602F054FA054628B97B
:1045F800716986F830413046FFF7D0FF284603B08E
:10460800F0BD43F02804EAE743F00404E7E743F089
:104618004004E4E743F08004E1E7042C13D8DFE822
:1046280004F00306090C0F0003F0EF04D7E703F0CA
:10463800D704D4E703F0FB04D1E703F0BF04CEE7C7
:1046480003F07F04CBE76FF00305D7E713B500232A
:104658000C460DF1070201218DF8073002F03CFAF3
:1046680078B99DF80730C3F300122270C3F3C00273
:10467800A270C3F380026270C3F38012DB09E27098
:10468800237102B010BD37B50D460DF10202F821B5
:10469800044602F04DFA70B901AA0421204602F03E
:1046A80067FA40B9BDF802201AB1019BB3FBF2F3D7
:1046B8002B602B68A36103B030BD037F0B70002013
:1046C800704737B50D460DF106022021044602F069
:1046D8002FFA28B9BDF8063023B9236A2B60207752
:1046E80003B030BDDB002B60236201232377F7E79B
:1046F8000529F8B504460E46154635D862B100EBD3
:10470800810301215A6B0023701E042807D8DFE8B3
:1047180000F00E171A1D240011460123F4E784F84F
:1047280028103444E5B984F82850002007E0C2F383
:104738004F224421204602F0BDF90028F1D0F8BDEF
:1047480084F82A10EDE784F82B10EAE75B00FE22D4
:104758006021204602F0D5F9EFE71B01EF22F7E7C9
:10476800012384F82830E0E76FF00300E7E7052924
:1047780096BF4018002390F82830137094BF00208B
:104788006FF00300704770B54318044693F828008B
:104798000E46154618B904EB8106726370BD0529EB
:1047A8001BD8DFE801F0030912141616626304EB44
:1047B800860400206563F1E7C2F34F2244212046B6
:1047C80002F078F90028E9D1F1E7E263EFE7226423
:1047D800EDE7C2F34F226421F1E76FF00300DDE754
:1047E80037B50446154605292CD8DFE801F003073C
:1047F80017191B1B436B2B60002021E00DF10602EB
:10480800442102F095F9D8B9BDF8062053029AB1AF
:104818002B60A363012384F8293011E0C36BEAE716
:10482800036CE8E70DF10602642102F081F938B95A
:10483800BDF806305B02DEE7A36B2B6084F8290025
:1048480003B030BD6FF00300FAE737B50D460DF140
:1048580007020121044602F03FF938B99DF80730F4
:1048680084F83031DB092B7084F84C3003B030BD4C
:104878002DE9F843037C0C4601F8083B0546FFF791
:1048880002FF40BB207304F110012846FFF719FF0F
:1048980008BB04F11401284600F021FCD8B904F142
:1048A800240705F1270904F1170806463A46B1B26C
:1048B8002846FFF795FF70B9013619F8013F08F847
:1048C800013F062E07F10407F0D104F13C01284608
:1048D800FFF7BBFF08B1BDE8F883211D2846BDE8F6
:1048E800F84301F030BD0000F0B50022054693B052
:1048F800882102F0CFF84FF47A72A5F852214FF4CC
:10490800C872A5F854214C4AC5F8582100234B4ACF
:1049180085F8F030C5F8D4202B6202A92846FFF7A5
:10492800A7FF044670B9ADF8080002AE0FCE05F136
:1049380010070FC70FCE0FC70FCE0FC796E80F008F
:1049480087E80F003E4BC5F834314FF4FA7301265F
:10495800A5F838314FF42063A5F83C313246802160
:1049680085F85061284602F095F832460746FF213F
:10497800284602F08FF8002211460743284602F025
:1049880089F83C4364B204430DF10702912128469B
:1049980002F0A2F864B29DF8073085F83A31044372
:1049A80032460021284602F075F864B2044300221A
:1049B800FF21284602F06EF864B2044300228021E9
:1049C800284602F067F864B2204340B2002488BB4E
:1049D800A1B2012228460134FFF78AFE062CF6D13F
:1049E80040BB04466885024604212846FFF780FE3E
:1049F80000BB024605212846FFF77AFED0B94FF4DE
:104A080090136B634FF4804201212846FFF7BBFEE9
:104A180080B94FF40C13FF22C5E90F3085F8302117
:104A28000121284602F036F8012385F8323108B909
:104A380085F8154113B0F0BD856B0100A47009001D
:104A480064008403012300F079BD2DE9F0428EB0A3
:104A58000C460C2304AA1421054602F005F88446E6
:104A680000286CD19DF81A309DF81B609DF817201E
:104A78009DF81810A07506EB03269DF816302060E7
:104A880002EB03229DF81930606003EB01239BB20F
:104A98005B029DF8121023619DF81330B5F852019E
:104AA80003EB012392B252029BB2E260A382B0F5FB
:104AB8007A7F9DF8101095F83171B6B20AD070431C
:104AC80000F5FA704FF47A76B0FBF6F02E7F002EE0
:104AD80039D186B2002F40D0B001C0B2B608E07517
:104AE8000DF10F002681CDE90040284601F086FE31
:104AF800844620BB9DF80FE084F818E005F15006C5
:104B08000FCE07AF0FC796E80700E37D87E80700D9
:104B1800D4E90301A28AADF83020D4E90149CDE9EE
:104B28000A01CDE9084907AC8DF833308DF834E037
:104B38000FCC50350FC597E8070086E80700604698
:104B48000EB0BDE8F0822E8C5E43B2EB262F4FEA02
:104B5800262C04D157B948F6E0260020BFE780B2DA
:104B68005043A2EB0C06B0FBF6F0B2E742F2B826CF
:104B7800B2E70000F7B517460E210DF106021D46F3
:104B88000B4C064601F0D4FFBDF8063004EA434357
:104B98003B6050B90DF106020C21304601F0C8FF08
:104BA800BDF8063004EA43442C6003B0F0BD00BFF2
:104BB8000000FE1F73B590F8DA30013B022B064661
:104BC8000C4634D801AB6A460121FFF7D3FF009B9E
:104BD800B3F57F0F054603D8019BB3F57F0F23D9A3
:104BE80015BB34B11349304602B0BDE8704001F03E
:104BF8000FBC0422FF21304601F04CFF2A46044630
:104C08007021304601F046FF2A460443FF21304612
:104C180001F040FF64B204432A468021304601F087
:104C280039FF64B2044365B2284602B070BD00255E
:104C3800FAE700BF5F06002037B50446012280214D
:104C4800057C01F027FF0122FF21204601F022FF09
:104C580000221146204601F01DFF94F83A219121C7
:104C6800204601F017FF01220021204601F012FF23
:104C78000022FF21204601F00DFF0022802120465E
:104C880001F008FF012D29D0032D37D0002D3CD18C
:104C980001222946204601F0FDFE01238DF8073048
:104CA800A0B103B030BD01460DF10702204601F066
:104CB80013FF9DF80730DB0705F1010508D538B962
:104CC800B5F5FA6FEFD16FF00600EAE70546F0E7B1
:104CD800B5F5FA6F08BF6FF00600E2E718B9294684
:104CE8002046FFF767FF02220021204601F0D2FE8E
:104CF8000028D6D1042384F83231D2E718B901212B
:104D08002046FFF757FF0422EEE76FF00700C8E7D9
:104D180038B5057C044625B1204600F054FD28B17D
:104D280038BDFFF789FF0028F6D0F9E7002DF7D145
:104D3800032384F83231F3E773B5064600250122D0
:104D48000B21304601F0A6FE002204460B21304616
:104D580001F0A0FE0DF1070204431321304601F0D3
:104D6800BBFE9DF8073064B2044301355B0760B2AF
:104D7800EDB205D0032D08D00028E0D002B070BDF8
:104D8800032D08BF6FF00B00F8E76FF00B00F5E795
:104D980038B50023037404460D46FFF7B9FF50B930
:104DA80029462046FFF751FE28B901462046BDE8AE
:104DB8003840FFF7C1BF38BD152970B505461646FE
:104DC8001C4667D10122FF2101F064FE0022114632
:104DD8000446284601F05EFE00220443FF212846CF
:104DE80001F058FE64B2044301228021284601F0F4
:104DF80051FE64B2044302228521284601F04AFE8E
:104E080064B204430422FF21284601F043FE64B241
:104E180004430022CD21284601F03CFE64B204433D
:104E28001122CC21284601F035FE64B20443072242
:104E3800FF21284601F02EFE64B204430022BE2161
:104E4800284601F027FE64B204430622FF212846C3
:104E580001F020FE64B204430922CC21284601F067
:104E680019FE64B204430022FF21284601F012FE15
:104E780064B204430122FF21284601F00BFE64B20C
:104E8800002204431146284601F004FE64B2204380
:104E980040B270BD042A17D80A2101F0FBFD002892
:104EA800F7D1231E18BF01231B01EF2284212846B6
:104EB80001F027FE0028ECD185F8DA600146284683
:104EC800BDE87040FFF738BF6FF00A00E1E7000067
:104ED80070B594B005464022002104A80EF0AEFD3E
:104EE800002301212846ADF806308DF803308DF8EF
:104EF8000430029300F0B8FC95F8142195F81311CA
:104F0800012A04D840F0AD80202940F2AC8001AAE3
:104F180002A9284600F02DFB0446002840F09E8098
:104F280095F85031002B40F0A280D5F84C11284656
:104F380001F06EFA0446002840F09080234621468E
:104F480004222846FFF738FF0446002840F08680F0
:104F58000122FF21284601F09DFD0DF106020646BB
:104F68008421284601F0E4FD22460643FF21284615
:104F780001F090FD76B2064374B2002C6ED1BDF8F4
:104F880006301B01C5F8D43004A92846FFF770FC89
:104F98000446002862D10DF103012846FFF7F2FA12
:104FA800044600285AD19DF8033085F8313104AE03
:104FB8000FCE05F110040FC40FCE0FC40FCE0FC4CF
:104FC80096E80F0084E80F000DF10302012128463E
:104FD80001F082FD0446002840D19DF8033085F891
:104FE8003031024601462846FFF7DEFA0446A8BBE0
:104FF800024602212846FFF7D7FA044670BB03236E
:10500800014685F832310DF10502284601F019F9FB
:10501800044618BB9DF8053085F8E8300DF1050207
:105028000121284601F00DF90446B8B99DF805306C
:1050380085F8E03003AA0321284600F001FF044662
:1050480060B9039BC5F8E43003AA0421284600F0A0
:10505800F7FE044610B9039BC5F8DC30204614B0AF
:1050680070BD0C2951E7284600F010F954E70149B2
:105078005DE700BF6C05002013B50C460DF1070273
:10508800132101F029FD9DF8073013F0180F03F0E4
:10509800070218BF6FF00500226002B010BD13B5FB
:1050A80090F8DA30042B0C460BD101A9FFF7E4FF86
:1050B800019B042B01D1012300E00023237002B0DF
:1050C80010BD01AA142101F007FD0028F7D19DF8B1
:1050D8000430DB07EFD42070F1E700F04ABA13B5CB
:1050E8000C460DF10602282101F022FD78B9BDF821
:1050F8000620C2F30B0312F4006F18BFA3F5805308
:105108004FF0FA0214BF13FB02F35343236002B0BB
:1051180010BDF0B54FEAD20C4FF0FF341C6002F01E
:105128000702664600278E4200D207B1F0BD845DB3
:10513800664503BF1441E4B215463D4614F0010725
:1051480004D005EBC6051D600136ECE70135082DD6
:105158004FEA5404F2D1F7E7034B800953F82000D3
:10516800003818BF012070471808002010B5B1EBAF
:10517800D20F4FEAD20402F0070381BF01229A40FE
:10518800035D13438ABF03556FF03100002010BD43
:105198000A460623B02101F049BC0A460623B0217D
:1051A80001F062BC2DE9F04F85B08046109E0E9D3F
:1051B80001968A4693461C464FF00009119B994573
:1051C80008D10023129A1660F3B16FF0310005B0D0
:1051D800BDE8F08F01AB324629465846FFF799FFE4
:1051E800019F7B1C0DD00F9BF818FFF7B5FF5045AA
:1051F80007D13A462046FFF7B9FF7E1C09F101099D
:10520800DCE76FF03103DDE721464046FFF7C0FFDA
:105218000028DCD102A94046FFF7BFFF25442346FA
:1052280002AAAB42D3D013F8014B12F8011B8C42EF
:10523800F7D0CAE770B5C02288B00E46012190F8B1
:105248003041054601F026FCF0B901A92846FFF7D0
:105258009FFDC8B90122FF21284601F01BFC98B91F
:105268003246B621284601F063FC68B90246FF21A0
:10527800284601F00FFC38B922460121284601F0E2
:1052880009FC08B985F8304108B070BDF0B50F4683
:1052980089B01646FF210122044601F0FBFB0246B5
:1052A800A8B94F21204601F0F5FB80B92C224E21E8
:1052B800204601F0EFFB024648B9FF21204601F0E5
:1052C800E9FB20B9B422B621204601F0E3FB002512
:1052D800C4F82451A4F82851DEB9354607ABB422E6
:1052E800CDE903730623CDE90032029504F59273E4
:1052F80004F5957231462046FFF754FF30B9012373
:1053080084F8153184F8137184F8146109B0F0BD7C
:10531800013505F1B400FFF71FFF0028DED12C2D61
:10532800F6D1DBE710B541F001020021044601F097
:10533800B1FB78B9204600F046FA58B90146204634
:10534800FFF7FAFC30B9024601462046BDE8104096
:1053580001F0A0BB10BD2DE9F74F4FF0000B8846B8
:105368001746FF21012205461E469DF838A09DF8E4
:105378003C908DF807B001F08DFB5A46044659461B
:10538800284601F087FB5A460443FF21284601F0CE
:1053980081FB64B2044364B2B8F1000F32D0BAF1B1
:1053A800000F06D00C9ACB21284601F095FB20432C
:1053B80044B2B9F1000F07D00DF10702EE212846DB
:1053C80001F08AFB204344B20122FF21284601F064
:1053D80061FB012204430021284601F05BFB64B213
:1053E80004430022FF21284601F054FB64B29DF8D3
:1053F80007300D9A204323F0100340B2137003B016
:10540800BDE8F08FBAF1000F06D03A46CB21284606
:1054180001F040FB204344B2B9F1000FD4D0334629
:105428008022EE21284601F06CFBCBE72DE9F04302
:1054380087B091460022054688468DF817201E46FB
:105448001BB390F8307101221146284601F022FB67
:10545800044658BB40212846FFF764FF044628BB92
:10546800B9F1010F13D10DF11703CDE90290CDE980
:1054780000830246034649462846FFF76CFF40B1C1
:105488000446204607B0BDE8F0831F46DBE788F8EE
:105498000000002EF5D03A460121284601F0FAFA1C
:1054A80004460028EDD185F83071EAE7002388F832
:1054B80000302046E4E72DE9F043054687B08846EA
:1054C80091461E4623B390F83071022201212846E6
:1054D80001F0E0FA044660BB01462846FFF722FFC8
:1054E800044630BBB9F1010F14D10DF11703CDE912
:1054F8000209009302460346CDF80480494628462F
:10550800FFF729FF40B10446204607B0BDE8F08305
:105518001F46DAE788F80000002EF5D03A46012148
:10552800284601F0B7FA04460028EDD185F8307115
:10553800EAE7002388F800302046E4E7F8B51D467E
:10554800164600232A4690F830710446FFF76EFF8E
:1055580070B903462A4631462046FFF7ACFF38B9F2
:105568003A460121204601F095FA08B984F83071CD
:10557800F8BD2DE9F04F002393B0CDE90A12C0F829
:105588002431A0F828310122FF21CDE90E33B0F8EB
:105598003C818DF8343005468DF8353001F07AFAC3
:1055A8000446002840F0E38002464F21284601F0D7
:1055B80071FA0446002840F0DA802C224E21284651
:1055C80001F068FA0446002840F0D1800246FF2125
:1055D800284601F05FFA0446002840F0C880B4224B
:1055E800B621284601F056FA0446002840F0BF804C
:1055F80002468021284601F04DFA0446002840F072
:10560800B68003460DF135020DA92846FFF796FF2F
:105618000446002840F0AB800323CDE90203B421FF
:10562800062305F5957A05F592790EAECDE9003198
:10563800049601464B4652462846FFF7B3FD0446FA
:10564800002840F094800DF1360128460E9FFFF7A0
:10565800F1FD0446002840F08A80BDF83630434505
:1056680040F2AA80C5F82401A5F8280107F1B40082
:10567800FFF772FD08B92B2F7DD90623B4224FF00E
:10568800030BCDE90032CDE9027B04964B46524626
:1056980001212846FFF786FD002840F08B800DF198
:1056A800360128460E9FFFF7C5FD064600287CD127
:1056B800BDF83630434540F2828001260696BDF893
:1056C8003630434560D2A3EB080383EAE372A2EBCA
:1056D800E3729DF81860099205F592734FF0030B79
:1056E8000793079B18689B881090ADF844303A469A
:1056F8000FAB06215046FFF70CFD0F9F7B1C56D0C1
:1057080007F1B400FFF728FD069B98423CD10BF146
:1057180001033A4648460893FFF728FD002849D177
:1057280049462846FFF734FD002843D10DF13601DC
:105738002846FFF77FFD00283CD1BDF83620A2EBB4
:105748000803002BB8BF5B42424516D9099A934219
:1057580018D910A92846FFF71BFD079A0799034691
:1057680010981060BDF844208A806BB11C46204612
:1057780013B0BDE8F08F013778E7DDF820B0099362
:105788000137AEE7DDF820B00A9BC3F800B00B9BE9
:105798001E70012385F815310A9B1B6885F81331A3
:1057A8000B9B1B7885F81431E1E70446DFE76FF0BF
:1057B8003104DCE70446DAE70026B3467EE7012336
:1057C800834606937BE737B5002304468DF80730F8
:1057D8004FF4FA650DF107012046FFF760FC58B950
:1057E8009DF80730012B07D0013D03D0204601F07A
:1057F800E5F9EFE76FF0060003B030BD02464FF061
:105808008043934202D8002013B970479B08F8E7F9
:10581800C11891424FEA50009CBFC018521A9B0809
:10582800F2E773B500228321054601F033F90446F7
:1058380088B94FF4FA660DF107028321284601F072
:105848004BF99DF807300343DBB204461BB9013E10
:10585800F1D16FF0060401228321284601F01AF9DC
:10586800204340B202B070BD2DE9F04F90F8F060CF
:1058780091B04FF00009072ECDE9079904460F466D
:1058880000F0A2820122802101F004F90122804661
:10589800FF21204601F0FEF84A4648EA000849463A
:1058A800204601F0F7F84FFA88F848EA000806227F
:1058B800FF21204601F0EEF84FFA88F848EA000880
:1058C8000DF115028321204601F006F99DF81520F7
:1058D8004FFA88F848EA000842F00402832120467B
:1058E80001F0D8F84FFA88F848EA00080722FF21A3
:1058F800204601F0CFF84FFA88F80122812148EAC2
:105908000008204601F0C6F84FFA88F848EA00086F
:10591800204601F053F94FFA88F848EA00080122B6
:105928008021204601F0B6F84FFA88F848EA0005C9
:1059380017F0010B6DB200F01E82F20700F11E8213
:105948006B229421204601F0A5F880462046FFF7F7
:1059580068FF06AA48EA00089021204601F008F9E5
:1059680045EA0805069B6DB224229421054320468A
:10597800C3F3062AC3F3C03901F08CF86DB20543AE
:105988002046FFF74EFF6DB2054306AA9021204638
:1059980001F0EEF8069B6DB21BBA2522942105434F
:1059A8002046099301F076F86DB205432046FFF7CB
:1059B80038FF6DB2054306AA9021204601F0D8F8B9
:1059C800069B6DB21A0E05431B0C6DB28DF828208C
:1059D8008DF8293017F00203029300F0DB8016F0EF
:1059E800020840F0D78002229421204601F052F8A4
:1059F80001902046FFF715FF019B0DF116020343A6
:105A0800902120461D4301F067F86DB27B22942156
:105A18000543204601F03EF86DB205432046FFF7E6
:105A280000FF6DB205430DF117029021204601F0E9
:105A380053F86DB2772294210543204601F02AF8E5
:105A48006DB205432046FFF7ECFE6DB2054306AA8A
:105A58009021204601F08CF8069B5A0E8DF82C20D8
:105A6800C3F386428DF82D20C3F3C6228DF82E206D
:105A78006DB2C3F30612DB0003F0780394210543EB
:105A88008DF82F20204678228DF8153001F002F885
:105A98006DB205432046FFF7C4FE6DB2054306AA62
:105AA8009021204601F064F8069B9DF8152002EB32
:105AB80053728DF83020C3F386528DF83120C3F32A
:105AC800C6328DF83220C3F306228DF833206DB22A
:105AD800C3F346029B0103F04003942105438DF86C
:105AE8003420204679228DF8153000F0D3FF6DB2AE
:105AF80005432046FFF795FE6DB2054306AA90219F
:105B0800204601F035F8069B9DF8152002EB9362BC
:105B18008DF83520C3F3C6428DF83620C3F306321C
:105B28008DF837206DB2C3F346129B0003F07C0357
:105B3800942105438DF8382020467A228DF81530B7
:105B480000F0A8FF6DB205432046FFF76AFE6DB26C
:105B5800054306AA9021204601F00AF8069B9DF805
:105B680015208DF83E8002EB93728DF83920C3F32F
:105B7800C6526DB28DF83A20C3F3064205438DF83C
:105B88003B20C3F34622C3F386036DB28DF83C2055
:105B98008DF83D3017F00403019300F0F18073078E
:105BA80000F1EE807B229421204600F073FF8046AE
:105BB8002046FFF736FE07AA48EA0008902120464B
:105BC80000F0D6FF45EA08084FFA88F848EA0005C9
:105BD8007C229421204600F05DFF6DB205432046EB
:105BE800FFF71FFE6DB2054308AA9021204600F07A
:105BF800BFFF6DB2732294210543204600F04AFF8F
:105C08006DB205432046FFF70CFE6DB2054306AAA8
:105C18009021204600F0ACFF069B6DB21B02742257
:105C28009421054320461FFA83F800F033FF6DB234
:105C380005432046FFF7F5FD6DB2054306AA9021FE
:105C4800204600F095FF6DB29DF81B307522942117
:105C58000543204643EA080800F01CFF6DB20543DF
:105C68002046FFF7DEFD6DB2054306AA90212046C7
:105C780000F07EFF069B6DB21B029BB27622942138
:105C880005432046039300F005FF6DB20543204607
:105C9800FFF7C7FD6DB2054306AA9021204600F024
:105CA80067FF6DB29DF81B20039B05436DB213433C
:105CB800002281212046039300F0ECFE06220543D2
:105CC800FF21204600F0E6FE6DB205430DF11502F6
:105CD8008321204600F000FF9DF815206DB2054392
:105CE80002F0FB028321204600F0D4FE6DB205438A
:105CF8000122FF21204600F0CDFE6DB205430122AE
:105D08000021204600F0C6FE6DB205430022FF21A7
:105D1800204600F0BFFE6DB20543002280212046D8
:105D280000F0B8FE6DB205436DB2039BFDB9BBF13F
:105D3800000F29D1029AAABB019AAAB1720713D4FB
:105D4800079AC4F81821089AC4F81C214FEA482277
:105D5800C4F820213BB1A3F5C8534FF47A725343DA
:105D68001B095B421BB2E3603E4384F8F06028469F
:105D780011B0BDE8F08FD946DA462BE6CA4629E6C7
:105D88004FF00008434693E7F007D3D40998BDF8CD
:105D9800282084F813A184F81491C4F82A01A4F8DF
:105DA8002E21C7E7B107C7D49DF8162084F8F12043
:105DB8009DF8172084F8F2200BA904F1F300029350
:105DC8000DF068FE029BB7E74D46D0E750B10138A9
:105DD800002330F0FF019AB203F1010303D100EB75
:105DE800022080B270474008F3E7C3B2000A03FA02
:105DF80000F0013070470000084B5A434FF47A73A3
:105E080002F5FA724FF4FA60B2FBF0F0B2FBF3F26B
:105E180003FB0100B0FBF2F0704700BF002F3A000F
:105E2800064B5A434FF47A7002F5FA72B2FBF0F25D
:105E38004A4302F5FA72B2FBF0F07047002F3A00BD
:105E48002DE9FF4102294FF00005074616468DF857
:105E58000350ADF804501CD80DF102022946FEF794
:105E6800A1FB044630B90DF103024621384600F083
:105E780033FE04469DF80300FFF7B7FF81B29DF893
:105E880002203846FFF7CCFF3060204604B0BDE85A
:105E9800F081032918D10DF102022946FEF782FB91
:105EA8000446002846D101460DF102023846FEF7A5
:105EB80079FB044628B901AA5121384600F038FE7A
:105EC8000446BDF80400D7E7042935D102A9FEF736
:105ED800BDFB9DF80B30ABB10DF1020229463846E7
:105EE800FEF760FB044658B901AA5121384600F074
:105EF8001FFE0446BDF80400FFF777FF85B214B112
:105F0800002015E01D460DF1020201213846FEF77A
:105F180049FB04460028F3D10DF1060271213846E9
:105F280000F006FE0446BDF80600FFF75EFF80B2EB
:105F3800401BA3E72846A7E728462C46A4E7F0B568
:105F4800022985B0054616461ED80DF10502002126
:105F5800FEF728FB0446A0B99DF8052031462846DF
:105F6800FFF74AFF83B2B3F5807F9ABF00F1FF3293
:105F7800D2B2FF22A5F8D8204621284600F08AFD93
:105F88000446204605B0F0BD03291FD10DF10502D6
:105F98000021FEF707FB9DF80520314604462846F8
:105FA800FFF72AFF80B2FFF711FF0246ADF806009F
:105FB800A5F8D800002CE4D15121284600F07AFD3C
:105FC80004460028DDD1C5F8E460DAE7042939D1B0
:105FD80002A9FEF73BFB9DF80B70B7B10DF1050266
:105FE80000212846FEF7DEFA04460028C9D10DF143
:105FF80006025121284600F09BFD0446BDF8060024
:10600800FFF7F3FE87B2002CBBD10DF10502012189
:106018002846FEF7C7FA04460028B2D19DF80520A5
:1060280031462846FFF7E8FE3844FFF7CFFE7121D6
:106038000246284600F03EFD04460028A1D1C5F8D6
:10604800DC609EE76FF003049BE7F0B585B00023A2
:106058008DF80330D30705460F46164605D439B9DF
:10606800A2F10C03DAB2062A11D96FF00300E6E0B8
:10607800012921D1A2F10803DAB2062AF5D8062BA4
:106088001AD8DFE803F03B1969198A199D00062B15
:1060980012D8DFE803F004112D112F113100182256
:1060A8005721284600F0F6FC08225621284600F021
:1060B800F1FC002840F0C3807408013CE4B2002FD2
:1060C80000F09180012FD0D101AA04212846FFF7C2
:1060D800B7FE50B922467021284600F0DBFC20B9F3
:1060E800019A04212846FFF72AFF85F8E06099E025
:1060F8003022D5E74022D3E75022D1E710224821A9
:1061080000F0C8FC08224721284600F0C3FC022200
:1061180004463221284600F0BDFC0C2204433021FD
:10612800284600F0B7FC64B204430122FF21284648
:1061380000F0B0FC64B2044364B230223021284637
:1061480000F0A8FC00220443FF21284600F0A2FC2E
:1061580064B2204340B2ACE72822482100F09AFC00
:1061680008224721284600F095FC032204463221E4
:10617800284600F08FFC044364B2092230212846E7
:1061880000F088FC01220443FF21284600F082FC2D
:1061980064B2044364B22022D0E73822482100F0D8
:1061A80079FC08224721284600F074FC03220446A3
:1061B8003221284600F06EFC044364B20822DDE771
:1061C8004822114600F066FC08224721284600F0C4
:1061D80061FC032204463221284600F05BFC04439C
:1061E80064B20722CAE702AA03212846FFF728FE5D
:1061F800B0B903AA02212846FFF722FE80B9224639
:106208005021284600F046FC50B9029A032128463E
:10621800FFF795FE20B9039A02212846FFF78FFE63
:1062280085F8E86058B969692846FEF7B7F930B9C2
:10623800024601230DF103012846FFF73CF905B09A
:10624800F0BD13B5144629B1012910D06FF0030031
:1062580002B010BD0DF10702502100F03DFC0028EE
:10626800F6D19DF8073001335B002370F0E70DF19C
:1062780007027021F1E7F0B5002385B04FF4FA6208
:10628800CDE9002344F61F63994206460F4604D819
:106298006FF00305284605B0F0BD02A9FEF7D6F950
:1062A80005460028F6D19DF809209DF808301343CB
:1062B8009DF80A201343A7F636341BD06A460221FC
:1062C8003046FFF7BDFD00283BD19DF808302BB1C3
:1062D800009B03F24E239C42DAD9E41A9DF80A3057
:1062E80023B3009B03F2B223B4EB430F4FEA4302FC
:1062F800CED9A41A9DF80B305BB101AA0321304610
:10630800FFF79EFD019B03F52573A342C0D2C0B9D8
:10631800E41A9DF80C30002BBCD0A4F226220421EC
:106328003046FFF70CFE77610546B3E79DF8093064
:10633800002BDFD0009B03F525739C42A8D9E41AF3
:10634800D8E70546A6E770B54FF4FA6286B0002391
:10635800CDE9022340F636330B600C4604A9064605
:10636800FEF774F90546002836D19DF811209DF8EE
:10637800103013439DF81220134319D002AA0221AA
:106388003046FFF75DFD002840D19DF810302BB155
:10639800029B03F24E222368134423609DF81230B7
:1063A800EBB1029B03F2B222236803EB42032360A2
:1063B8009DF81330EBB99DF814305BB101AA0421A4
:1063C8003046FFF73DFD019B03F226222368134464
:1063D8002360D8B923687361284606B070BD9DF85C
:1063E8001130002BE4D0029B03F525722368134477
:1063F800DDE703AA03213046FFF722FD039B03F5DF
:1064080025722368134423600028D4D00546E3E7A7
:106418002DE9F743002406460D46204615F804806A
:10642800B8F1000F00D010B103B0BDE8F083671CCD
:10643800B8F1FF0F15F8079029D1A71CEB5DB9F14A
:10644800030F36D8DFE809F0020B131B271D2C4475
:10645800E27802EB0323A6F834313C46DEE7271D39
:106468002C44E27802EB0323A6F83631F5E7271D22
:106478002C44E27802EB0323A6F83831EDE7271D18
:106488002C44E27802EB0323A6F83C31E5E7B8F1A7
:10649800040F0ED802344246291901A80DF007FB53
:1064A800434601AA4946304604EB080700F0BEFA05
:1064B800D3E76FF00300D0E773B500230E461360EF
:1064C8000DF1070105461446FEF7F7F840B99DF8A7
:1064D80007302BB1B38A2A6A534380331B0A2360DF
:1064E80002B070BD13B5CB681360144601AAFFF75C
:1064F800E3FF18B92368019A1344236002B010BD62
:10650800F8B5B0F85451D0F8580168438030000A03
:106518000E464543DDE90717144652B1B60206EBAD
:106528005202B2FBF4F202EB4202524302F500427D
:10653800140C069A534301F50042120C062003324C
:10654800B2FBF0F2C2EBC202B2F5803F38BF0331B2
:1065580003F500433EBFB1FBF0F1C1EBC10101F50A
:1065680000414FEA134334BF090C1B4903FB03F3F3
:1065780038BF494303EB57030B44B3FBF7F39B03C3
:10658800FE2205F120007F33B3FBF2F35C434FF4A6
:106598007A7704F5FA748009B4FBF7F42401FFF75D
:1065A8002DF904F5FA74BC4228BF4FF4FA63064685
:1065B80029BFB4FBF3F300205B19B4FBF7F428BF41
:1065C800B3FBF4F0FFF71AF9099B864294BF1E60EB
:1065D80018600020F8BD00BF0000F0FF2DE9F04F63
:1065E80091B0CDE90723036A0E930B690993054619
:1065F800CB680B930F460FAAFFF774FF0EAA394614
:106608002846FFF759FF58BB0F9C95F8E0B0D5F81E
:10661800DC3005934FF47A7606FB04F101F500416E
:1066280004910E990A910499D5F8E4300693BBF1C8
:10663800080F04F180040CBF0223032324F0FF0A8F
:10664800090C95F8E820DFF8A081CDF83CA00C9162
:1066580009D1079BC3F80080089BC5F840811860E2
:1066680011B0BDE8F08F06990D932846FFF7C4FBDB
:106678005A46059981462846FFF7BEFB0D9B5B49A4
:106688000C9A814403FB09F94FEAC92940F2776360
:1066980009F5FA79240AB9FBF6F903FB09F909F5B2
:1066A800FA79B9FBF6F909FB04F404F18003099CB3
:1066B80074430C40B4FBF2F44D4A1B0A944228BFC1
:1066C8001446012B38BF01230C204FF4167258438F
:1066D8005443FFF793F83B7E3A894FEA400B002B6F
:1066E8007FD14249049B0B4003F5FA71414B5A4351
:1066F80041F25C23B2FBF3F20A9B7343B3F5481FE4
:1067080028BF4FF44813A1EB4303B1FBF6F1B3FBE9
:10671800F6F31B02B3FBF1F63602C6F58036564394
:1067280006F50046360C06F5803676087643B60B35
:106738004FF44870704304F5004300F500401B0C0B
:106748005B43000C00FB0030FFF758F80304642299
:10675800323341F28837B3FBF2F340F6B532B3FB7C
:10676800FBF302FB0377244B9F429CBF42F210735A
:10677800B7FBF3F7DDE90532134403F5FA734FF479
:106788007A7B4FF4FA62B3FBFBF0B3FBF2F202F54B
:10679800C812B2FBF0F088BF4FF47047FFF72EF82D
:1067A800000200F5FA70B0FBFBF0404307FB07005E
:1067B800FFF724F80BFB00F0079B0B9A404528BF16
:1067C80040461860089BC5F84001CDE902934FF494
:1067D800487300930194334651462846FFF790FECC
:1067E8003EE74FF48036A3E7AE878F020000FFFF35
:1067F800666666009A9906000F279F242DE9F04FD8
:106808008BB0002711F0780FDDE914B80446019227
:1068180099468DF80E708DF80F708DF810708DF800
:106828001170ADF812700997C1F3C30A00F0AF8078
:10683800AAF10503DBB20A2B01D86B4AD75C0DF12C
:106848000E0200212046FDF792FF9DF80E500646E5
:10685800D5B1002840F09D8009AB05AA59462046CD
:10686800FFF7BCFE002840F09680099BABF80A3081
:10687800014606AA2046FDF7B3FF069D25B1059BF4
:106888009D422CBF0025012520B904AA02212046DB
:10689800FDF76DFF9DF8106026B300287DD107AA8B
:1068A80002212046FDF79CFF88B90122FF212046DE
:1068B80000F0F0F858B90DF11202B621204600F0A8
:1068C80037F920B90246FF21204600F0E3F8BDF869
:1068D8001230079E5B02C4F848311EB19E422CBF9D
:1068E8000026012628B90DF1110203212046FDF7E3
:1068F8003EFF9DF8113093B1002873D1B9F1000F14
:1069080003D0019B1B02B3FBF9F908AA0321204617
:10691800FDF766FF089B4B4594BF0023012320B970
:10692800012F3CD1FF2288F8002098F800200AB9EE
:10693800ABF80A200DF10F02012120460193FDF763
:1069480016FF08BB9DF80E20019B002A08BF0125F1
:10695800BAF1040F18BF9DF80F2084F82E501ABF03
:10696800B2FA82F25209012284F82F209DF81020F1
:10697800002A9DF8112008BF0126002A08BF01231C
:1069880084F8306084F831300BB0BDE8F08F01270F
:1069980055E700257EE735467CE70026A9E70AF19A
:1069A800FF32092A0AD8DFE802F0050505090907B8
:1069B800090B070B0522B6E70422B4E7012E01D123
:1069C8000322B0E7BAF1040F01D0012B01D1022252
:1069D800A9E7012D1BBF002388F8003088F8005074
:1069E8002B46A2E70023A0E7223D010807B502F1E4
:1069F8000A03009393B20A4690F86011D0F85C013C
:106A080001F0B2FB03B05DF804FB13B502F10A0311
:106A180090F860410093D0F85C0193B20A4644F0C4
:106A2800010101F037FC02B010BD00003F2BF8B5A2
:106A38000E46054611461C4611D80A4F38461A46D6
:106A480000F8016B0DF033F8621C39462846FFF751
:106A5800CDFF00280CBF00206FF01300F8BD6FF0C9
:106A68000300FBE7000F002073B515468DF80710EB
:106A780001220DF1070104461E46FFF7B7FF28B9AA
:106A8800324629462046FFF7C0FF08B16FF01300D1
:106A980002B070BD08B5064B19705A70194602222B
:106AA800FFF7A4FF002814BF6FF01300002008BDF3
:106AB800000F002008B5074B1970110A59709A7019
:106AC80019460322FFF792FF002814BF6FF0130046
:106AD800002008BD000F002037B515468DF80710B7
:106AE80001220DF107010446FFF780FF28B90122B2
:106AF80029462046FFF789FF08B16FF0130003B05D
:106B080030BDF7B515460DF1070206460F461C467F
:106B1800FFF7E2FF50B99DF807301D4044EA05022F
:106B2800394630468DF80720FFF7B4FF03B0F0BDB3
:106B380073B514468DF8071001220DF107010646BA
:106B4800FFF754FF18B16FF0130002B070BD074D86
:106B5800022229463046FFF758FF0028F3D12A7849
:106B68006B7803EB02232380EFE700BF000F0020C0
:106B780073B514468DF8071001220DF1070106467A
:106B8800FFF734FF18B16FF0130002B070BD0A4D63
:106B9800042229463046FFF738FF0028F3D16B78E6
:106BA8002A781B0403EB0263EA781344AA7803EB00
:106BB80002232360E9E700BF000F002008B5022088
:106BC800FBF790FF002008BD7047000010B50320B8
:106BD80000F072FC01F0AAFD064B18600F20FBF7CD
:106BE80077FF044618B9FBF7E4FD204610BD0124E1
:106BF800FBE700BF280800204FF0E022136923F0CC
:106C08000203136170474FF0E022136943F0020357
:106C180013617047014BD3F8900570470070FF1F50
:106C2800014BD3F8940570470070FF1F014BD3F850
:106C3800980570470070FF1F024A536823F001034C
:106C480053607047002004E0024A536823F00203AF
:106C580053607047002004E0024A536823F004039D
:106C680053607047002004E08068C0F380007047DC
:106C7800F7B5002301930446002800F0E980856DEC
:106C880025B9FBF7EBF8E56584F8545023689A6852
:106C9800D00040F1A1809A68D10000F1B480A26DC3
:106CA80042F01002A265E26D42F00102E2650125A0
:106CB8001846FFF7D9FFA26D02F01002024340F018
:106CC800C980A26D206922F4817242F00202A26595
:106CD8009A68D2075DD4226BA67E94F82CC0003A3D
:106CE80018BF01221703D4E902120A43217E42EA9F
:106CF8008132617E42EAC13242EA4632002842EAE3
:106D08004C02B4BF20F000414FF400113A430A434B
:106D180094F82010012903D1002E76D142F4803254
:106D2800616A21B1A66A01F4E07131430A43D96866
:106D3800E66C21F4FE3121F4FF711143D96094F817
:106D48003C206168012A01F0404C4CEA060609D152
:106D5800D4E910273A433243A66C324342EA0C0284
:106D680042F001061F693E4A3A4032431A6121F057
:106D78000042B2F1804F0CD0B1F1004F09D0394E2A
:106D8800D6F8082701F4701122F470120A43C6F8E5
:106D980008275A69666BA16B22F0070232435A61D1
:106DA8005A6922F0700242EA01125A61002835D16C
:106DB8009A6A62F00F029A625B6903F007039E42C7
:106DC8003CD10023E365A36D23F0030343F00103E3
:106DD800A365284603B0F0BD9A68234922F0104203
:106DE80022F0170242F080529A60204A1268B2FBE1
:106DF800F1F2013252000192019A002A3FF44BAF9E
:106E0800019A013AF7E7002552E7A16D41F0200108
:106E1800A165E16D41F00101E16581E7B0F5001F71
:106E2800CAD19A6AE269013A92006FF00F0102F042
:106E38001C0201FA02F2216E0A43BCE7A36D23F09B
:106E4800120343F01003A365E36D43F00103E36508
:106E58000125BEE7A36D43F01003A365F8E700BF63
:106E680002FCFF1F00200140400D030028080020FD
:106E7800F8B54569082D04460E460AD00368DB6854
:106E8800D80705D5A36D43F02003A3650120F8BDFD
:106E98000425FBF71FFE074623681A682A4221D0FB
:106EA800A26D42F40072A265DA6812F4406F14D140
:106EB800A27E92B91A6812070FD51846FFF7D4FEBA
:106EC80028BB5A6822F00C025A60A26D22F4807224
:106ED80022F0010242F00102A265207E00BB0C22D2
:106EE8001A60D4E7711CD8D0FBF7F4FDC01BB04280
:106EF80001D8002ED0D123681B682B40CCD1A26DBD
:106F080084F8543042F00402A2650320BFE7A26D62
:106F180042F02002A265E26D42F00102E265DCE780
:106F28000020B4E70368186C70470000F7B5002329
:106F3800019390F85430012B044600F0C580056891
:106F48000669012380F854302846FFF78DFE002893
:106F580040F0B480D1E90020022826F0040300F0B4
:106F68008280B3F1004FC2F3110E13D1AB6A43EA2A
:106F78000E03AB628B68686903EA022323F07C4343
:106F880023F0FF0320EA02210B43002A6B6126DB72
:106F9800002055E0236E00F01F074FF00F0C0CFA8D
:106FA80007FC6FEA0C0623EA0C0CBEF1000F11D1A6
:106FB800C2F38463BB4043EA0C0323668008E36999
:106FC80001309842D6D8A86AC2F38363BB40064012
:106FD8003343CEE792FAA2F3B3FA83F3EAE73B49E5
:106FE8003B48D1F80837824203F0E07519D11B02FB
:106FF800CED4D1F8083723F0E0732B4343F40003D1
:10700800C1F80837334B1A68334BB2FBF3F20C2341
:1070180002FB03330193019B002BB9D0019B013B79
:10702800F8E72E48824210D113F08070B0D1D1F821
:10703800083723F0E0732B4343F08073C1F8083717
:10704800002384F8543003B0F0BD254882429FD114
:1070580013F480009CD1D1F8083723F0E0732B4358
:1070680043F48003EAE7B3F1004F01BFAB6AC2F310
:1070780011018B43AB62002A8ADA15481349824210
:10708800D1F8083709D1D1F8082703F0A07322F006
:10709800E0721343C1F808377AE71048824204D1F6
:1070A800D1F8082703F44003F1E70D4882427FF442
:1070B8006FAFD1F8082703F0C073E8E7A26D42F07C
:1070C8002002A2651846BBE70220BCE70020014069
:1070D800001000B028080020400D0300004000B850
:1070E800002000B4026838B504461046FFF7BCFD1E
:1070F80008B9002038BD9368990707D4936823F02E
:10710800004323F0170343F010039360FBF7E2FCFE
:10711800054623689B685B07EBD5FBF7DBFC401B48
:107128000228F6D923689B685A07F2D5A36D43F065
:107138001003A365E36D43F00103E3650120D9E77C
:1071480073B50023026801939368DD07044602D5EE
:10715800002002B070BD9168214B194209D0A36D7F
:1071680043F01003A365E36D43F00103E3650120D9
:10717800EFE7936823F0004323F0170343F001037C
:107188009360184BD3F8083718021CD4637E012B80
:10719800DED0FBF79FFC144E054622681368DB0718
:1071A800D6D49368D9075FBF9368334043F001038F
:1071B8009360FBF78FFC401B0228EED923681B68FD
:1071C800DA07EAD4CBE7094B094A1B68B3FBF2F3A9
:1071D80001330193019B002BD8D0019B013BF8E7B9
:1071E8001700008000200140E8FFFF7F28080020EA
:1071F800400D030038B504460068FFF735FD054625
:1072080020BB94F85430012B20D0012384F854304B
:107218002046FFF795FFB0B9A36D226823F4706389
:1072280023F0010343F48073A3651C23E065136016
:1072380084F85400936823F0004323F0170343F0C5
:107248000403936038BD84F85450FBE70220F9E743
:10725800026838B5936891680446C80701D40020CD
:1072680038BD9907FBD4936803F00503012B19D1A6
:10727800936823F0004323F0170343F0020393605D
:1072880003231360FBF726FC054623689B68DB078E
:10729800E5D5FBF71FFC401B0228F6D923689B683D
:1072A800DA07F2D5A36D43F01003A365E36D43F04D
:1072B8000103E3650120D3E770B5044600284BD0ED
:1072C800836D43F002038365FFF70CFF054668B939
:1072D8002046FFF7BDFF054608B90123A3652268CC
:1072E800936823F0104323F01703936023685A68C8
:1072F80022F4677222F003025A6040F29F321A6049
:10730800D968164A0A40DA601A6922F040421A61BE
:107318005A6922F007025A611A6A02F0F0221A62C8
:107328005A6A02F0F0225A62DA6A02F0F022DA624D
:107338009A6A0B4A00269E62D2F8083723F0FE7339
:10734800C2F808372046FAF79DFDE6652666A66569
:1073580084F85460284670BD0125FBE700023E838F
:107368000020014010B590F85430012B044615D088
:10737800012380F85430FFF7B5FE58B92046FFF7CF
:1073880067FF38B9A36D23F4807323F0010343F03A
:107398000103A365002384F8543010BD0220FCE7E4
:1073A800F7B50023019390F85430012B04467FD0A1
:1073B800012380F85430FFF74BFF23689A6812F0D6
:1073C8000102054607D0A36D43F01003A36500230F
:1073D80084F854302DE0A16D364F21F4817141F0CD
:1073E8000201A165DE68D96826F4FF4626F07C060E
:1073F80021F40041360421F00301360CD96008203D
:107408009968394041F0004199609968002913DA78
:107418000199013101910199B1F52E3FF5D3A36D81
:1074280023F0120343F01003A365002384F85430BB
:107438000125284603B0F0BDD3F8B410013801F097
:107448007F010A44DCD199681A48014041F00101E2
:107458009960D3F8B41021F07F0141EAD202C3F851
:10746800B4209A68024042F002029A60FBF732FBAD
:10747800074623689A68D20708D4DA683243DA6084
:10748800A36D23F0030343F001039FE7FBF722FBFF
:10749800C01B0228EDD923689B68D907E9D5A36DDD
:1074A80043F01003A365E36D43F00103E365BFE711
:1074B8000225BEE7E8FFFF7F0749CA6822F4E062B9
:1074C8000302120403F4E063120C134343F0BF6396
:1074D80043F40033CB60704700ED00E0164B30B545
:1074E800DC68C4F30224C4F10703251D042B28BF5C
:1074F8000423062D4FF0FF358CBF033C002405FA0A
:1075080003F321EA0303A54022EA0502A340002869
:1075180043EA0203ACBF00F16040084A4FEA031394
:10752800B8BF00F00F00DBB2AABF00F561401354EA
:1075380080F8003330BD00BF00ED00E014ED00E03E
:10754800002807DB044A4109012300F01F0083409B
:1075580042F82130704700BF00E100E000280CDB52
:107568004309064900F01F0020330122824041F8F8
:107578002320BFF34F8FBFF36F8F704700E100E008
:1075880070B5D0E913456560446D14B1D0E916456E
:107598006560D0E9105404F01C060124B4406C6006
:1075A800046863608368102B0BBFA260A160E16070
:1075B800E26070BD0268416CD3B210B5083B142478
:1075C800B3FBF4F30B4CA24288BF0B4A21F0030132
:1075D80099BF01F1804202F50232521807338264E2
:1075E800064AC26403F01F03012202FA03F303658B
:1075F80010BD00BF070402401C080240800802407A
:1076080038B500285ED002682F4B9A424FF014011B
:107618004CD82E4B1344B3FBF1F32D499B00C0E922
:107628001013022380F825301368056923F4FF43FB
:1076380023F070031360D0E9024323432B434569C9
:1076480011682B4385692B43C5692B43056A2B4376
:107658000B431360FFF7AEFFB4F5804F04BF002360
:1076680043604268816C02F07F030B60D0E9131419
:10767800013A032A4C6020D8164A174981651A44F2
:10768800013B9200012103F0030301FA03F30021F7
:107698004265C3651160114A536400230122C36324
:1076A80080F8243080F82520184638BD0C4B134448
:1076B800B3FBF1F30B499B00B1E70023C0E9153395
:1076C800C365EAE70120F0E707040240F8FFFDBFC1
:1076D800000002403F8200104009024000090240B9
:1076E800F8FBFDBF0004024038B5002841D002680D
:1076F800136823F0010313601F4B9A424FF01401E3
:1077080030D81E4B1344B3FBF1F31D499B00C0E96D
:107718001013012403F01C0304FA03F30025156079
:107728004B60FFF747FF836C41681D60D0E9133257
:107738005A604A1E032A06D8124B0B449B009440F9
:107748001D60114B5C640023C363C0E91533C0E9B5
:107758000B33C0E90D33C36580F8253080F8243039
:10776800184638BD094B1344B3FBF1F308499B0095
:10777800CDE70120F5E700BF07040240F8FFFDBF91
:10778800000002403F82001000090240F8FBFDBFE4
:107798000004024070B590F82450012D04463BD0F7
:1077A80090F825600125AE4280F824504FF000067D
:1077B8002CD1022580F825500568C6632E6826F06E
:1077C80001062E60FFF7DCFE036BBBB12B6843F0AC
:1077D8000E032B60A36C1A68D20342BF1A6842F4E6
:1077E80080721A60636D1BB11A6842F480721A6065
:1077F8002B6843F001032B60002070BD2B6823F039
:1078080004032B602B6843F00A03E2E78023C36379
:1078180080F824602846F0E70220EEE7034640B1EE
:1078280090F82520022A06D00422C263002280F89C
:107838002420012070470268806C116821F00E0135
:107848001160016821F480710160116821F0010163
:107858001160D3E9100202F01C0101228A40426043
:10786800D3E9132151605A6D32B1116821F4807146
:107878001160D3E9162151600122002083F82520E8
:1078880083F82400704710B590F82530022B03D0F8
:107898000423C363012010BD03681A6822F00E0296
:1078A8001A601A6822F001021A60826C136823F4C5
:1078B80080731360D0E9101303F01C020123934076
:1078C8004B60D0E913325A60436D33B11A6822F421
:1078D80080721A60D0E916325A60012380F8253088
:1078E800836B002480F8244013B198472046D2E7E0
:1078F8001846D0E770B4426C046C036826681D68AB
:1079080002F01C020421914031420FD015F0040FFF
:107918000CD01A6892065EBF1A6822F004021A6038
:10792800036B6160002B33D070BC18470221914073
:10793800314217D015F0020F14D01A68940606D4F5
:107948001A6822F00A021A60012280F82520114ADA
:1079580093428CBF104B114B5960002380F82430A0
:10796800C36ADFE708219140314211D029070FD5BA
:10797800196821F00E011960012303FA02F262600E
:10798800C36380F82530002380F82430436BC9E7AF
:1079980070BC7047800002400004024000000240B2
:1079A8000A4A536943F4802330B55361EFF31084D6
:1079B80072B60023CD58C5500433B3F5807FF9D192
:1079C8001369DB03FCD484F3108830BD00400058F1
:1079D800064B5A69002ABFBF054A9A6002F18832ED
:1079E8009A60BABF5869C00F00207047004000581D
:1079F80023016745044B5A6942F000425A615869AD
:107A0800C043C00F704700BF0040005870B505461E
:107A1800FBF760F8124E04463369D90313D433696F
:107A2800DA0744BF012232614CF2FA32134011D115
:107A38000B4E306910F480200BD0FBF74BF8001B7D
:107A4800A842F6D304E0FBF745F8001BA842E3D3AD
:107A5800032070BD024A1361024A01205360F8E70F
:107A680000400058400F00202DE9F041184D98467D
:107A78002B78012B06460C46174626D001232B707F
:107A88004FF47A7000236B60FFF7C0FFA0B9012E96
:107A980016D1104A536943F0010353612760BFF3BD
:107AA8006F8FC4F804804FF47A70FFF7AFFF094A6C
:107AB800536923EA0603536100232B70BDE8F08164
:107AC80039462046FFF76CFFEDE70220F6E700BFD6
:107AD800400F002000400058054A536923F47E7384
:107AE80043EAC00040F4803040F002005061704723
:107AF800004000582DE9F041234F3B78012B054603
:107B080088463FD001233B704FF47A7000237B6096
:107B1800FFF77CFF044688B92B68042B13D11B4A56
:107B2800536943F4803343F0040353614FF47A708C
:107B3800FFF76CFF0446154B1A681B6800233B705F
:107B48002046BDE8F0814FF0FF33C8F800306E687A
:107B5800D5E901321344B3420AD93046FFF7BCFFD6
:107B68004FF47A70FFF752FF50B1C8F8006004462E
:107B7800064A536923F47E7323F002035361DAE75C
:107B88000136E5E70224DBE7400F002000400058FB
:107B98002DE9F04F524C00234FF00F090A6832FAD2
:107BA80003F501D1BDE8F08F012505FA03F818EABD
:107BB800020200F08E804E68032706F003054FEAA4
:107BC800430E07FA0EFC6F1E012F6FEA0C0C32D819
:107BD800876807EA0C0ACF6807FA0EF747EA0A0728
:107BE8008760476827EA0808C6F300179F4047EAF6
:107BF80008074760C76807EA0C088F6807FA0EF796
:107C080047EA0807022DC76017D14FEAD30800EBEF
:107C1800880803F0070AD8F820704FEA8A0A09FA98
:107C28000AFB27EA0B0B0F6907FA0AF747EA0B0763
:107C3800C8F8207001E0032DDCD1076805FA0EF5BD
:107C480007EA0C073D4316F4403F056041D023F096
:107C5800030707F1804707F5803703F0030CBD6879
:107C68004FEA8C0C4FF0070E0EFA0CFEB0F1904F55
:107C780025EA0E0E2FD01B4DA8422ED005F58065A3
:107C8800A8420CBF0225072505FA0CF545EA0E05A2
:107C9800BD602568D74316F4801F0CBF3D401543CF
:107CA8002560656816F4001F0CBF3D4015436560EC
:107CB800D4F8805016F4803F0CBF3D401543C4F8FB
:107CC8008050D4F88450B60354BF3D401543C4F8DF
:107CD8008450013362E70025D6E70125D4E700BFC9
:107CE8000008005800040048374A2DE9F04F0023E7
:107CF8004FF0010A4FF0070B4FF00F0931FA03F468
:107D080001D1BDE8F08F0AFA03FC1CEA010654D041
:107D180023F0030404F1804404F5803403F00307DE
:107D2800A568BF000BFA07F8B0F1904F08EA050EF6
:107D380045D0264DA84244D005F58065A8420CBF21
:107D480002250725BD40754517D1D2F8805025EA90
:107D58000605C2F88050D2F8845025EA0605C2F814
:107D68008450156825EA06051560556825EA060554
:107D78005560A56825EA0805A560056803265C0026
:107D880006FA04F423FA06F6254300EB8606056096
:107D980003F00705376AAD0009FA05F527EA050774
:107DA8003762856825EA04058560456825EA0C057B
:107DB8004560C56825EA0404C46001339EE70025D0
:107DC800C0E70125BEE700BF0008005800040048CE
:107DD8000369194214BF0120002070470AB181616C
:107DE8007047816270470000044AD168014208B5B3
:107DF80002D0D060FBF754FB08BD00BF0008005854
:107E080003689A69910744BF00229A629A69D20767
:107E18005EBF9A6942F001029A61704730B5039DCE
:107E280004682B4343EA0243064A6068C1F3090128
:107E38000B4342EA555223F0004320EA0200034371
:107E4800636030BDFF63FF0303682DE9F0419C695F
:107E580014F0100405460F4616466FD01022002471
:107E6800DA61A0462B689A69900661D4B8F1000FD0
:107E780035D044F0040401202E68B369D90541BF08
:107E88004FF48072F26144F0010401205A0541BFA9
:107E98004FF4806244F00804F26101209B054FD53D
:107EA8004FF4007344F00204F3612846FFF7A8FF7B
:107EB800736823F0FF7323F48B3323F4FF7323F0E9
:107EC800010373606B6C23436B64202385F8413096
:107ED800002385F8423085F84030012032E07A1CD2
:107EE800C1D0FAF7F7FD801BB84201D8002FB9D1ED
:107EF8002B68596895F8422098690004D2B20AD5CF
:107F0800490408D4202A06D05A6842F480425A60AC
:107F1800FAF7E0FD06462B689B699B06A2D4FAF7A0
:107F2800D9FD801B1928F6D920244FF0010899E7BC
:107F3800B8F1000F9DD12022DA619AE720469BE72D
:107F48000028B2D1BDE8F08170B504460D4616464A
:107F580023689B699B0701D5002070BD32462946DE
:107F68002046FFF771FFA0B96A1CF1D0FAF7B2FDFD
:107F7800801BA84201D8002DEAD1636C43F020038E
:107F88006364202384F84130002384F8423084F865
:107F980040300120E1E770B504460D4616462368D7
:107FA8009B695B070ED4324629462046FFF74CFFF3
:107FB80038BB23689A69910625D59A69520703D573
:107FC800228D0AB1002070BD9A6912F010021CBF00
:107FD8001022DA614FF0200118BF04226264D961CF
:107FE8005A6822F0FF7222F48B3222F4FF7222F0D8
:107FF80001025A60002384F8411084F8423084F862
:1080080040300120DFE7FAF765FD801BA84201D860
:10801800002DC4D1636C43F020036364202384F8EB
:1080280041300023EBE72DE9F041069F04468846DE
:1080380016461D462268936938EA03030CBF0123DC
:108048000023B34201D0002015E06B1CF3D0FAF7EF
:1080580041FDC01BA84201D8002DEBD1636C43F051
:1080680020036364202384F84130002384F84230DD
:1080780084F840300120BDE8F08170B504460D4613
:10808800164623689B699B0601D5002070BD3246C1
:1080980029462046FFF7D8FE90B9FAF71BFD801B4A
:1080A800A84201D8002DECD1636C43F0200363642F
:1080B800202384F84130002384F8423084F840308B
:1080C8000120E3E710B5044600284AD090F8413073
:1080D80003F0FF021BB980F84020FAF7F3F92423D4
:1080E80084F8413023681A6822F001021A60626835
:1080F80022F070621A619A6822F400429A60D4E908
:108108000221012924D142F400429A605A6842F0BF
:10811800007242F400425A60DA6822F40042DA60DF
:10812800D4E904210A43A16942EA0122DA60D4E9C8
:1081380007210A431A601A6842F001021A600020F7
:108148002023606484F84130206384F8420010BD25
:1081580042F4044202299A6004BF4FF400625A6054
:10816800D4E70120F3E700002DE9F347984690F89B
:1081780041300A9F202B04460E46914640F08680E7
:1081880090F84030012B00F081804FF0010A80F810
:1081980040A0FAF79FFC19230546009052464FF479
:1081A80000412046FFF73FFF18B1012002B0BDE8AB
:1081B800F087212384F84130102384F8423060642A
:1081C800A4F82A80638DC4F824909BB2FF2B6063C7
:1081D8002F4B26D9FF22228500934FF0807331461A
:1081E8002046FFF71BFE638D9BB22A463946204680
:1081F800FBB9FFF742FF0028D7D123682021D961B6
:108208005A6822F0FF7222F48B3222F4FF7222F0B5
:1082180001025A6084F8411084F8400084F8420052
:10822800C4E7628D009392B222854FF00073D2B2F8
:10823800D5E7FFF789FE0028B7D1636A226813F8EB
:10824800011B91626362638D228D013B9BB2638542
:10825800638D013A92B29BB22285002BC3D0002ACB
:10826800C1D100953B4680212046FFF7DCFE00285F
:108278009BD1638D9BB2FF2B03D9FF2222850090EF
:10828800ABE7628D009092B22285CEE702208DE79F
:10829800002000802DE9F347984690F841300A9F66
:1082A800202B04460E46914640F0878090F84030D7
:1082B800012B00F082804FF0010A80F840A0FAF705
:1082C80009FC19230546009052464FF40041204608
:1082D800FFF7A9FE18B1012002B0BDE8F0872223FC
:1082E80084F84130102384F842306064A4F82A806E
:1082F800638DC4F824909BB2FF2B6063304B26D962
:10830800FF22228500934FF0807331462046FFF705
:1083180085FD638D9BB22A4639462046FBB9FFF797
:10832800ACFE0028D7D123682021D9615A6822F0F1
:10833800FF7222F48B3222F4FF7222F001025A609B
:1083480084F8411084F8400084F84200C4E7628D44
:10835800009392B222854FF00073D2B2D5E7FFF7AF
:108368001AFE0028B7D123685A6A636A1A70636ACA
:10837800228D01336362638D013B9BB26385638DFC
:10838800013A92B29BB22285002BC2D0002AC0D1FA
:1083980000953B4680212046FFF745FE00289AD1EC
:1083A800638D9BB2FF2B03D9FF2222850090AAE799
:1083B800628D009092B22285CDE702208CE700BF43
:1083C8000024008010B590F84120202A0346D4B23A
:1083D8001CD190F84020012A18D0242280F841208E
:1083E8000268106820F001001060106820F48050C6
:1083F80010601068014311601168002041F001010C
:10840800116083F8414083F8400010BD0220FCE76A
:1084180010B590F84120202A0346D4B21BD190F819
:108428004020012A17D0242280F8412002681068D1
:1084380020F001001060106820F4706040EA01210B
:1084480011601168002041F00101116083F841407A
:1084580083F8400010BD0220FCE70000024A1368C0
:1084680043F4807313607047000400580D4B10B537
:108478005B690C4628B99A0507D500F027F820B1A2
:1084880010BD9B0501D400F019F8074A1369012CA7
:1084980023F00403136101D130BFF1E740BF20BFCF
:1084A80020BFEDE70004005800ED00E0024B18681B
:1084B80000F4C060704700BF00040058024A136807
:1084C80043F4804313607047000400580C4A136853
:1084D80023F4804313600B4B1B6832214B430A493A
:1084E800B3FBF1F35169890500D533B9536913F426
:1084F800007F14BF032000207047013BF2E700BF54
:10850800000400582808002040420F000B4A136856
:1085180023F0070343F002031360094B1A6901288B
:1085280042F004021A6105D130BF1A6922F0040230
:108538001A61704740BF20BF20BFF6E7000400580B
:1085480000ED00E04FF0B0431868C0F340407047BA
:108558004FF0B0431868C0F3400070474FF0B04286
:10856800536823F47F4343EA0023536070474FF076
:10857800B0431868C0F34060704700007FB54FF003
:10858800B0432C4AD3F80831C0F3031003F00F03AB
:1085980052F82040284A52F82330B4FBF3F4FFF78E
:1085A80085FF264B054693E80700B5F5007F04AB29
:1085B80003E9070010D0224B9C4218D303F5B703F8
:1085C80003F67F539C4229D903F5741303F510630E
:1085D8009C4225D802230BE01A4B9C4207D91A4B20
:1085E8009C421BD903F5370303F5D853F0E7002362
:1085F80004AA02EB830353F80C4C144D2B6823F0A8
:10860800070323432B60FAF765FA06462B6803F045
:1086180007039C4206D1002004B070BD0123E7E7A0
:108628000024EAE7FAF756FA801B0228EED903205D
:10863800F2E700BF903D0108303D0108F83B010812
:10864800C0CF6A00BFEA21013F93340200400058BE
:108658004FF0B04310B59A68D96812F00C0205D0F3
:108668000C2A4AD101F00303012B50D14FF0B0413D
:108678002B480B6813F0080306D00B6813F00803A7
:1086880037D1D1F8941007E00C68240756BFD1F809
:1086980094300968C3F3032350F82330002A0CBF31
:1086A800184600204FF0B0418A6802F00C020C2AEC
:1086B8001ED1CA6802F00302022A2ED0032A06D16C
:1086C8000B68184A13F4801F174B18BF13464FF056
:1086D800B042D068D168D268C0F306205843C1F3CD
:1086E80002130133B0FBF3F0530F0133B0FBF3F087
:1086F80010BD0B68C3F30313CEE7042A0AD0082A77
:1087080005D11B6813F4801304D10748CAE7002376
:108718001846C7E703480023C4E7024BD7E700BF62
:10872800903D01080024F4000048E80108B5FFF76F
:108738008FFF4FF0B043044A9B68C3F3031352F80A
:108748002330B0FBF3F008BD303D01082DE9F041BE
:108758000446002853D04FF0B0439D68DE68036894
:108768009B0605F00C0506F0030668D5026A1DB1E4
:108778000C2D46D1012E44D1002A40D04FF0B043F1
:10878800A16A1A68170756BFD3F894301B681B09EB
:1087980003F0F00399421FD90846FFF7EFFE0028BF
:1087A8002DD14FF0B042136843F0080313601368EB
:1087B800A16A23F0F0030B431360606AFFF7CEFE53
:1087C800FFF7B4FFAB4B1860AB4B1868FAF780F9AA
:1087D800002834D0BDE8F0814FF0B042136843F070
:1087E80008031360136823F0F0030B431360606AF7
:1087F800FFF7B4FE0846FFF7C1FE0028E0D00120CD
:10880800E8E74FF0B043002A54D01A6842F001025A
:108818001A60FAF75FF90746FFF79AFE002842D078
:108828004FF0B042136843F0080313601368A16A5D
:1088380023F0F0030B431360606AFFF78FFE236891
:10884800D80748D42368990700F18C8023681E074D
:1088580040F1FA80A3694FF0B046002B00F0E180A8
:10886800D6F89430E16903F01002914200F0C48018
:1088780003F00302022AC2D0D80740F1B380D6F829
:10888800943023F00103C6F89430FAF723F9074629
:10889800D6F89430990740F1A580FAF71BF9C31B65
:1088A800112BF5D904E0FAF715F9C01B0228B3D942
:1088B80003208FE71A6822F001021A60FAF70AF912
:1088C8000746FFF745FE0028B9D0FAF703F9C01BA1
:1088D8000228F6D9ECE7082D03D00C2D05D1032E7C
:1088E80003D16368002BADD189E74FF0B043A1688D
:1088F8001A6822F480120A431A606268B2F5803F4F
:1089080010D11A6842F480321A60FAF7E3F8074681
:10891800FFF718FE002895D1FAF7DCF8C01B642889
:10892800F6D9C5E7B2F5041F04D11A6842F400125B
:108938001A60E6E7196821F480311960196821F492
:1089480000111960002AE0D1FAF7C4F80746FFF7CA
:10895800F9FD00283FF476AFFAF7BCF8C01B64288D
:10896800F5D9A5E7042D236903D00C2D0ED1022ECD
:108978000CD1002B3FF443AF4FF0B042616953680C
:1089880023F0FE4343EA016353605FE74FF0B046CC
:10899800BBB1336843F480733360FAF79BF807463A
:1089A80033685A0507D57368626923F0FE4343EAC2
:1089B800026373604AE7FAF78DF8C31B022BEFD9FD
:1089C80076E7336823F480733360FAF783F8074651
:1089D80033685B057FF53AAFFAF77CF8C31B022BC7
:1089E800F6D965E74FF0B042E169D2F8943023F048
:1089F80010030B43C2F894304FF0B047D7F89430C7
:108A080043F00103C7F89430FAF764F80646D7F83C
:108A180094309A0718D4FAF75DF8831B112BF6D90E
:108A280046E7D6F8943023F00103C6F89430FAF7F5
:108A380051F80746D6F894309B0705D5FAF74AF857
:108A4800C31B112BF6D933E72368580754D50B4FAE
:108A58003B68D90514D4FFF701FDFAF73BF8064641
:108A68003B68DA050CD4FAF735F8831B022BF7D9E3
:108A78001EE700BF280800202C080020000400582A
:108A8800E3684FF0B046002B58D023F08003052B45
:108A980002BFD6F8903043F00403C6F890304FF088
:108AA800B046FAF717F8D6F8903043F001030746B6
:108AB800C6F8903041F28838D6F890309B0705D434
:108AC800FAF708F8C31B4345F6D9F1E6E36823F043
:108AD8000403812B1BD1F9F7FDFFD6F8903043F042
:108AE8008003C6F8903007464FF0B04641F2883808
:108AF800D6F89030180504D5E06A00284AD100203D
:108B080068E6F9F7E7FFC01B4045F1D9D0E6F9F769
:108B1800E1FFD6F8903023F08003C6F8903007467E
:108B28004FF0B04641F28838D6F890301905E3D5B1
:108B3800F9F7D0FFC01B4045F6D9B9E6F9F7CAFFE7
:108B4800D6F8903023F080030746C6F8903041F2FB
:108B58008838D6F890301A0516D4F9F7BBFFD6F83E
:108B6800903023F00103C6F8903007464FF0B04824
:108B780041F28836D8F890309B07BDD5F9F7AAFF9F
:108B8800C31BB342F6D993E6F9F7A4FFC01B4045CF
:108B9800DFD98DE60C2D4ED04FF0B04302281A686D
:108BA80022F080721A6033D1F9F794FF0546FFF777
:108BB800DEFC38BBD4E90C314FF0B0420B43D0682F
:108BC8002D4901400B43E16B0B43216C0B43616C56
:108BD8000B43A16B43EA0123D360136843F080730E
:108BE8001360D36843F08053D360F9F773FF0446EA
:108BF800FFF7BDFC002882D1F9F76CFF001B0A289B
:108C0800F6D955E6F9F766FF401B0A28CFD94FE693
:108C1800F9F760FF0446FFF7AAFC30B94FF0B042FD
:108C2800164BD1680B40D360D4E5F9F753FF001B0E
:108C38000A28F0D93CE601283FF4CCAD4FF0B04308
:108C4800226BDB6803F0030191427FF4D8AD616BBE
:108C580003F070028A427FF4D2ADA16B03F4FE42A6
:108C6800B2EB012F7FF4CBAD626C03F0604393420B
:108C78003FF445AFC3E500BF8C80C111FCFFFEEE99
:108C88002DE9F0410D46044610B90120BDE8F081F8
:108C9800684E336803F007038B4216D323689A079C
:108CA80027D54FF0B047A268BB6823F0F003134301
:108CB800BB60F9F70FFF0646BB68DB0319D4F9F769
:108CC80009FF831B022BF7D911E0336823F0070350
:108CD8000B433360F9F7FEFE0746336803F00703DA
:108CE800AB42DBD0F9F7F6FEC01B0228F5D903200A
:108CF800CCE72368580617D54FF0B0476269D7F814
:108D0800083123F00F0343EA1213C7F80831F9F7C3
:108D1800E1FE0646D7F80831D90305D4F9F7DAFE9B
:108D2800831B022BF6D9E2E723685A0713D54FF0C5
:108D3800B047E268BB6823F4E0631343BB60F9F70C
:108D4800C9FE0646BB689B0305D4F9F7C3FE831B1F
:108D5800022BF7D9CBE72368180714D54FF0B04793
:108D68002269BB6823F4605343EAC203BB60F9F786
:108D7800B1FE0646BB68590305D4F9F7ABFE831B61
:108D8800022BF7D9B3E72368DA070FD4294C2368F5
:108D980003F00703AB4239D8FFF7C8FC264B18602D
:108DA800264BBDE8F0411868F9F792BE6268022ABE
:108DB8001DD1FFF7C7FB00283FF467AF4FF0B0465F
:108DC80041F28838B36823F003031343B360F9F71B
:108DD80081FE0746B368626803F00C03B3EB820FA9
:108DE800D4D0F9F777FEC01B4045F3D97FE7032AB3
:108DF80002D1FFF7BCFBDEE712B9FFF7A9FBDAE700
:108E08004FF0B0431B685B05D8D43EE7236823F0D6
:108E180007032B432360F9F75DFE0646236803F03A
:108E28000703AB42B8D0F9F755FE801B0228F5D9E5
:108E38005DE700BF00400058280800202C080020EB
:108E480008B5FFF773FC4FF0B043044A9B68C3F3BF
:108E5800022352F82330D84008BD00BF703D0108F6
:108E680008B5FFF763FC4FF0B043044A9B68C3F3AF
:108E7800C22352F82330D84008BD00BF703D010816
:108E88004FF0B043D3F89000C0F3400070474FF064
:108E9800B0410209D1F8883002F47F22000123EAA8
:108EA800020300F47F200343C1F8883070474FF075
:108EB800B041020CD1F88830120423EA020343EAD5
:108EC8000040C1F88800704770B5066816F480360F
:108ED800044638D0FFF7C2FAF9F7FCFD614E0546A3
:108EE8003368DB0529D54FF0B043616BD3F8902088
:108EF80002F44072914214D0D3F89010D3F8902025
:108F080042F48032C3F89020D3F8902021F44070C6
:108F180022F480328D07C3F89020C3F8900000F146
:108F280090804FF0B042616BD2F8903023F44073D8
:108F38000B43C2F89030002605E0F9F7CBFD401B43
:108F48000228CDD903262568E8070AD54FF0B04195
:108F58006268D1F8883023EA124392B21343C1F809
:108F68008830A9070AD54FF0B041A268D1F88830F7
:108F780023EA124392B21343C1F88830AA0609D5EE
:108F88004FF0B0422169D2F8883023F440630B4394
:108F9800C2F88830AB0502D5206AFFF788FF68055C
:108FA80002D5606AFFF783FF290502D5A06AFFF79B
:108FB8007EFF6A0602D56069FFF769FF2B0602D5B6
:108FC800A069FFF764FFE80502D5E069FFF75FFFD6
:108FD800E90610D54FF0B042E168D2F8883023F4A2
:108FE80040730B43C2F88830B1F5807F02BFD36865
:108FF80043F08073D3602A040ED54FF0B042216B42
:10900800D2F8883023F040430B43C2F8883019B9AE
:10901800D36843F08073D3606B0410D54FF0B0422F
:10902800E16AD2F8883023F040530B43B1F1005F76
:10903800C2F8883003D1D36843F48033D360304614
:1090480070BDF9F747FD41F288360546FFF718FF6E
:1090580001283FF466AFF9F73DFD401BB042F5D952
:1090680070E700BF0004005830B590F82C30012B91
:1090780002464FF0020022D0174B82F82D00CA2476
:10908800012582F82C505C6253245C62B1F5807F24
:10909800146B996914D121F488519961596C24F0A1
:1090A800010421F0004159641463DD650A4BFF2176
:1090B80059620020012382F82D3082F82C0030BD3F
:1090C80021F408519961D96C24F0020421F000417F
:1090D800D9641463D865E9E70028004070B50B4EE1
:1090E800036B756D1D40EA07044603D50123F3653C
:1090F800F9F761FEAB0704D50223F365204600F0BB
:10910800CBF9012384F82D3070BD00BF0028004042
:1091180038B50A4CE36823F02003E360F9F7DAFC7A
:109128000546E3689B0601D5002038BDF9F7D2FC57
:10913800401BB0F57A7FF4D90320F6E700280040F9
:109148002DE9F041114DEC6814F0400407461AD19E
:10915800EB6843F08003EB60F9F7BCFC4FF00308C1
:109168000646EB685B0601D4032C02D12046BDE815
:10917800F081F9F7AFFC801BB0F57A7F84BF87F8E0
:109188002D800324EDE70024F0E700BF002800400D
:1091980038B50F4CE36823F08003E360A3699B06AE
:1091A800054606D4FFF7B4FF10B1032085F82D005B
:1091B80038BDA36923F02003A361FFF7A9FF10B10D
:1091C800032085F82D00A36943F02003A361EFE78E
:1091D8000028004038B5044600284BD090F82D30C0
:1091E80003F0FF021BB980F82C20F9F77BFA022361
:1091F800214D84F82D30EB68DB0632D4CA236B622C
:1092080053236B622046FFF79BFF78BBAB6923F0C3
:109218008E6323F04003AB6121696368AA690B433D
:109228001343A2691343AB61D4E9022343EA02431F
:109238002B61D4E90931EA680B4322F4F85213434D
:10924800EB602046FFF7A4FF80B9D4E90713AA69A9
:109258000B4322F06042134362691343AB61FF235F
:109268006B62012384F82D30002002E0024BFF22BC
:109278005A6238BD0120FCE7002800400023092875
:1092880003D840EA0310C0B270470A380133C0B2AD
:10929800F5E700002DE9F04790F82C30012B054642
:1092A8004FF0020069D0012385F82C304E4B85F829
:1092B8002D00DE6806F44076B6F5807F78D04C69DC
:1092C800087891F8019091F802A091F82470002A8A
:1092D80055D19B6913F0400308BFCB70FFF7CEFF51
:1092E80080464846FFF7CAFF02465046FFF7C6FFCA
:1092F80081463846FFF7C2FF0B6ACF78234343EA1B
:10930800875343EA090343EA084343EA022343EA4B
:109318000063354ACA205062532050628C6A8869BB
:10932800B4F5807F946945D124F48854946101246C
:10933800D465B6F5807F09BFCB69136403435364D2
:1093480018BF5064284B4A681A672A6B42F001021A
:109358002A639A6942F488529A61244AD2F8803082
:1093680043F40033C2F880301F4BFF225A620020BA
:10937800012385F82D3085F82C00BDE8F087B4F17D
:10938800803F07D0B4F5000F04D09B6913F0400369
:1093980008BFCB700B6ACA781C4344EA0A0444EA43
:1093A800004343EA092343EA825343EA0763B0E7E9
:1093B8000023AEE724F4085494610224D465B6F57A
:1093C800807F09BFCB6993640343D36418BFD0641B
:1093D800054B4A685A672A6B42F002022A639A6967
:1093E80042F40852B8E700BF0028004000080058BF
:1093F80090F82C20012A03464FF0020012D00A4AA6
:1094080083F82D00CA21516253215162916941F0BC
:1094180020019161FF2151620020012283F82D2053
:1094280083F82C00704700BF0028004090F82C20DB
:10943800012A03464FF0020019D00D4A83F82D0087
:10944800CA2151625321516291690A4841F0800151
:109458009161D0F8801041F48021C0F88010FF217C
:1094680051620020012283F82D2083F82C007047D8
:109478000028004000080058064B5A6D520610B5E7
:10948800044603D54022DA65F9F798FC012384F8ED
:109498002D3010BD002800407047890001F180413F
:1094A80001F531410A607047890001F1804101F5F9
:1094B8003141086870470000034AD2F8903043F4FD
:1094C8000043C2F89030704700040058034AD2F8AD
:1094D800903023F40043C2F89030704700040058DD
:1094E800074B1A6822F040021A6040F441704FF4AA
:1094F800B85218605A601A6842F040021A60704701
:109508000000015837B5054600284ED0837903F08E
:10951800FF046BB1032C0BD0254B4FF400629A610A
:109528002868FFF7DDFF002401232B71AC602FE0D2
:1095380000236B712846F9F7E5F91E4AD2F89030F6
:1095480043F48053C2F89030002CE5D102234FF049
:10955800B042AB71D2F8943023F40043C2F894308F
:10956800154B1B681C214B43DB0C64214B430193B7
:10957800019B93B90124AC60FFF79EFF0C4B9A68DE
:1095880042F400629A604FF400629A61002CC7D0DE
:109598000123AB71204603B030BD019B013B019311
:1095A800D2F894305B04E3D4E6E70124F2E700BF85
:1095B80000040058000800582808002037B5174D47
:1095C8002B6802461C204343DB0C642043431448A9
:1095D8000193019B93B901209060114C21732B6872
:1095E8001C214B43DB0C64214B430193019B6BB95A
:1095F800012090600A4BDB6803B030BD019B013B42
:10960800019383689C07E4D50020E6E7019B013BB2
:109618000193A368DB07E9D5ECE700BF2808002021
:109628000000015837B5184D2B6802461C204343EB
:10963800DB0C6420434315480193019BA3B9012027
:109648009060124CFF2323732B681C256B43DB0CA3
:1096580064256B430193019B73B9012090600B4B08
:10966800DB680B7003B030BD019B013B019383683D
:109678009C07E2D50020E4E7019B013B0193A36826
:10968800DB07E8D5EBE700BF2808002000000158F9
:109698000F4B13B51B680F4C182253431B0D642244
:1096A8005343014601936269019B02F0040223B906
:1096B80002238B60012002B010BD019B013B019386
:1096C800606910F00200F6D0002AECD11046F2E7EB
:1096D800280800200004005807B50379012B0FD192
:1096E8000A4B1B68182253431B0C0193FFF7EEFE2D
:1096F800019B013B0193019B002BF9D1FFF7DCFE95
:1097080003B05DF804EBFFF7C3BF00BF28080020D3
:10971800F8B51E468379012B154604460F46DAB282
:109728002DD14379012B2AD0022342718371FFF78F
:10973800D3FF0D212046FFF7C9FEFFF73FFF390A87
:109748002046FFF73BFFF9B22046FFF737FF2E44CC
:10975800B5420ED12046FFF7AFFEFFF799FFA0688C
:1097680001230038A3714FF0000318BF0120637173
:10977800F8BD15F8011B2046FFF720FFE8E7022097
:10978800F6E7F8B51E468379012B154604460F46C1
:10979800DAB22FD14379012B2CD04271FFF79CFF0D
:1097A8001D212046FFF792FEFFF708FF390A2046E1
:1097B800FFF704FFF9B22046FFF700FF002120461B
:1097C800FFF7FCFE2E44B5420ED12046FFF774FE8B
:1097D800FFF75EFFA06801230038A3714FF0000374
:1097E80018BF01206371F8BD29462046FFF71AFF0C
:1097F8000135E8E70220F6E7F8B51F468379012B23
:10980800154604460E46DAB22CD14379012B29D0ED
:109818004271FFF761FF06F0EF03A3F184025342A0
:109828005341237131462046FFF750FEFFF7C6FE2D
:109838002F44AF4210D1FFF73FFE842E02D02046BE
:10984800FFF726FFA06801230038A3714FF000033B
:1098580018BF01206371F8BD15F8011B2046FFF7FA
:10986800ADFEE6E70220F6E7F8B51E468379012B40
:10987800154604460F46DAB227D14379012B24D086
:109888004271FFF729FF39462046FFF71FFEFFF711
:1098980095FE00212046FFF791FE2E44B5420ED1D9
:1098A8002046FFF709FEFFF7F3FEA0680123003802
:1098B800A3714FF0000318BF01206371F8BD29465A
:1098C8002046FFF7AFFE0135E8E70220F6E737B597
:1098D8000023ADF8043001AA022312210546FFF740
:1098E800C3FFBDF80440022364BA01AAA4B2194612
:1098F8002846FFF781FFE20702D5284609F0F6F966
:10990800A30702D5284609F0F7F9600702D52846CB
:1099180009F01CFA210702D5284609F01DFAE206CB
:1099280002D5284609F01EFAA30602D5284609F0F2
:1099380007FA600602D5284609F0E4F9210606D59B
:1099480014F4807118BF0121284609F0E1F9A20535
:1099580002D5284609F0ECF9630402D5284609F037
:1099680007FA03B030BDF8B51E468379012B1546BA
:1099780004460F46DAB227D14379012B24D042712D
:10998800FFF7AAFE0E212046FFF7A0FDFFF716FEFF
:1099980039462046FFF712FE2E44B5420ED1204626
:1099A800FFF78AFDFFF774FEA06801230038A37152
:1099B8004FF0000318BF01206371F8BD15F8011BB3
:1099C8002046FFF7FBFDE8E70220F6E7F8B51E465C
:1099D8008379012B154604460F46DAB22BD1437919
:1099E800012B28D04271FFF777FE1E212046FFF792
:1099F8006DFDFFF7E3FD39462046FFF7DFFD002147
:109A08002046FFF7DBFD2E44B5420ED12046FFF776
:109A180053FDFFF73DFEA06801230038A3714FF006
:109A2800000318BF01206371F8BD29462046FFF7DF
:109A3800F9FD0135E8E70220F6E7026852E8003F41
:109A480023F0C00342E8003102680029F5D102F191
:109A5800080353E8003F23F4000302F1080C4CE824
:109A680000310029F3D12023C0F888307047000066
:109A780010B5026852E8003F23F4907342E80031C1
:109A880002680029F5D10F4C02F1080353E8003FA2
:109A9800234002F1080C4CE800310029F4D1C36ED0
:109AA800012B07D152E8003F23F0100342E80031B0
:109AB8000029F7D12023C0F88C300023C366436700
:109AC80010BD00BFFEFFFFEFF8B504461346D4F8FB
:109AD8008850202D32D1F1B1EAB1E06FA4F85620B8
:109AE800A4F8542000262122C4F890602165C4F807
:109AF8008820226888B1124FC762124F0763124F3D
:109B08002832C0E90D76FDF745FE30B11023C4F8C0
:109B18009030C4F8885001200FE0236840221A6270
:109B2800226802F1080353E8003F43F0800302F182
:109B3800080141E800300028F3D1F8BD0220FCE715
:109B4800559B00089D9B0008A99B000808B5034683
:109B5800806A1B681B6813F0200317D1A0F85630E1
:109B6800026802F1080353E8003F23F0800308323B
:109B780042E8003102680029F2D152E8003F43F080
:109B8800400342E800310029F7D108BDF9F76CFA23
:109B9800FBE7704708B5806AFFF7FBFF08BD704711
:109BA800806A38B50468D0F88830D0F88C50A2683C
:109BB800120606D5212B04D10023A0F85630FFF752
:109BC8003CFFA3685B0606D5222D04D10023A0F82C
:109BD8005E30FFF74DFFD0F8903043F01003C0F827
:109BE8009030FFF7DCFF38BD08B5806A0023A0F885
:109BF8005E30A0F85630FFF7D2FF08BD704700006E
:109C08000368D9691A682DE9F04140F60F06314218
:109C18009D68044610D18E0640F1978002F0200618
:109C280005F080573E4300F09080436F002B00F012
:109C38008580BDE8F0411847AB4EAC482E40104037
:109C4800304300F08280CF0709D5D00507D5012021
:109C58001862D4F8900040F00100C4F890008F0713
:109C680009D5E80707D502201862D4F8900040F01B
:109C78000400C4F890004F0709D5E80707D5042069
:109C88001862D4F8900040F00200C4F890000F0762
:109C98000BD502F02000304307D008201862D4F812
:109CA800900040F00800C4F890000E050AD5500155
:109CB80008D54FF400601862D4F8903043F02003C0
:109CC800C4F89030D4F89030002B37D08B0609D5E3
:109CD80002F0200205F080552A4303D0636F0BB1D0
:109CE800204698472668D4F89020B36802F02802E6
:109CF80003F0400353EA0205204621D0FFF7B8FEDF
:109D0800B3685F0617D5226802F1080353E8003FDD
:109D180023F04003083242E800310029F3D1D4F897
:109D2800800040B1724B8363FDF7ADFD30B1D4F8CC
:109D38008000836B7DE72046FFF731FFBDE8F081A7
:109D4800FFF72DFFC4F89050F8E7E06E012840F0C7
:109D58008980CE0640F18680D00640F183801022AB
:109D68001A629A6851064BD5D4F8802011684A685F
:109D780092B2002AE2D0B4F85C009042DED9A4F88E
:109D88005E200A6892062FD453E8002F22F48072CE
:109D980043E800210029F7D103F1080252E8002F17
:109DA80022F0010203F1080040E800210029F3D164
:109DB80003F1080252E8002F22F0400203F10800E4
:109DC80040E800210029F3D12022C4F88C20E16664
:109DD80053E8002F22F0100243E800210029F7D1B0
:109DE800D4F88000FDF71AFD02232367B4F85E302B
:109DF800B4F85C10C91A89B22046FFF7FFFE9DE748
:109E0800B4F85E20B4F85E00B4F85C1080B292B288
:109E1800002893D0891A89B200298FD053E8002FDF
:109E280022F4907243E800200028F7D1314D03F165
:109E3800080252E8002F2A4003F1080646E80020ED
:109E48000028F4D12022C4F88C206067E06653E82B
:109E5800002F22F0100243E800200028F7D1022347
:109E68002367C9E7CF0209D56E0207D54FF48012E0
:109E780020461A62BDE8F04100F0A0BD08060BD5E7
:109E880002F0800005F40005284305D0A36F002BDD
:109E98003FF454AF2046CCE64F0611D556060FD5F1
:109EA80053E8002F22F0400243E800210029F7D1AF
:109EB8002023C4F88830A1672046F9F7D5F83DE794
:109EC8000D0206D5500004D52046BDE8F04100F04B
:109ED80077BDCB017FF532AF002ABFF62FAF204602
:109EE800BDE8F04100F06BBD010000102001000446
:109EF800F19B0008FEFFFFEFD0F88C20B0F860104F
:109F0800222A08B5036855D15B6A826D0B4013702D
:109F1800836D01338365B0F85E30013B9BB2A0F8D6
:109F28005E30B0F85E309BB2002B42D1026852E836
:109F3800003F23F4907342E8003103680029F5D10B
:109F480003F1080252E8002F22F0010203F1080C85
:109F58004CE800210029F3D12022C0F88C20184AAF
:109F680041679342016705D1C26E012A0ED0F9F705
:109F780089F81EE05A681102F6D553E8002F22F03E
:109F8800806243E800210029F7D1EDE70022C2668C
:109F980053E8002F22F0100243E800210029F7D1EE
:109FA800DA69B0F85C10D20644BF10221A62FFF7D3
:109FB80025FE08BD9A6942F008029A61F9E700BFD8
:109FC80000800040D0F88C20B0F86010222A08B534
:109FD800036852D15A6A1140826D22F8021B8265C9
:109FE800B0F85E20013A92B2A0F85E20B0F85E2088
:109FF80092B2002A40D153E8002F22F4907243E82D
:10A0080000210029F7D103F1080252E8002F22F0BD
:10A01800010203F1080C4CE800210029F3D12022A9
:10A02800C0F88C20174A41679342016705D1C26E78
:10A03800012A0ED0F9F726F81EE05A681102F6D563
:10A0480053E8002F22F0806243E800210029F7D16D
:10A05800EDE70022C26653E8002F22F0100243E821
:10A0680000210029F7D1DA69B0F85C10D20644BFA4
:10A0780010221A62FFF7C2FD08BD9A6942F0080271
:10A088009A61F9E7008000402DE9F74F0368B0F8BE
:10A098006080DF691A689D68D0F88C1001922229C7
:10A0A800044640F0B480B0F86890DFF86CA1DFF89F
:10A0B8006CB10026B9F1000F01D0BB0621D4B4F869
:10A0C8005E309BB2D3B1B4F868209A4216D92268A0
:10A0D80002F1080353E8003F23F08053083242E8B6
:10A0E800003122680029F2D14D4B636752E8003FE6
:10A0F80043F0200342E800310029F7D103B0BDE85E
:10A10800F08F2368A26D5B6A03EA08031370A36DDE
:10A118000133A365B4F85E30013B9BB2A4F85E300E
:10A128002368DF6978072CD0F9070AD5019AD20588
:10A1380007D501211962D4F8901041F00101C4F843
:10A148009010B80709D5E90707D502211962D4F894
:10A15800901041F00401C4F890107A0709D5E80777
:10A1680007D504211962D4F8903043F00203C4F8EB
:10A178009030D4F8903023B12046FFF710FDC4F892
:10A188009060B4F85E309BB2002B93D1216851E8FF
:10A19800003F23F4807341E8003023680028F5D19C
:10A1A80003F1080252E8001F01EA0A0142E8001020
:10A1B8000028F5D120215B45C4F88C106067206722
:10A1C8000AD05968090207D553E8001F21F08061B9
:10A1D80043E800100028F7D1E16E012913D1E666A3
:10A1E80053E8001F21F0100143E800100028F7D1C0
:10A1F800D969CA0644BF102119622046B4F85C1018
:10A20800FFF7FCFC56E72046F8F73CFF52E79A694F
:10A2180042F008029A6171E7FEFFFFEF00800040FC
:10A22800019F00082DE9F74F0368B0F86080DF69E7
:10A238001A689D68D0F88C1001922229044640F0D3
:10A24800B280B0F86890DFF868A1DFF868B100263E
:10A25800B9F1000F01D0BB0621D4B4F85E309BB22F
:10A26800D3B1B4F868209A4216D9226802F10803DB
:10A2780053E8003F23F08053083242E80031226857
:10A288000029F2D14C4B636752E8003F43F02003AA
:10A2980042E800310029F7D103B0BDE8F08F236808
:10A2A800A26D596A08EA010122F8021BA265B4F8F6
:10A2B8005E20013A92B2A4F85E20DF6978072CD0BC
:10A2C800F9070AD5019AD20507D501211962D4F8F0
:10A2D800901041F00101C4F89010B80709D5E907BA
:10A2E80007D502211962D4F8901041F00401C4F88E
:10A2F80090107A0709D5E80707D504211962D4F820
:10A30800903043F00203C4F89030D4F8903023B171
:10A318002046FFF744FCC4F89060B4F85E309BB266
:10A32800002B95D1216851E8003F23F4807341E860
:10A33800003023680028F5D103F1080252E8001F15
:10A3480001EA0A0142E800100028F5D120215B4506
:10A35800C4F88C10606720670AD05968090207D5CD
:10A3680053E8001F21F0806143E800100028F7D16E
:10A37800E16E012913D1E66653E8001F21F01001B0
:10A3880043E800100028F7D1D969CA0644BF102154
:10A3980019622046B4F85C10FFF730FC58E72046F5
:10A3A800F8F770FE54E79A6942F008029A6173E779
:10A3B800FEFFFFEF00800040CD9F000838B504463F
:10A3C80003682169A2681D68C0690A4361690A4374
:10A3D8007D49024329400A431A605A68E16822F419
:10A3E80040520A435A60794AA16993421CBF226AC3
:10A3F80011439A6822F06E4222F430620A439A604E
:10A40800DA6A616A22F00F020A43DA62704A9342FA
:10A418001CD14FF0B043D3F8883003F0030343F462
:10A428004033A3F54033013B022B00F2C780694A51
:10A438009B5CB0F5004F40F08980082B24D8DFE8FA
:10A4480003F061C08323802323236500624A93427B
:10A4580009D14FF0B043614AD3F8883003F00C03B8
:10A4680043F44023E4E7594A93420DD14FF0B043F7
:10A47800D3F8883003F44063B3F5006F1AD005D8D9
:10A4880053B1B3F5806F12D0012009E0B3F5406FE6
:10A49800FAD14FF400400EE0FEF7D2FC58B9002084
:10A4A8004FF00113A3660023C4E91D3338BDFEF73E
:10A4B800CFF8F3E74A4865684A4B626A05EB4501FD
:10A4C80033F81220B0FBF2F39942DDD8B3EB053F25
:10A4D800DAD800231946F7F717FB090241EA106199
:10A4E8006B080002C0182A464FF0000341F1000132
:10A4F800F7F70AFB3C4BA0F540729A42C4D8236890
:10A50800D860CCE7FEF79CFC0028C8D06168354BC2
:10A51800626A33F81220B0FBF2F24B0803EB4203F5
:10A528004FF6EF72B3FBF1F3A3F110019142ABD8F0
:10A5380023F00F02216892B2C3F342031343CB60A6
:10A54800ADE7FEF785F8DFE72548DFE7082B9BD85E
:10A5580001A252F823F000BFA9A50008B5A500087C
:10A56800C1A5000891A40008BBA5000891A4000893
:10A5780091A4000891A4000885A500084FF40040A4
:10A588006368616A174A32F81120B0FBF2F000EBF9
:10A598005300B0FBF3F04FF6EF73A0F11002ACE7F5
:10A5A800FEF74EFC00283FF47AAFE9E7FEF758FCC7
:10A5B800F8E7FEF74DF8F5E70948E1E7B0F5004F91
:10A5C800F4D1FEF74DFC9FE7F369FFCF0080004010
:10A5D80000380140D03D010800440040D33DF50754
:10A5E8000024F400E03D0108FFFC0F00836ADA074D
:10A5F80010B506D50168C46A4A6822F400322243BD
:10A608004A609C0706D50168046B4A6822F48032C8
:10A6180022434A60590706D50168446B4A6822F408
:10A62800802222434A601A0706D50168846B4A686B
:10A6380022F4004222434A60DC0606D50168C46B56
:10A648008A6822F4805222438A60990606D50168F6
:10A65800046C8A6822F4005222438A605A060FD595
:10A668000168446C4A6822F480122243B4F5801FC2
:10A678004A6005D14A68846C22F4C00222434A60C9
:10A688001B0606D50268C16C536823F400230B43EC
:10A69800536010BD2DE9F041DDF8188004460E46E0
:10A6A80015461F462268D36936EA03030CBF012307
:10A6B8000023AB4201D0002027E0B8F1FF3FF2D0E1
:10A6C800F8F708FAC01B4045206802D8B8F1000F17
:10A6D8001DD150E8003F23F4D07340E80032002A2F
:10A6E800F7D100F1080353E8003F23F0010300F11C
:10A6F800080141E80032002AF3D12023C4F8883049
:10A70800C4F88C3084F884200320BDE8F081036805
:10A718005A07C7D5C3691B05C4D54FF40063036244
:10A7280050E8003F23F4D07340E80032002AF7D104
:10A7380000F1080353E8003F23F0010300F108018A
:10A7480041E80032002AF3D12023C4F88830C4F845
:10A758008C30C4F89030D5E773B504460026C0F8AD
:10A768009060F8F7B7F923681B681A07054619D4EB
:10A7780023681B685B070AD56FF07E4300930022AD
:10A788002B464FF480012046FFF784FFB0B9002024
:10A798002023C4F8883084F88400C4F88C30E0663C
:10A7A80020670CE06FF07E430093324603464FF477
:10A7B80000112046FFF76EFF0028D9D0032002B011
:10A7C80070BD10B5044650B3D0F888301BB980F876
:10A7D8008430F8F735FB22682423C4F888301368DE
:10A7E80023F0010313602046FFF7E8FD012816D087
:10A7F800A36A13B12046FFF7F9FE23685A6822F4CA
:10A8080090425A609A6822F02A029A601A6842F0C6
:10A81800010220461A60BDE81040FFF79DBF0120E5
:10A8280010BD000030B581658168A0F85C20002368
:10A83800B1F5805FA0F85E20436735D10369002B2E
:10A8480040F2FF1318BFFF23A0F860300023C0F8C0
:10A8580090302223C0F88C30016801F1080353E8D6
:10A86800003F43F00103083141E800340368002C3D
:10A87800F2D1456E84680169B5F1005F34D1B0F852
:10A888006850954230D8B4F5805F1DD1254A264CD2
:10A89800002918BF22464267C1B153E8002F42F48D
:10A8A800807243E80021F7E729B90369002B14BF38
:10A8B8007F23FF23C8E7B1F1805FC5D10369002B6F
:10A8C8000CBF7F233F23BFE7174AE4E703F10802E1
:10A8D80052E8002F42F0805203F1080040E80021BE
:10A8E8000029F3D1002030BDB4F5805F0FD10F4AA5
:10A8F8000F4C002918BF2246426751B153E8002F78
:10A9080042F4907243E800210029F7D1EAE7084AA7
:10A91800F2E753E8002F42F0200243E80021002923
:10A92800F7D1DFE72DA2000891A00008CD9F00080D
:10A93800019F0008D0F88C30202B30B415D1B9B164
:10A94800B2B100230468C3660A4B9C420AD063680C
:10A958001B0207D554E8003F43F0806344E8003504
:10A96800002DF7D130BCFFF75DBF022030BC704727
:10A978000120FBE700800040436E30B52BB901236E
:10A98800A0F86A30A0F8683030BD0368094D9A68AD
:10A998009968094C490FC2F342626B5C615CDB0049
:10A9A800B3FBF1F3A0F86A30AB5CA25CDB00B3FB4D
:10A9B800F2F3E7E7003E0108F83D010870477047E9
:10A9C80070471FB504AB03E9060090F88430012BEB
:10A9D80004463AD0012380F884302423C0F8883014
:10A9E80003681A6822F001021A609A6822F4401279
:10A9F8000A439A6071B95A68BDF80C009DF80E10A8
:10AA080022F0100202435A605A6822F07F4242EA5A
:10AA180001625A601A6842F001021A60F8F75AF89F
:10AA28006FF07E42034600924FF4800100222046D8
:10AA3800FFF730FE38B92023C4F88830002384F8A3
:10AA4800843004B010BD0320F8E70220F9E790F83D
:10AA58008430012B0FD0012380F88430016851E83D
:10AA6800002F42F0020241E80023002BF6D180F8C3
:10AA78008430184670470220704710B590F884302B
:10AA8800012B044617D02423C0F8883003681A68BD
:10AA9800196821F00101196042F000524FF000518D
:10AAA80041661A60FFF768FF2023C0F8883000204D
:10AAB80084F8840010BD0220FCE770B590F884305B
:10AAC800012B044617D005682423C0F888302E6867
:10AAD8002B6823F001032B60AB6823F06043194314
:10AAE800A960FFF749FF20232E60C0F888300020B6
:10AAF80084F8840070BD0220FCE770B590F88430BB
:10AB0800012B044617D005682423C0F888302E6826
:10AB18002B6823F001032B60AB6823F060631943B3
:10AB2800A960FFF729FF20232E60C0F88830002095
:10AB380084F8840070BD0220FCE7000038B5094D98
:10AB4800002455F8043B33B90134E3B2052B64B251
:10AB5800F7D1002038BD002CF6D01B699847002893
:10AB6800F2D0F7E7701000207FB50A2301A88DF80E
:10AB7800043003F0D9F80038044B059A1A6018BF5E
:10AB88000120404207B05DF804FB00BF68100020B8
:10AB980070B504460B46144962784A700020A278C2
:10ABA8000A7208701A884A729A788A72DB780B746B
:10ABB8006368CB600D4B1B68DA6A2AB1237803F00F
:10ABC800FB030B2B00D09047094E002556F8043B99
:10ABD8001BB19B6A0BB1204698470135EBB2052B98
:10ABE8006DB2F3D170BD00BF480800206C10002082
:10ABF8007010002070B50446114801230370637873
:10AC08004370A3788372E368C360E37803762369AB
:10AC18004376237943720B4B1B689B6A03B19847B1
:10AC2800094E002556F8043B1BB1DB690BB12046E1
:10AC380098470135EBB2052B6DB2F3D170BD00BF5B
:10AC48005C0800206C1000207010002038B501F05E
:10AC580011FE0C4D052455F8043B5BB15B694BB103
:10AC680055F8043C9B682BB1984718B155F8043C3B
:10AC78005B699847013C14F0FF04ECD1BDE838400B
:10AC8800FFF75CBF70100020014B1868704700BFC9
:10AC98006810002000B58BB0012368468DF800309D
:10ACA80002F0BCFC38B99DF80400003818BF012038
:10ACB8000BB05DF804FB0020FAE7000030B58BB05C
:10ACC800054601F0BBFD0446002839D1FFF7E2FF35
:10ACD800012838D168468DF8004002F09FFC10B179
:10ACE8004FF0FF3004E09DF80430AB4202D1002061
:10ACF8000BB030BD012DF3D0022D11D0002DF7D1AE
:10AD0800002BF4D068468DF8045002F099FD002815
:10AD1800E6D10E4B1B681B6B002BE8D09847E6E783
:10AD2800002BDDD168468DF8045002F089FD00281B
:10AD3800D6D1064B1B681B6B002BD8D02846EDE7F5
:10AD48006FF00100D4E76FF00200D1E76C1000202B
:10AD580070B5324C324B94F9042094F9055090B0F8
:10AD6800012602288DF804608DF809208DF80A5014
:10AD78000AD18DF80800D871197202F09FFB01A85A
:10AD880002F0D2FF10B070BD4FF480701A715D717F
:10AD9800D8801972234B8DF808601B7853BB1E238B
:10ADA80006A88DF81C208DF8183002F049FD1F23E5
:10ADB8008DF8183006A823798DF81C3002F040FD74
:10ADC80021238DF8183006A863798DF81C3002F01D
:10ADD80037FD20238DF8183006A863798DF81C30CC
:10ADE80002F02EFD28238DF8183006A80E4B079385
:10ADF80002F026FD02F062FB012306A88DF8183048
:10AE08008DF81C3002F01CFD084B1B685B6A0BB107
:10AE1800034898476078FFF751FFB3E78410002094
:10AE28003008002064100020000300016C1000208E
:10AE380008B501F003FD40B9FFF72CFF012806D043
:10AE4800084B197AD879FFF783FF012008BD064B14
:10AE58001B68DB6898470028F7D1BDE80840FFF772
:10AE68006DBE00BF30080020701000202DE9F041B1
:10AE780086B005460C46164601F0E0FC002840F076
:10AE88008D8001F0EDFC40B9FFF704FF012807D0E1
:10AE9800444B197AD879FFF75BFF6FF002046DE035
:10AEA800414F3B68DB68984730B13A682B78127895
:10AEB8009A4201D0002B6ED13C4FDFF8F4803C72EF
:10AEC800003C18BF012498F8043068788DF80440D5
:10AED80069468DF8123002F049FB002840D0002363
:10AEE8008DF804300393ADF810306FF0060495E840
:10AEF8000300304B83E8030098F80430BB723146F6
:10AF080001A803F009F82C4B059A1A6011283FD8BC
:10AF180001A353F820F000BF7FAF0008A5AF0008D9
:10AF280099AF000899AF000899AF000899AF0008D9
:10AF380099AF0008A3AE000899AF000899AF0008C0
:10AF480099AF000893AF000899AF000899AF0008BF
:10AF5800A5AF0008A5AF0008A5AF00088DAF000891
:10AF68002B788DF808306B78ADF810306B68039348
:10AF78004FF0FF34BBE7E31D18BF0024204606B09E
:10AF8800BDE8F0816FF00404F8E76FF00504F5E719
:10AF98004FF0FF34F2E76FF00304EFE76FF00104BE
:10AFA800ECE700BF30080020701000205C0800208B
:10AFB800841000206C0800206810002010B504469A
:10AFC8008AB018B94FF0FF300AB010BD00236846A8
:10AFD8008DF8003002F022FB0028F3D19DF80430F0
:10AFE8002370F1E7F0B587B000220B462A498DF8A7
:10AFF800072001220A7042784A700446002A41D18B
:10B0080002790A721A884A729A788A72DB780B7403
:10B018000369CB60C378214D8DF80830037B8DF828
:10B028000930836803932B68DB6A0BB102A8984741
:10B038002B689B6B13B1227E02B19847184E0025EE
:10B04800374656F8043B53B11A6A42B11A78E37886
:10B058009A4219D156F8043C20461B6A9847013594
:10B06800EBB2052B6DB2ECD10DF10700FFF7A6FF8F
:10B0780063793BB10021012204A8ADF810100591B5
:10B08800FFF7F4FE07B0F0BD002DE8D13B68DB68A0
:10B0980098470028DED1E2E7480800206C1000201D
:10B0A8007010002010B504468AB018B94FF0FF3070
:10B0B8000AB010BD1F2368468DF8003002F0AEFAC2
:10B0C8000028F3D1024A9DF9043023701371EFE789
:10B0D8008410002000B58BB02223019068468DF8BB
:10B0E800003002F0ADFB003818BF012040420BB021
:10B0F8005DF804FB70B5634C014618228EB02046FB
:10B1080005F066FFF8F73EFF23784068012202FA4F
:10B1180003F1014004D15C4B084607F04FFFFEE7FE
:10B128005A495B481A4602F011F818B14FF0FF303F
:10B138000EB070BD262304A88DF8103002F080FBF5
:10B14800544E554D002870D1012333702B68DB69AC
:10B158000BB100209847262304A88DF8103002F080
:10B168005DFA059B93F84820227093F8182193F80C
:10B178001A316270A370454BD3E9020105F01AFE3B
:10B1880005460028D2D1454E062304A88DF8103074
:10B1980002F044FA059B736104A802F051FB0223F4
:10B1A80004A88DF81030059602F038FA0836032303
:10B1B80004A88DF81030059602F030FA0F2605F035
:10B1C800BDFE012304A88DF814308DF8106002F03C
:10B1D80037FB10230DEB03008DF810308DF8145059
:10B1E80002F02EFB04238DF8103004A8A3788DF804
:10B1F800143002F025FB39238DF8103004A8636958
:10B20800059302F01DFB02A920788DF8086003F071
:10B2180051FF003818BF0120E0711420FFF75AFFD2
:10B22800E07903F003F8284682E727238DF81030E9
:10B238002B681B6943B104A802F0F0F92B68059844
:10B248001B694FF4EE619847262304A88DF8103047
:10B2580002F0F6FA50B9012304A88DF8103002F074
:10B26800DDF99DF81430002B7FF46EAF3378002B96
:10B278007FF46CAF052204A88DF81020059302F026
:10B28800DFFA78E784100020083E01089C100020AF
:10B29800B4100020641000206C1000204C10002016
:10B2A80037B500230D4601930446C0B900F0D0FA23
:10B2B8000190019BC3B10E4A0E4942F824300E4A50
:10B2C800DA620E4A1A630E4A5A630E4A1268926983
:10B2D8009A6128465B68F2229847002006E001A997
:10B2E80000F0BCFA0028E4D04FF0FF3003B030BDC6
:10B2F80070100020580F002059AD000875AE0008E6
:10B3080071AB00086C100020154B07B51860154B81
:10B31800154A1A60154A5A60154A9A60154ADA6041
:10B32800154B02681A6042685A6082689A60C2685F
:10B33800DA60124A01911A61114982695A61002042
:10B34800FFF7AEFF48B901A800F086FA003818BF29
:10B358000120404203B05DF804FB4FF0FF30F9E7ED
:10B368006C100020B4100020FDAB0008EDAF000801
:10B3780009B4000899AB00089C1000206DF0000883
:10B388003C08002051B118B1012804D000207047B2
:10B39800044B0B607047044B0B60F7E74FF0FF302E
:10B3A800704700BF000300010300010108B502F067
:10B3B80059FF002814BF6FF00100002008BD08B530
:10B3C80002F0A4F8002814BF6FF00100002008BDA7
:10B3D80010B504468AB018B94FF0FF300AB010BD56
:10B3E800202368468DF8003002F018F90028F3D1C0
:10B3F800024A9DF9043023705371EFE7841000204E
:10B408002DE9F0412F4D304F00232B7043786B709E
:10B418003B689B6A8AB004460BB128469847DFF818
:10B42800AC80002658F8043B1BB15B6A0BB1204680
:10B4380098470136F3B2052B76B2F3D12378052B62
:10B448002FD00C2B35D0012B25D1214C0623684653
:10B458008DF8003002F0E2F80199E07905F0F0FC8F
:10B4680010B91C4B019A5A611B48FFF71BFE1B4879
:10B47800FFF7AEFF6B788BB9A371194B5878FFF7BC
:10B488001DFC3B685B6A0BB1114898476B7813B990
:10B49800E07905F065FD0AB0BDE8F081FF23A371EE
:10B4A800EFE7104B01225A74227A9A74627ADA749E
:10B4B800F1E76378002BEED00AB0BDE8F041FFF762
:10B4C80053BB00BF5C0800206C10002070100020E7
:10B4D800300800204C1000203408002035080020D7
:10B4E800841000204808002030B58BB0FFF767FFB4
:10B4F8000446F0B903F0BEFD831C1DD0F8B9134D06
:10B508002B685B69DBB1262368468DF8003002F0B2
:10B5180085F82B6801985B694FF4EE61984703F052
:10B52800BBFD78B92CB9094B1B68DB690BB101204D
:10B53800984720460BB030BD6FF00704EFE74FF097
:10B54800FF34ECE74FF0FF34F3E700BF6C10002046
:10B5580030B5064D064C30B129B12860A160627142
:10B568000123237030BD00232B60FAE7F010002080
:10B57800C4100020014B1878704700BFC410002089
:10B58800024B187800B15878704700BFC4100020EB
:10B5980070470000064B1A784AB15A783AB10278D7
:10B5A800012A04D1027912B19A8901329A8170472D
:10B5B800C4100020074B1A7852B15A7842B1027869
:10B5C800052A05D1017A427AD973012098731A7431
:10B5D800704700BFC410002013B51A4C23783BB342
:10B5E80063782BB3A27BA36862B10022A273032203
:10B5F800A27105221A70E27B5A70227C9A7001228D
:10B60800A27004E0A278012A14D0042AF7D0E0221C
:10B618008DF800200C48A27901938DF8012008F0DC
:10B6280049F80A4B1B6B1BB1E17801226846984721
:10B6380002B010BD0222A271A2895A70110A1970B3
:10B64800E5E700BFC4100020D810002078080020CB
:10B65800FFF7C2BF30B5794C23788DB0002B43D0AB
:10B66800437B002B40D0657825B1837B13B9A38930
:10B678000133A381C178E02936D1002D36D1027B70
:10B68800042A31D18368187801282DD158780128E7
:10B698002AD19878012827D1DB78012B24D10220E0
:10B6A8006380A071E56002A863708DF80C30217189
:10B6B8008DF80820257402F0C3F8284602F0B6FD7C
:10B6C8005F4B1B685B6803B1984700225D4B009293
:10B6D8004FF0FF315C4807F041FF41F288315A488A
:10B6E80008F022F8FFF778FF0DB030BD83681A78AC
:10B6F800A2700A2AF8D8DFE802F0062124282A3D99
:10B7080044658D8F9900504807F086FF00236370C9
:10B71800A3814B4C04238DF80830236802A81B78BA
:10B728008DF80C3002F08CF82368587802F07EFD12
:10B7380023689B68002BD7D09847D5E70223A371CD
:10B74800D2E740F201136380CEE70123FBE7A56847
:10B75800037BA37104222A7062799A4228BF1A4691
:10B7680000230133D9B28A42BED98168C95C01314C
:10B77800E954F6E705238DF8083002A802F0D4FA58
:10B78800B2E7314807F048FF00236370A3812C4CCF
:10B7980004238DF80830236802A81B788DF80C3034
:10B7A80002F04EF82368587802F040FD23689B6841
:10B7B80003B19847254BDB6A002B95D00121022065
:10B7C800984791E7027B032A0DD106228DF80820BD
:10B7D800B3F801305BBAADF80C3002A802F0A4FA55
:10B7E8000123A37080E7072AF7D18DF80820B3F862
:10B7F800012052BAADF80C201A79D978120242EA1F
:10B80800014259790A4364214A4304929B798DF88D
:10B818001430E2E70A23AEE700228DF808205B78AF
:10B828008DF80C3002A802F00BF85DE70D228DF8B8
:10B8380008205B788DF80C309FE700BFC41000200B
:10B84800F010002059B60008D81000207808002011
:10B858000048704778080020002070474FF0FF30FC
:10B8680070470000044B054A93F81831022B18BFA3
:10B87800062382F88034704764180020D81F0020FF
:10B88800034BD3F8483313B15B6903B118477047CA
:10B89800D81F0020034A137843F002031370FFF700
:10B8A800EFBF00BFD41F00201FB50A4B8DF8090059
:10B8B80093F87C208DF80A2093F88C2093F84800A0
:10B8C8000D3202A98DF8082003F0F4FBC0B205B0D0
:10B8D8005DF804FB6418002010B50D4C04F57D706C
:10B8E80007F09AFE94F8103413B1012384F80F344A
:10B8F800084B93F81831022B02BF94F8813443F0B7
:10B90800100384F88134BDE81040FFF7B9BF00BFC9
:10B91800D81F00206418002010B50C4CD4F8403310
:10B9280043F08003C4F8403394F8103413B1002076
:10B93800FFF7D2FF94F8813423F0120343F0120387
:10B9480084F88134BDE81040FFF78CBFD81F002071
:10B958002DE9F0412C4D95F81831022B07460E467B
:10B9680002D02A4BDB6A984702F01BFD044628B137
:10B97800022002F00CFD002002F00EFD95F81831AF
:10B98800012B17D102F00FFD804630B1002002F0E4
:10B99800FFFC002002F001FD444602F006FD48B11C
:10B9A800002002F0F6FC002002F0F8FCBDE8F041AF
:10B9B800FFF758BF002CF9D1154C94F8802494F85F
:10B9C8001034B2B90BB184F83574384602F090FEE1
:10B9D800E86A07F0E7FDD4F8B4339842E6D30D4897
:10B9E80007F01AFE94F8813443F0100384F8813488
:10B9F800DCE70BB184F83564304602F079FE95F83F
:10BA08001831022BEED1D1E7641800201445010843
:10BA1800D81F002070230020074A10B5137843F080
:10BA280001031370FFF72CFFBDE81040034B012200
:10BA38000021022007F0C2BAD41F0020513E01089D
:10BA4800074A10B5137843F004031370FFF718FF83
:10BA5800BDE81040034B01220021022007F0AEBAD6
:10BA6800D41F0020613E01082DE9F0410F4616461B
:10BA78001D46804607F08CFD0A4A0B4C1378278137
:10BA880043F00803C4E90008137066812573FFF7C3
:10BA9800F7FEBDE8F041054B01220021022007F026
:10BAA8008DBA00BFD41F0020E0240020713E010899
:10BAB80013B507F06DFD0D4B6C461860204607F076
:10BAC800BBFC94E803000A4A0A4B83E80300137896
:10BAD80043F010031370FFF7D3FE074B0122002138
:10BAE800022002B0BDE8104007F068BAF024002038
:10BAF800D41F0020102300207E3E01082DE9F041CC
:10BB080092B0064602F04DFC002840F05681AC4D3C
:10BB180095F81831012B09D02B6BAA4C93B194F8E6
:10BB28000431BBB1042B6FD0032003E002F03BFCCF
:10BB380018B10F2012B0BDE8F08102F036FC0028E1
:10BB4800EAD0F6E7B5F81E31D4F81424013B534384
:10BB58002B63E4E79C4803F0E4F9002840F02981CE
:10BB680094F80C3123802B6B0C930DF1180895F881
:10BB780039308DF83830404695F81C318DF83A3018
:10BB880007F080FCD5F82431009302AF98E806004E
:10BB9800D5F82031384607F00CFC97E803000FABC6
:10BBA80083E80300EB6A0D9300238DF84430238863
:10BBB800ADF8463095F82C3101228DF839201BB9A3
:10BBC8008DF844208DF83930804B0093804B95F8E0
:10BBD8004800A3F173020CA903F0E1FAC0B10B28E5
:10BBE800A8D1D4F8841499B1002EA3D0D4F8403346
:10BBF800784843F02003C4F8403307F095FD7548B2
:10BC080007F058FD002095E76F4803F0BEF9A4E758
:10BC180095F8487095F9693095F9392095F87D10AF
:10BC28006D4E384603F0CDFA009641B2EB6C95F8AC
:10BC380050203846143603F063FA0096EB6C95F8FA
:10BC4800502095F9701095F8480003F059FAD4F887
:10BC5800C413AB6DD4F8D8230B44C4F8B033EB6DE0
:10BC68001344C4F8B43394F80431042B07D02B6E72
:10BC78000B44C4F8B0336B6E1344C4F8B4330023D8
:10BC8800089395F82C3183B108A802F061FC0028CC
:10BC98004AD195F9390094F837629DF82070FFF77A
:10BCA80003FE3E4480B2B0423CD300238DF81330EB
:10BCB80095F839308DF8213095F838308DF82230E4
:10BCC800D5F880300993D5F884300A93238894F8FE
:10BCD8001164ADF82C3095F84800404B8DF8206081
:10BCE8000DF1130208A903F01FFA012384F8353473
:10BCF80095F8393084F836349DF8133084F83734A1
:10BD0800D4F81434C4F84464C4F83C34C4F84C344B
:10BD180002F04DFB50B1D4F8140402F05AFB28B1DC
:10BD2800102007E7082005E7132003E795F81831E6
:10BD3800012B01D102F04FFB02F03CFB00230593DD
:10BD480094F8043195F9395094F81164BBB1042B77
:10BD58007FF4EAAE05A802F037FE60BB94F80C3415
:10BD68001BB994F80E34012B02D9059B013B0593AE
:10BD7800154B05983246E9B202F098FE02E01248E7
:10BD880002F06CFEA8B9D4F8403394F80C11218065
:10BD980043F00203C4F8403394F8103423B994F8FC
:10BDA8000C34013384F80C340D4B0E489B6A9847C9
:10BDB80028E71120BEE61220BCE60E20BAE600BF36
:10BDC80064180020D81F0020E020002094180020CC
:10BDD8005C2400204023002090230020EC23002036
:10BDE80014450108DA1F002073B5144C144D04F5EE
:10BDF8007876EB6C95F8502095F9781095F848000E
:10BE0800009603F07DF940F2012395F84800A4F864
:10BE1800F23304F21C42314603F07EF958B194F82B
:10BE28001C3484F85E34074B00205B6B984794F809
:10BE3800F33384F8803402B070BD00BFD81F0020EF
:10BE48006418002014450108F8B5334D95F81841D9
:10BE5800012C06464BD0022C51D064B938B9D5E92B
:10BE68001B0105F1740383E803002046F8BD01288F
:10BE78003DD0022801D00324F7E7284F85F81801A0
:10BE880007F5737EBEE80F0007F5787CACE80F0075
:10BE9800DEF80030CCF8003095F8E93087F8F36325
:10BEA800E3B195F80031022B18D1D5F804316B674E
:10BEB800C7F8E43395F87D3095F8082187F8F03312
:10BEC80095F88C3085F8782087F8F13397F81124A5
:10BED80087F8E02340F20133A7F8F233002387F80C
:10BEE80010340F4BDB6A9847FFF77EFFBDE702F07F
:10BEF80063FA04460028B8D185F81861B5E7002828
:10BF0800B9D1064B85F81801062283F88024044B22
:10BF1800DB6A98473446A8E764180020D81F002039
:10BF280014450108F0B5484C484EB4F8DC20228787
:10BF3800D4E92D0194F8B12084F8692004F16C0249
:10BF480082E80300D4E92F0104F1740282E80300B7
:10BF5800B4F8C420A4F87C20D4F8CC20C4F88420F9
:10BF68008FB0D4F8D020D4F8C810C4F888200025A1
:10BF7800374AC4F880100123A4F81E31C6F80C24EF
:10BF8800C4E94E5584F82C51A56284F81B5184F8F5
:10BF98003A50C4F83051A4F8345186F8105484F853
:10BFA80041518DF8143004F5087394F84800A4F84A
:10BFB8004251039303A904F52D73049303F088F801
:10BFC800E36EC6F8D03394F87D3086F8DC3394F805
:10BFD8008C3086F8DD334FF48073A6F8DE3386F8AC
:10BFE800CC5306F573770FCF06F578740FC43B680A
:10BFF800236040F20123A6F8F233D6F8483386F8D6
:10C008001154CDE901551BB15A685B69019202933D
:10C01800104B0693A3F144020792A3F1140208926D
:10C028000D4A0A9225330993A2F19C030B93A2F1BE
:10C0380098030C9301A9131D06A802F274620D93CC
:10C0480002F0A4F90FB0F0BD64180020D81F00203A
:10C05800000101003424002048190020F8B50D4FD4
:10C068000D4C0E4E0D4607F0D7FA3B6B984796F8E5
:10C07800480004F21C42294603F04EF848B194F8EF
:10C088001C3484F85E34706D7B6B9847EB7C84F8C5
:10C098008034F8BD14450108D81F0020641800201A
:10C0A8000D4890F8113480F8B8330C4B93F8692098
:10C0B80080F8BB2393F87D2093F88C3080F8C9333F
:10C0C800002380F8C823A0F8CA3300F56E7100F584
:10C0D8006070FFF7C3BF00BFD81F0020641800209E
:10C0E8000F4890F88034CBB190F8113480F8CC33F5
:10C0F8000C4BDA6EC0F8D02393F87D2093F88C307F
:10C1080080F8DD334FF4807380F8DC23A0F8DE3349
:10C1180000F5737100F56670FFF7A0BF704700BFA8
:10C12800D81F00206418002070B5344C2421204604
:10C1380004F064FF636A984218BF60624FF01C0104
:10C148002F4814BF0125002504F058FF636C98425E
:10C1580018BF60644FF0FC012A4818BF45F002057B
:10C1680004F04CFFD4F84431984218BFC4F8440195
:10C178004FF0D401244818BF45F0040504F03EFFF1
:10C18800D4F81C32984218BFC4F81C024FF0900132
:10C198001E4818BF45F0080504F030FFD4F8B03247
:10C1A800984218BFC4F8B0024FF49461184818BFF9
:10C1B80045F0100504F022FFD4F85437984218BF10
:10C1C800C4F854074FF01401124818BF45F0200571
:10C1D80004F014FFD4F86C3798420F4B18BFC4F81A
:10C1E8006C07D3F8483318BF45F040052BB11B69DD
:10C1F8001BB12846BDE87040184770BD6418002080
:10C208008C180020AC180020AC190020841A0020DB
:10C21800181B0020BC1F0020D81F00202DE9F04F5C
:10C2280091B00026BD4F8DF81560054688469346A7
:10C23800ADF81860B146C14502D311B0BDE8F08F22
:10C2480015F8090002F0C2F948444045F5DC15F834
:10C25800093009F10104023BE4B2112BEDD801A227
:10C2680052F823F0B5C20008E5C20008A5C30008CB
:10C27800D1C3000861C4000885C40008F9C40008D7
:10C288002DC50008ABC5000843C2000843C200081A
:10C298000BC6000843C2000843C20008C1C6000814
:10C2A800E7C600082BC7000869C70008052002F088
:10C2B80039FA88B10521002002F0F8F92B5D87F8DA
:10C2C800503409F1030409F102095FFA89F9E4B26B
:10C2D80015F8093087F85134A146ACE700238DF8EA
:10C2E80016308DF817308DF81C308DF82030002E60
:10C2F80052D18B4E631E2B440D9396F81A318DF84C
:10C308003A3096F87C308DF8393096F839308DF817
:10C318003B3096F838308DF83C3096F868308DF818
:10C328003D30D6F828310C9308AB019307AB009346
:10C3380096F84800A8EB09090DF117030DF116024C
:10C348000CA98DF8389002F0FBFE8DF8150000F06E
:10C35800070007280BD19DF8163086F839309DF86C
:10C36800173086F838309DF81C3086F8683000267B
:10C378004FF0050906E001220DF11501032002F036
:10C388003BF80136F2B29DF82030B3FBF9F1914247
:10C39800F1D8013B2344DCB201269DE72B5D6049BF
:10C3A80003F00F03012281F81B3109F1020902FA97
:10C3B80003F3A1F81E315FFA89F9002206A90420C7
:10C3C80002F01AF84C4687E707238DF815302B5DE5
:10C3D800C3F3021203F00F038DF8303009F10303A1
:10C3E800DBB28DF83120EA5C09F10403DBB209F114
:10C3F8000504EB5C09F102095FFA89F91B0443EAB9
:10C40800022315F80920DFF81891134364225343D7
:10C4180099F848000D930CA902F0A1FE00F007035B
:10C42800072BE4B28DF815000ED19DF8303089F84D
:10C43800703089F878300D9BC9F86C30C9F87430C1
:10C448009DF8313089F869308DF81800012206A965
:10C45800052001F0D1FF3FE7D7F8483363B11B68E7
:10C4680053B198470BF03F038DF818008DF8193039
:10C47800022206A90620ECE7FF20F3E703238DF844
:10C4880015302B5D8DF824300CAB089309F10303AC
:10C49800DBB209F10604EA5C09F10403DBB208A97E
:10C4A800EB5C1B0443EA022309F10202D2B209F150
:10C4B8000509AA5C1343642253435FFA89F90C9374
:10C4C80000230D9315F809308DF83830144B93F884
:10C4D800480002F04AFEC3B20028E4B28DF81530D5
:10C4E800FFF6FAAE8DF81830012206A90720B0E74A
:10C4F8002B5D03F00F03012B4FF47A7238BF012331
:10C508005343074A09F10209936503F57A73D36522
:10C518005FFA89F9002206A9082051E7D81F0020F0
:10C52800641800202B5D9C4CC3F340128DF81D202D
:10C5380094F84800C3F3001207A903F00F038DF81D
:10C548001C208DF81E3002F016FE09F10209013098
:10C558005FFA89F93FF436AFBDF81C308F4AA4F86A
:10C568007C309DF81E309DF81CA0D05CF5F74EFA83
:10C578000223C4F880000CA994F848008DF83030E4
:10C588008DF832A002F096FD94F93930089040B247
:10C598009842B8BF184684F83900002206A9092035
:10C5A8000EE703238DF815302B5D8DF8303009F137
:10C5B8000303DBB209F10504EA5C09F10403DBB209
:10C5C80009F10209EB5C5FFA89F91B0443EA0223CB
:10C5D80015F809201343642253430D936E4B0CA99D
:10C5E80093F8480002F0CDFDC3B20028E4B28DF8FC
:10C5F8001530FFF671AE8DF81830012206A90A2011
:10C6080027E70A2002F08EF800283FF465AE0A21D9
:10C61800002002F04BF80023ADF8263009F10203A0
:10C62800DBB24FF47A71EA5C09F10303DBB20DF176
:10C63800300AEB5C1B0443EA02232A5D134309F129
:10C648000402D2B209F1060409F10509AA5C5FFAED
:10C6580089F943EA026315F8092003934A43121241
:10C668005046ADF8242006F0E7FE039B03F19653ED
:10C6780003F5A91303F5EC530893D7F83C3300935B
:10C688000DF1200999E80600D7F838330AA806F012
:10C6980090FE0B9B00939AE806000A9B484606F01A
:10C6A8006DFE99E8030006F09FFE01F08FFE01235E
:10C6B800E4B287F830340FE60D2002F033F8002892
:10C6C8003FF40AAE0D21002001F0F0FF97F8803406
:10C6D800043B012B7FF600AE01F074FEFCE509F186
:10C6E8000203DBB22A5DE95C09F10303DBB209F15D
:10C6F8000504EB5C09F104095FFA89F91B0415F8D4
:10C70800090043EA012313436421594300F00F0051
:10C7180001F059FEE4B28DF81800012206A9112093
:10C7280097E60E2001F0FEFF00283FF4D5AD0E215C
:10C73800002001F0BBFF09F10203DBB2184AE85CF4
:10C748002B5D126809F1040409F103095FFA89F9FC
:10C7580043EA002015F80910E4B201F036FEBBE503
:10C768002A5D09F1020309F1040409F10309DBB2A6
:10C778005FFA89F9E95C15F809301B0443EA0123DB
:10C7880013436420584301F022FEE4B28DF81800E8
:10C79800012206A913205CE6641800208B3E0108DC
:10C7A800E02400200E4B93F88124920703D593F8D8
:10C7B8007F24012A06D90B4A92F81A1111B1916AFD
:10C7C80001319162002283F80C2483F8102483F845
:10C7D8000F24D3F8402322F00202C3F84023704705
:10C7E800D81F00206418002010B5124C04F55A70A8
:10C7F80006F012FFD4F84033012023F02003C4F8D8
:10C808004033FFF77BF998B10B2811D00A4B93F806
:10C81800393084F83634092094F80E3484F83934E1
:10C8280084F8350401F064FFBDE81040FFF7BABF93
:10C8380010BD00BFD81F002064180020074BD3F894
:10C848004023012A06D03AB993F88204013818BF68
:10C85800012070470020704701207047D81F002032
:10C86800034BD3F84003431E58425841704700BF5A
:10C87800D81F00202DE9F04FA5B0EFF3108172B654
:10C88800C04A00201368106081F31088BE4C002B4A
:10C8980000F0DA80D9065FFA83FB6BD5BB4D95F8BB
:10C8A8001831022B02D0BA4BDB6A9847EFF3108895
:10C8B80072B6B84F06F06CFE3E68D4F8B013361A5C
:10C8C8003144B54806F030FFB34806F0F3FED4F81B
:10C8D800B413B248314406F027FFB04806F0EAFE28
:10C8E80088F3108895F81831022B02D094F8103488
:10C8F8008BB116230EA995F848008DF8383002F050
:10C90800D9FBD4F8B4130C900144A54806F00CFFE9
:10C91800A34806F0CFFE3B6894F81124EB620AAFF7
:10C9280038468DF86020199306F0ACFDD5F824310F
:10C93800009304AE97E80600D5F82031304606F09B
:10C9480038FD96E803001BAB83E80300D4F81434E1
:10C958001A9395F82C3195F84800003B18BF01232D
:10C9680018A98DF8613002F0AEFB94F810340BB9B9
:10C9780084F835341BF0080F3AD08A4B834D5F6832
:10C988001E89B3F90A8093F90C90D5F8E420039234
:10C998000023079384F83834A4F81A3484F81D3433
:10C9A800C4F82034A4F8243484F82634C4F828348D
:10C9B80084F81834C4F82C3484F83034744B94F860
:10C9C8008024DB6A84F87F24A4F87C8484F87E942D
:10C9D8009847724806F020FE3146384601F0DFFCE1
:10C9E8008246002800F0E680A4F8728484F87494E3
:10C9F8001BF0040F1AD0654B93F81831022B02D0A4
:10CA0800634BDB6A98470220FEF72CFF84F8350455
:10CA180001F06EFE94F8103413B1012384F80F343A
:10CA280094F8813443F0100384F881341BF0020F2A
:10CA380003D006210520FEF78BFF1BF0010F03D062
:10CA480004210320FEF784FF01F0C6FC94F881243A
:10CA5800D0065FD5002384F88234D4F84033190611
:10CA680044BF23F08203C4F8403312F0050F00F0EE
:10CA7800C5820C2001F056FE002800F0BF8294F811
:10CA88008134DF0700F1BA825E0740F1CB82D4F827
:10CA9800403323F00203C4F84033D4F8402382BB68
:10CAA80094F8815415F001011EBF2B4662F3000370
:10CAB80084F8813494F881345E0744BF6FF38203AD
:10CAC80084F88134012384F8823421B1D4F84433C2
:10CAD80035481B6898476D070BD5344801F02EFE82
:10CAE80001F05CFE28B194F8813443F0040384F823
:10CAF800813401F060FC94F881346FF3041384F8F6
:10CB08008134012384F8823494F8813443F020037B
:10CB180084F8813494F8813418070AD56FF3C30375
:10CB2800234984F88134D4F84433A1F12000DB6828
:10CB3800984794F8813499070AD56FF341031C4943
:10CB480084F88134D4F84433A1F164005B689847D1
:10CB580094F88034022B01D1FFF746F994F8813418
:10CB68009A0640F1EC826FF3451384F88134D4F8C7
:10CB78004033002B40F0E38225B0BDE8F04FFFF7CB
:10CB8800D3BA00BFD41F0020D81F0020641800208B
:10CB980014450108F02400205823002070230020A9
:10CBA800CC230020E02400200C2400202024002096
:10CBB8005424002095F81831012B0CD101F0F3FB17
:10CBC800804668B1504601F0E3FB504601F0E5FBB2
:10CBD800042384F87F347EB9012384F819344AE1A8
:10CBE80001F0E3FB0028F6D0404601F0D2FB4046B6
:10CBF80001F0D4FB0523ECE73B7802935B09013B8A
:10CC0800062B00F2ED81DFE813F00700EB0192003C
:10CC1800EB018F00EB01DB01102EDDD995F82C31EB
:10CC28000E97F6B28DF83C60002BD5D118A804F009
:10CC3800F9F80EAA18A9FF2002F04CF89DF8483020
:10CC4800C3F3030307468DF8203095F8480095F89C
:10CC58007D308DF82130072208A902F03EFA002F16
:10CC68005AD1002858D09DF843309DF84220119998
:10CC7800C5F8E4101B0443EA02239DF84120022072
:10CC88001343C5F8E03004F0DBF89DF8483095F818
:10CC9800480085F82A71C3F30212C3F3030385F829
:10CCA800703085F878309DF8493085F86920012B77
:10CCB80038BF01234FF47A725343AB651344EB65D5
:10CCC8004FF001080DF14A03113E0CA90C9385F8A9
:10CCD80068808DF8346002F008FA0223404685F82F
:10CCE8002C3101F01FFD18B14146384601F0DEFC39
:10CCF80094F81034002B00F0798194F8383413B18B
:10CD08000020FEF7E9FD94F8813443F0100384F81D
:10CD18008134FEF7A7FD6BE6012001F003FD002832
:10CD2800E6D001210720E1E7012384F8183495F8BB
:10CD38007D308DF8223094F81C348DF8213095F828
:10CD48008C3095F848000D3308A98DF8203002F092
:10CD5800B1F9A6F10D031BB2069023EAE37300B202
:10CD680083423FF739AF0B2E7FF636AFA24B2193A4
:10CD780018A8FF2318978DF864608DF8883002F0A2
:10CD880075F8804600287FF427AF9DF86C301A9913
:10CD9800C4F82C1413F00F0203D09DF8800000286B
:10CDA8006CD19DF8880000286AD0002A7FF414AF5F
:10CDB8009DF88020002A0CBF022703270022079233
:10CDC800D5F8EC2091425DD195F8E910002959D0A9
:10CDD800D5F80C1195F8EAA00968079195F818118B
:10CDE800022902D1032184F87F14032F7FF4F4AEC3
:10CDF80013F0600F7FF4F0AE03924FF00108152393
:10CE080095F848008DF8203008A902F053F995F8F4
:10CE18002A310690BAF1000F37D0BAF1010F3ED18E
:10CE2800012B34D16FF009063E4106F00106C6F128
:10CE38000206F6B281B2BDF86E2007AB304601F0AB
:10CE4800CFFD70B3072824D1082384F8193495F846
:10CE58002A315BB9029B03F0E003A02B06D16A6B71
:10CE6800239B9A4202D1012385F83A30079BC4F8E4
:10CE78002834C4F86034FEF74FFDB9E547469DE70E
:10CE880001279BE74FF0010AB9E70426D2E70326FA
:10CE9800D0E7082803D10A2384F81934E6E70123E8
:10CEA800FAE718AB00930399079B3246504601F006
:10CEB80063FE20B102280CBF0B230C238DE6079BD1
:10CEC800C4F82834C4F860349DF86C3084F8190428
:10CED800C3F3401384F8263484F8383494F87F3444
:10CEE80084F81A84012B98BFA862B8F1010FC4F81E
:10CEF800200484F8240484F8350433D1022284F809
:10CF0800182495F83A20002A3BD19DF86C20D206C7
:10CF180037D4012B94F834149DF86C2005D80129D6
:10CF280001D1960601D501F001FB022F37D0032F5E
:10CF380009D09DF86C10012F4A4601F00F011CA87A
:10CF480031D0FFF76BF99DF8803084F81B34219BB2
:10CF5800C4F820349DF8883084F82434012384F8F8
:10CF6800253426E0029A02F0E002A02A11D195F8B1
:10CF78002A11012285F83A2009B92399696384F8AE
:10CF8800182495F81821002AC3D1012284F81D24F9
:10CF9800BFE7002285F83A2084F81824B5E79DF801
:10CFA800881021984A46FFF739F99DF8803084F8AF
:10CFB8001B3494F8813443F0020384F8813497E6F3
:10CFC800DFF83480013EB2B2791C404604F000F824
:10CFD8000323A4F81834C4F8208484F82464E8E708
:10CFE800012384F81934FEF797FC81E695F8183187
:10CFF800022B7FF488AE83E61022002094F8813457
:10D008005D070FD5012001F08DFB88B3012001F0E9
:10D018005FFB08B984F80C04D4F8403323F002030A
:10D02800C4F8403394F88114C8077FF536AD94F8F6
:10D0380034340BB1032B26D1424B94F80C0493F8EB
:10D048006820904208D28A0750D593F818311BB14E
:10D0580094F87F34002B49D13B4806F0DDFAD4F828
:10D06800403323F02003C4F84033FFF79BFB14E55B
:10D07800062001F057FB0028CED1072001F052FB13
:10D088000028C9D1CEE7012B30D194F80F24002A0B
:10D098003FF403AD94F80E3494F80D04834204D29F
:10D0A80011F0020218BF94F83824264D95F82A1179
:10D0B800002941D132BB834218D20133DBB2DF07EA
:10D0C80084F80E3412D522238DF8603095F87C3020
:10D0D8008DF8623095F8480095F839308DF8613050
:10D0E80018A901F0E7FF0E9085F8390094F881340B
:10D0F80000206FF3041384F8813484F80F04FFF7D9
:10D1080073FBCAE494F838648EB902238DF868304A
:10D1180005F50873189395F8480005F52D7318A9B7
:10D12800199301F0D5FF84F8106484F8386494F8F2
:10D138000E3484F839348FE7002AD7D08CE725B02D
:10D14800BDE8F08F64180020402300202DE9F04F3F
:10D158008A468BB091460746002800F08D81002949
:10D1680000F08A810368002B00F086814368002B59
:10D1780000F082818368002B00F07E81C368002B59
:10D1880000F07A81104601F091FF002800F07681C6
:10D19800BC4CBD4D384601F03FFA4FF4EE62002119
:10D1A800204603F029FF4FF4A1620021284603F02E
:10D1B80023FFB64BC4F8283100264FF001080F238F
:10D1C80005A948468DF8143084F8489084F8186109
:10D1D80084F88C6085F80E8485F80D8401F06AFF68
:10D1E800801B18BF01204FF00A0B84F81C0105A909
:10D1F80094F848008DF814B001F05CFF4FF0060970
:10D2080084F8DC0005A994F848008DF8149001F022
:10D2180051FF102384F8DD0005A994F848008DF823
:10D22800143001F047FF1123C4F89C0005A994F8B5
:10D2380048008DF8143001F03DFF1223C4F8A00017
:10D2480005A994F848008DF8143001F033FF132332
:10D25800C4F8A40005A994F848008DF8143001F02A
:10D2680029FF14230DEB0301C4F8A80094F8480023
:10D278008DF8143001F01EFF1723C4F8AC0005A97F
:10D2880094F848008DF8143001F014FF182384F83E
:10D29800B10005A994F848008DF8143001F00AFF90
:10D2A8001923C4F8B400C4F8BC0005A994F84800D0
:10D2B8008DF8143001F0FEFEC0B21E2384F8B800C9
:10D2C80084F8C00005A994F848008DF8143001F0DE
:10D2D800F1FE1F2384F8C40005A994F848008DF8CE
:10D2E800143001F0E7FE202384F8C50005A994F85E
:10D2F80048008DF8143001F0DDFE2123C4F8C80081
:10D3080005A994F848008DF8143001F0D3FE0B23DA
:10D31800C4F8CC0005A994F848008DF8143001F041
:10D32800C9FE0C23A4F8D00005A994F848008DF88C
:10D33800143001F0BFFED4F89C306365D4F8A030F7
:10D34800A365D4F8A430E365D4F8A8302366D4F8EC
:10D35800AC30636604F5087307A90490A4F8D200FA
:10D36800079394F848008DF8246004F52D7308930A
:10D3780084F8B080C4F894B084F89890C4F84CB09D
:10D3880084F8509084F8688001F0A2FEC5F848A39C
:10D39800FEF7C8FD32463E4B00964FF0FF3105F5CB
:10D3A8005A70C4E90B66C5F8447385F8816484F83B
:10D3B8001981C5F8408306F0D1F83246354B0096FE
:10D3C8004FF0FF3105F5607006F0C8F83246324B71
:10D3D80000964FF0FF3105F5667006F0BFF832464B
:10D3E8002E4B00964FF0FF3102AE05F57D7006F02A
:10D3F800B5F8304606F046F896E8030004F5907351
:10D4080083E80300264BC5F84C33264BC5F8543344
:10D41800254BC5F85C33254F254BC5F85033254BB4
:10D42800C5F8583305F553703B68984704F5A47060
:10D4380003F016FB20B1112630460BB0BDE8F08F83
:10D44800204601F09DFA0028F5D100F0C7FFB8B9D1
:10D45800194801F0F7FA06460028ECD17B6998478D
:10D4680003F094FDBB6D94F819019847FB6A98473F
:10D47800012385F88234DFE70326DDE70926DBE7A9
:10D488001326D9E764180020D81F002000030001E4
:10D49800F1C70008A9C00008E9C00008E1B8000801
:10D4A800B9BA000871BA00089DB800081445010807
:10D4B80049BA000821BA00084C19002008B5034BE6
:10D4C8000020C3F84003FEF7CDF908BDD81F00209F
:10D4D80010B5FFF7B3F90A4C60B90A4B93F8183145
:10D4E800022B02D1084BDB6A98470123C4F840336A
:10D4F800002010BDD4F84003013818BF0120F8E718
:10D50800D81F0020641800201445010838B5134CB2
:10D5180004F55A7006F080F804F5607006F07CF89F
:10D5280004F5667006F078F804F57D7006F074F876
:10D5380000F040FF0A4B0025DB6A9847C4F84053C7
:10D54800FEF7F2FD074908484FF4EE6203F040FD8C
:10D558000123C4F84033284638BD00BFD81F002037
:10D568001445010864180020F410002030B52A4B37
:10D5780089B0054693F8DD008DF8020093F8DC00C9
:10D588009A6A8DF803000020019202900C46002947
:10D598003ED00592D3F8882006921A8FD3F8281126
:10D5A800039152BA93F81A11ADF81C2093F87C2015
:10D5B80093F848308DF810008DF811108DF81E2062
:10D5C8008DF81F300DF1030201AB0DF1020103A824
:10D5D80000F06EFE9DF90200FEF766F9607002A881
:10D5E80000F0B6FFB0B9029A0F2A0DD863789A42B4
:10D5F8000AD81544AB42A3EB02012CBF002001203E
:10D608002170C00009B030BD002323700820F9E75D
:10D618000320F7E71320F5E7641800201FB5044638
:10D62800002800F0FD8000783F2800F2F380DFE852
:10D6380010F0400046004B005000540058005D00B8
:10D64800F100F100F100F100F100F100F100F1004A
:10D65800640068006C0077007E0081008400890007
:10D6680087008B008F009200950098009B009E0019
:10D67800A200AA00A600AE00B100B500BE00BA0024
:10D68800BC00F100C200F100F100F100F100F1006E
:10D69800F100F100F100F100F100F100F100F100FA
:10D6A800F100F100CA00CE00D300D700DB00DF0094
:10D6B800E8005D4B93F81831237104B010BD5A4B44
:10D6C80093F82C31237102E0606803F065FB0020B9
:10D6D800F3E7606803F0A6FBF9E7534B93F81A31B8
:10D6E800F0E7514BD3F8E0306360F0E74E4B211D73
:10D6F80093F82C0103F0AEFBE9E74B4B93F8193193
:10D70800E0E7494B93F88C30DCE71D238DF80830AF
:10D71800454B02A993F8480001F0CCFC6060D6E7BD
:10D72800424B043493E8030084E80300CFE7404BFE
:10D738000434F7E73F4B0434F4E73F4B0434F1E794
:10D748001B23E3E71A23E1E7374B93F86830B9E77F
:10D75800354B5B6DC8E7344B9B6DC5E7324BDB6DD2
:10D76800C2E7314B1B6EBFE72F4B5B6EBCE72E4BFE
:10D7780093F8DD30A6E72C4B93F83930A2E72A4B13
:10D7880093F8DC309EE7284B93F838309AE7264B1D
:10D79800DB6CA9E7244B93F8503093E7224BD3F87E
:10D7A8008430636093E7204B9EE7244B9CE71E4B35
:10D7B800D3F8CC30F5E71C4BD3F82831636001F07F
:10D7C8000DFDA06083E7184BD3F890308CE7164B1B
:10D7D800B3F88830A3807AE7134BB3F88A30F9E7B7
:10D7E800114BB3F8D030F5E70F4BB3F8D230F1E76F
:10D7F8000D4B93F848200AB1062A13D1B3F84C37D9
:10D80800E8E7094B93F848200AB1062A0AD1D3F869
:10D81800503769E7204604B0BDE8104000F0CEBD9F
:10D8280003204AE7182048E764180020D018002091
:10D8380018190020D818002020190020F410002002
:10D8480073B5044600285ED0A04DD5F840339A073A
:10D8580000F15F8202783F2A00F25682DFE812F078
:10D86800400046004E0056005A005F0064007000F9
:10D878007A007F00840089008E00930098009D0044
:10D88800A7005402AC00CC00DF00060128011901F2
:10D898002C013C014001440148014C015001620146
:10D8A8008A0178019C01A201A901AE01B3015402C9
:10D8B80018025402540254025402540254025402EC
:10D8C80054025402540254025402540254025402A0
:10D8D800540227022C02310236023B0240024A025D
:10D8E800007902B0BDE87040FEF7AEBA0379022BAA
:10D8F80009D0774A82F82C31002005E0406803F00F
:10D908003DFA0028F8D0032002B070BD406803F04B
:10D9180079FAF6E76E4B027983F81A21ECE76C4B3B
:10D928004268C3F8E020E7E7694D416895F82C01A3
:10D9380003F086FA0028E6D16368C5F8E430E3E727
:10D9480041680029DFD0002001F0A8F90028D3D0D1
:10D958001120D9E741680029D5D00120F4E74168B2
:10D968000029D0D00820EFE741680029CBD0092052
:10D97800EAE741680029C6D00C20E5E7416800299C
:10D98800C1D00D20E0E741680029BCD00E20DBE7BC
:10D9980041680029B7D00F20D6E74E4C4C4B007990
:10D9A80083F81901A36D9847E36A9847A4E7484BA1
:10D9B800027983F88C209FE7454D037A8DF8003073
:10D9C80095F8480095F87D308DF8013007226946B2
:10D9D80001F083FB002896D0636895F8480000930F
:10D9E8000022694601F079FB00288CD06C35D4E917
:10D9F800010185E803007FE7354D037A8DF8003093
:10DA080095F8480095F87D308DF801300722694671
:10DA180001F063FB00283FF476AFB435E7E72C4DFF
:10DA2800037A8DF8003095F8480095F87D308DF828
:10DA380001300722694601F050FB00283FF463AF2C
:10DA4800D4E9010105F1740383E8030095F818315E
:10DA5800022B7FF451AF95F82C31002B3FF44CAFDB
:10DA68001C4BDB6A9847FEF7BFF945E7184D037A68
:10DA78008DF8003095F8480095F87D308DF8013024
:10DA88000722694601F029FB00283FF43CAFBC356A
:10DA9800ADE74368009301238DF804300C4B6946C9
:10DAA80093F8480001F026FB00287FF425AF2AE709
:10DAB800436800930023EFE703795A1E0E2A3FF6C6
:10DAC80022AF034A82F8683016E700BFD81F00204B
:10DAD8006418002014450108904B42685A650BE70A
:10DAE8008E4B42689A6507E78C4B4268DA6503E714
:10DAF8008A4B42681A66FFE6884B42685A66FBE61C
:10DB0800864C037994F848008DF80030062269465F
:10DB180001F0E3FA00283FF4F6AE9DF8003084F8EF
:10DB2800DD30E9E67D4C03798DF8003094F8480043
:10DB380094F87C308DF802300522694601F0CDFA60
:10DB480000283FF4E0AE9DF8003084F83930D3E681
:10DB5800724C037994F848008DF800300A2269461F
:10DB680001F0BBFA00283FF4CEAE9DF8003084F8EF
:10DB7800DC30C1E6694C037994F848008DF8003030
:10DB88000922694601F0A9FA00283FF4BCAE9DF8C5
:10DB9800003084F83830AFE6604B4268C3F8942010
:10DBA800DA64A9E65D4B027983F8982083F850205F
:10DBB800A2E65A4B4268C3F884209DE6574B426858
:10DBC800C3F8CC2098E6012B40F0A380544C2421C4
:10DBD800204603F013FA636A984201D0172093E6AF
:10DBE8001C2104F1280003F009FA636C9842F5D16E
:10DBF800FC2104F1480003F001FAD4F844319842BA
:10DC0800ECD1D42104F5A47003F0F8F9D4F81C324F
:10DC18009842E3D1902104F5087003F0EFF9D4F8A5
:10DC2800B0329842DAD14FF4946104F52D7003F0C4
:10DC3800E5F9D4F854379842D0D1142104F5EB60B3
:10DC480003F0DCF9D4F86C379842C7D1334E21463B
:10DC580030464FF4EE6203F0BBF920464FF4EE6213
:10DC6800002103F0C9F995F8113485F8E033736F92
:10DC7800C5F8E43396F87D3085F8F03340F2012397
:10DC8800A5F8F233274B96F819019B6D984733E6B0
:10DC98008379012B3FF637AE204B42684068C3F8C2
:10DCA800282100F089FE00283FF42EAE50E61B4BD9
:10DCB8004268C3F890201FE6184B8288A3F8882092
:10DCC8001AE6164B8288A3F88A2015E6134B828839
:10DCD800A3F8D02010E6114B8288A3F8D2200BE6D7
:10DCE8000E4B93F848200AB1062A14D1A288A3F84B
:10DCF8004C2701E6094B93F848200AB1062A0AD1B5
:10DD08006268C3F85027F7E502B0BDE8704000F03C
:10DD180057BB0120F8E51820F6E500BF641800207D
:10DD2800F4100020144501082DE9F04186B00023C5
:10DD3800ADF800300646002800F0E280FEF77EFDD0
:10DD480020B10124204606B0BDE8F08100F02CFD8A
:10DD58000028F6D100F022FD014618B969481422BE
:10DD680003F04AF9684D95F88134012243F0040321
:10DD780085F8492485F8813433788DF804300021FA
:10DD8800013B8DF805208DF807100D2B00F2B080AF
:10DD9800DFE803F007AEAEAE525A7DAEAE85AEA256
:10DDA8008F9ED5F8404314F02004CAD1DFF85C8177
:10DDB800574FFEF7B7F8224696F9051098F848002D
:10DDC80001F0E5F988F83900B37988F83830204649
:10DDD80007238DF80530FEF737F8FF2307F586701F
:10DDE800A5F80C3185F80441C5F8087103F01AF854
:10DDF80007F58A7002F0D0FF2046FDF77FFE044643
:10DE080040B196F9051098F84800012201F0BFF9D1
:10DE180088F83900D5F884343361002C6CD000F0D0
:10DE2800BDFC00288ED195F8813485F8100460F384
:10DE3800820385F8813485E700226946022000F0D4
:10DE4800DBFA10B31324E5E795F811348DF80830A0
:10DE58002E4BB28893F839108DF8091093F83810C2
:10DE68008DF80A10D3F880100391D3F88410049128
:10DE780093F84800ADF8142002A901F09DF9D5F8EF
:10DE8800403343F00203C5F840330024C2E7214B76
:10DE9800B28896F90C10B068DB6B9847EFE702A9D7
:10DEA8000D2000F027FB0028EFD0002269460D2046
:10DEB800C5E7164B93F81831D3B9347904F0070045
:10DEC80000F077FA8DF80040012269461020B6E785
:10DED800002269461220B2E78DF8072000F05AFAAE
:10DEE800044638B900F053FA204600F055FA91E795
:10DEF80002248FE701248DE701A800F0A1FB21E7A8
:10DF080003241FE720240020D81F002064180020C5
:10DF1800DA1F0020144501082DE9F04F91B00026C2
:10DF28000391054618B9032011B0BDE8F08FFEF73C
:10DF380085FC8246002840F06481B84C14220146D2
:10DF4800074604F2344003F057F8012384F83534C7
:10DF580084F80E342A789A4200F0B080032A00F040
:10DF6800BF80002A40F0C98084F80D34022295F859
:10DF78000490D5F80880AE8995F90EB062F347177A
:10DF88009A46A74B022493F87C2093F848008DF812
:10DF9800244009A98DF8262001F08CF8BAF1000F69
:10DFA80000F02D819E4B93F81A21B2B940B2584522
:10DFB800B8BF584693F87C208DF814008DF81620C9
:10DFC80093F84800052205A901F087F80028AAD08F
:10DFD800934B9DF8142083F83920198F1A8F93F8E2
:10DFE8002C010291996A069152BA002800F0058125
:10DFF80093F81B0100B9186393F81801ADF83C2099
:10E00800013893F87C208DF83E20D0F1000B93F86E
:10E0180048208DF83F204BEB000B824A93F83A00DA
:10E0280093F81A4101900D914FF00100D3F8881030
:10E03800D3F828318DF830000E910B93511C06ABA4
:10E048000BA88DF8314000F033F9019B4FEA0B1B08
:10E058004BEA431B4FF0000A4BEA801B4BEAC41300
:10E06800D0456E4C019308BF56463246414604F5EA
:10E078009C709B46CDE907AAA4F800A084F810A4D8
:10E0880002F0A6FFF9B2A770C7F34217F2B2042F45
:10E09800634E019B84F8372233D0072F00F09D8010
:10E0A800022F32D00220029B33875C4B002283F878
:10E0B80010245A4BD3F884342B6135E7EB7B082BBB
:10E0C80028BF082384F80D34042395F80490D5F864
:10E0D8000880AE8995F90EB063F34717924650E76A
:10E0E80084F80D34D5F804802E8995F90AB067F0C4
:10E0F8001F079A464FF0000943E7D346D046D1465A
:10E108003FE74FF0010084F81004474F84F80D11E1
:10E11800042084F80401FF20D6F8E41084F80C01E8
:10E1280084F8143107A807F59B73C4F8087184F8BC
:10E138002891C4F8101184F83021C4F82C3100F06B
:10E1480043FC002857D1079BA4F8380408A8A4F872
:10E158001631C4F8403400F0FBF960BB089BABB142
:10E1680096F93900FDF7A0FB94F837322BB3089BDA
:10E178000F2B19D807F58B7208A90F2000F0F4F9B6
:10E18800C8B9089B63F3030B84F814B10398FDF72F
:10E19800B5FC002887D1069B86F83A00B36200F0E8
:10E1A800B7F980B3132080E707F2864208A900F088
:10E1B800DBF90028EAD0132075E707F286473A46CC
:10E1C80008A900F0D1F90028F5D1089B84F82801A6
:10E1D800C4F82C7184F83031D8E7B8F1000FD5D0E5
:10E1E800002AD3D04146E01C02F0F2FE94F8373200
:10E1F80001332380CAE7122055E7072055E7204658
:10E2080057E7012090E62B7884F8343494F8813469
:10E2180043F0010384F881344BE700BFD81F002086
:10E22800641800209C180020DA1F002037B50B4D19
:10E238008DF8040004460F2295F8480001A900F063
:10E248004CFF40B1064A85F81C4192F8813443F0EE
:10E25800200382F8813403B030BD00BF6418002069
:10E26800D81F002010B5FFF733F90446A0B90B48B2
:10E2780005F0D2F90A4805F0CFF90A4805F0CCF9BB
:10E28800094805F0C9F900F095F8FDF74BFE074B72
:10E29800DB6A9847204610BD0124FBE74023002095
:10E2A8005823002070230020CC23002014450108A7
:10E2B8002DE9F04F90F802908BB004468A460192FF
:10E2C800B9F1000F60D14579816890F9102090F973
:10E2D80011801960002D55D0817C8DF81610C07CF6
:10E2E8004FF0020B05A9CDE902238DF814B000F018
:10E2F800E1FE029A47B2BA421646B8BF3E46BA4253
:10E308000CDC039BC3F800904D46019B8AF8006023
:10E3180083F8008028460BB0BDE8F08FA268A18979
:10E32800E3898A420B4434BF002501259A42ECD385
:10E33800082305A9E07C8DF8143000F0BBFEE289C3
:10E34800A368B3FBF2F102FB1133012B4FFA80F8FB
:10E35800DBD122238DF81430E07CA37C8DF8156086
:10E3680005A98DF8163000F0A5FE46B2B742CCD10B
:10E378002579002DC9D0E07C8DF824B007A900F0DC
:10E38800A7FEC1E71646C0E70025C3E770477047F8
:10E3980070477047002070477047704770470020EB
:10E3A8007047002070470020704700207047002009
:10E3B80070477047704770470220704702207047C7
:10E3C8000220704770470020704770477047002050
:10E3D80070470020704770477047000010B5054C23
:10E3E800FC222046002102F007FE0020C4E90000BC
:10E3F80010BD00BFF42400202DE9F04180461546E9
:10E40800002942D0244B002403F1010C1A462001B4
:10E41800103312F8016F002E39D19A42F9D11F4FEB
:10E428003B680BB9C7F800C07B680BB1C3F800C0E4
:10E438003B18002201349A6083F80C800D302301C8
:10E44800AAB23844FD50C7F804C002F0C1FDB8F1C3
:10E45800050F17D0A8F10808B8F1020F8CBF4FF0CC
:10E4680000084FF0010807EB041400236371D7F884
:10E47800F83084F8048001332B44C7F8F83030466C
:10E48800BDE8F0814FF00108EDE70126F7E7013418
:10E498000F2CB9D10226F2E7FB240020F424002037
:10E4A80010B510B3124A1368984204D10368136078
:10E4B800002304E00B4613B119688842FAD1516869
:10E4C800884208BF53600BB101681960D2F8F83070
:10E4D8008168013B00245B1A04602146C2F8F830C9
:10E4E800102202F089FD204610BD0120FCE700BF84
:10E4F800F4240020054B1B6813B11A798242FAD123
:10E50800002B0B600CBF032000207047F424002070
:10E5180010B5054B186800B910BD037B04680BB92A
:10E52800FFF7BEFF2046F6E7F424002010B5074B9E
:10E53800186800B910BD03790468052B02D0083BA0
:10E54800022B01D8FFF7ACFF2046F2E7F4240020A5
:10E5580028B1044BD3F8F83003600020704701203D
:10E56800704700BFF42400202DE9F04107460E460D
:10E5780015463AB331B3144B1C6800232CB9304606
:10E58800FFF7E6FF0020BDE8F081A268F91A013222
:10E59800914210D32279EA54581C22895FFA80F8F4
:10E5A800611D55FA80F002F013FDA36824689844B1
:10E5B8005FFA88F3E2E720462468FFF771FF002C32
:10E5C800F9D1DCE70120DEE7F42400200238C0B2EC
:10E5D80011289ABF014B185C002070479B3E010828
:10E5E80030B50B4B93F820200446084672B1002141
:10E5F8001C330578A54208D001319842CDB20CBF32
:10E6080004480430AA42F4D8002030BD1046FCE784
:10E61800F0250020FC25002010B5084C00232060C0
:10E62800142204F10C00FF2184F82030C4E9010011
:10E6380002F0E2FC012384F8213010BDF02500200F
:10E6480010B50E4A92F82010042915D8936804785A
:10E658001C7044785C70C078D870013100209870C4
:10E6680082F8201002F11C018B4214BF043302F11E
:10E678000C039360012010BD0020FCE7F02500206A
:10E68800094B93F8200068B15A6803F11C018A42CB
:10E6980000F1FF3014BF043203F10C0283F82000AC
:10E6A8005A600120704700BFF025002010B5074BC5
:10E6B80093F820200446084632B15968FFF790FFC6
:10E6C80010B101234470837010BD00BFF0250020F5
:10E6D80008B5064B93F820202AB15968FFF780FF48
:10E6E80008B1407808BD0120FCE700BFF0250020F4
:10E6F80030B50A4A92F82010536882F8210061B1B7
:10E70800916801241C32DD78587005B99C709342D9
:10E718000CBF034B04339942F5D130BDF0250020DE
:10E72800FC25002008B5044B5968FFF759FF00384D
:10E7380018BF012008BD00BFF02500202DE9F341D6
:10E748000422154E044600210DEB020096F82080A5
:10E7580002F052FC0025EBB2984502D802B0BDE8A1
:10E76800F0817368197821705A7862709F785FB168
:10E77800336820469B689847FFF782FF17B901A8BE
:10E78800FFF75EFF0135E6E7DB788DF804108DF8BA
:10E7980005208DF80730EFE7F0250020014B93F8AE
:10E7A80020007047F0250020034B93F82000042830
:10E7B80094BF002001207047F02500201FB50024D9
:10E7C800CDE90244C41F8DF800408DF801100C0AF1
:10E7D800ADF80420090C120C8DF803108DF80620F2
:10E7E8008DF8073002461B0A012168468DF8024061
:10E7F8008DF8083002F05DFA002818BF0F2004B029
:10E8080010BD2DE9F04188B017460D460F9A06460F
:10E8180000284DD000240121CDE904448DF81010C2
:10E828009DF838108DF81510ADF81630190CCDE993
:10E8380000441B0ECDE902448DF81930ADF81A20BA
:10E84800130C120E07948DF818108DF81C308DF8E3
:10E858001D20E3B24FEA0318002D5FFA88F803DCA5
:10E86800002008B0BDE8F081013310218DF81F3079
:10E878003A466B460DEB010002F0B1F90346C8B900
:10E88800102DAC46A8BF4FF0100CDAB2624503F168
:10E89800010303DB103D2DB20134DAE708EB020077
:10E8A80020326A44315C12F8202C4A403254ECE79A
:10E8B8000A20D6E70F20D4E70138032815D8DFE867
:10E8C80000F002080C100A4B1B681B690B60002043
:10E8D8007047074B1B685B69F8E7054B1B689B692A
:10E8E800F4E7034B1B68DB69F0E70520704700BFBE
:10E8F800142600202DE9F041C4B00C464A9E174664
:10E908001D468046B8B3B1F5807F36D84FF488727B
:10E918000021684602F070FB492300934FF480738E
:10E92800ADF804302B0C8DF80830330CADF80650D8
:10E93800ADF80A608DF80C3022460023414604A841
:10E948002D0E360E8DF80E308DF809508DF80D60AD
:10E958008DF80F4002F03CFB04F110014B9A3B4646
:10E9680089B2684602F025F910B1012818BF0F20B6
:10E9780044B0BDE8F0810A20FAE70E20F8E700006D
:10E9880010B590B10A4C28220021206002F034FB17
:10E998002368084A1A6000204FF0FF32C3E90302D7
:10E9A800C3E90522C3E9072210BD0920FCE700BF1F
:10E9B8001426002000010101024B1B68186000208A
:10E9C800704700BF1426002030B1044B1B68DB6879
:10E9D80001330360002070470A2070471426002086
:10E9E80073B50E46002101911D4633B301A9FFF707
:10E9F80063FFD0B9019C631C04D0A3B2D31A002BC7
:10EA080010DDE2180E4B2A601B689B786BB9121B4D
:10EA180063EB0303B24273F10003ACBF0120002093
:10EA2800C00002E003D12C60072002B070BD230CA7
:10EA38001B0403F580331A44E4E70A20F5E700BF16
:10EA48001426002028B1044B1B681C3343620020A5
:10EA580070470A20704700BF142600201FB50446DF
:10EA6800F0B1002303A8039302F07AF90E4ABDF827
:10EA78000C30126820469380E38200F052FA60B9A5
:10EA880004F11803009321680123132202F088F887
:10EA980040B9204600F045FA00B1112004B010BD7D
:10EAA8000A20FBE70F20F9E714260020F0B50546F9
:10EAB80087B01C463BB32F4E3368DB68834257D878
:10EAC80094F82020002A14BF09220822834205D383
:10EAD800204600F05AFA70B111200AE00023019094
:10EAE8000093A36894F82810606AFFF78AFE00284C
:10EAF800EED007B0F0BD23792168B4F808C0A76844
:10EB0800043B9AB209B90A20F3E7B2F5807F2DD801
:10EB1800ADF80EC08DF817304FEA174C04F12C03EE
:10EB28003F0E8DF8117000932F0C08234FF0490EFB
:10EB3800ADF80C008DF814708DF816002F0E0DEB43
:10EB48000300CDF808E08DF810C0ADF812508DF82C
:10EB5800157002F025F808B10F20CAE7204600F02A
:10EB680014FA0028B8D13368DD60C2E70E20C0E788
:10EB78000620BEE7142600202DE9FF410A9D8046A5
:10EB88000F4616461C46002D5AD0002303A91046EE
:10EB98000393FFF791FE18B1062004B0BDE8F08199
:10EBA800039B9C4201D80133F6D1284600F05EF958
:10EBB800002847D1264B1A78424503D01A79424596
:10EBC80042D10120AA68BA4240D103EB8002EB6A25
:10EBD80092F801802979CDE90043043992782868B0
:10EBE8003B4689B2FFF786FE0028D6D195F820303B
:10EBF8000194002B4FF00103009314BF42460822F2
:10EC080095F82810686A3B46FFF7FBFD0028C4D139
:10EC1800013E032EC1D8DFE806F002070B0F0D4BAB
:10EC28001B681C611C62B8E70A4B1B685C61F9E74A
:10EC3800084B1B689C61F5E7064B1B68DC61ACE779
:10EC48000A20AAE71020A8E70C20A6E70220A4E7DC
:10EC5800B4080020142600201FB50A460B2A4FF0DE
:10EC68000001CDE90011CDE9021107D00C2A13D01B
:10EC78000A2A0FD00B2005B05DF804FB012802D149
:10EC880020238DF80030684602F013F8002818BFDA
:10EC98000F20F0E73023F4E70B21F4E738B50546F9
:10ECA80002F002F8044678B97DB9094B1B680B21BC
:10ECB8009878FFF7D1FF38B90C21FFF7CDFF18B9C5
:10ECC8000A21FFF7C9FF00B10F24204638BD00BF55
:10ECD800142600202DE9F04380468FB00C461746D5
:10ECE800002A6BD0002969D0002529461D2206A8D4
:10ECF800059504F0A3FE8DF81350344D2B680DF1E3
:10ED080014099E88CDF804900DF1130302933B7902
:10ED180000933B6832462146404601F0E6FF002852
:10ED28004ED138683A79494602F052F9384600F02F
:10ED38004FF8002846D13C7AFA79BB79240444EA92
:10ED480002241C432B689A6894423DD99C609DF824
:10ED580013000B21FFF780FF034658BB0C21FFF778
:10ED68007BFF034630BB0A21FFF776FF034608BB4B
:10ED78007B7ABA7AFF7A3F0447EA02271F433A466A
:10ED8800334621460920FFF719FD034690B933465B
:10ED98003A4621460820FFF711FD034650B92A6874
:10EDA8009DF8131091700021D1604FF0FF31C2E936
:10EDB8000411916118460FB0BDE8F0830A23F9E702
:10EDC8000F23F7E71023F5E70323F3E714260020C2
:10EDD80010B50446002845D00168002942D011F832
:10EDE800013B43710322063002F0F2F82046032269
:10EDF80050F8091B043102F0EBF82168CB79E36085
:10EE08000A7A43EA0223E3604A7A43EA0243E36068
:10EE18008A7A43EA0263E360CB7A23740B7B6374D8
:10EE28002379212B1AD110220D3104F1120002F09E
:10EE3800CFF81D222168501C8B5C6362085C43EA92
:10EE48000023901C6362085C033243EA0043636258
:10EE58008A5C43EA02636362002010BD112B03DC65
:10EE68000D22E7E70220F8E70120F6E710B504468F
:10EE7800002854D00168002951D00B7843714B7891
:10EE880083608A7843EA02238360CA7843EA0243AC
:10EE980083600A7943EA026383604B7903738B7951
:10EEA800C381CA7943EA0223027BC38102F00F02BD
:10EEB8000831103002F08CF8237B002203F00F0396
:10EEC80084F8202084F82820227903F10800111AF8
:10EED80004290DDD21680933043AD21A085C84F844
:10EEE8002000D2B2606A84F82820194402F070F831
:10EEF800237922681A44002012F8043CE36212F8CD
:10EF0800031C43EA0123E36212F8021C43EA0143AB
:10EF1800E36212F8012C43EA0263E36210BD0220A7
:10EF2800FCE710B5044660B3036853B30279162AA8
:10EF380029D942791A700146082251F8060B013086
:10EF480002F050F82146082251F80E0B093002F061
:10EF580049F82368E28A5A74E38A22681B0A937480
:10EF68002368A269DA74A36922681B0A13752368E7
:10EF7800628B5A752368E27E9A75172323710020E5
:10EF880010BD0120FCE70220FAE738B50446002846
:10EF980063D00168002960D0037B90F8282003F033
:10EFA8000F03002A57D108332079043213449842BA
:10EFB80055D363790B702368A2685A70A3682268D6
:10EFC8001B0A937023686289DA702368E27A1A71DF
:10EFD8002368227B5A712368E2899A71E38922683F
:10EFE8001B0A2146D371227B51F8100B02F00F0245
:10EFF800083001F0EDFF237B94F8282003F00F037D
:10F0080003F108052AB1226894F82010515503F13C
:10F018000905206894F82820616A284401F0D8FF7F
:10F0280094F828302268E16A2B44D1545A1CE16ACA
:10F03800206892B2090A81549A1C2168E08D92B224
:10F048008854DA1C216894F82F0092B2043388544B
:10F058002371002038BD0933A6E70120FAE7022012
:10F06800F8E70000024B1A8810431880704700BF69
:10F078001826002008B5074B1B883BB1FEF728FA75
:10F0880000280CBF00206FF0020008BD6FF00100DF
:10F09800FBE700BF1826002010B5034B00241C8096
:10F0A800FEF70CFA204610BD18260020B0FA80F0B2
:10F0B8004009704782B018B9084602B000F0D0B8CD
:10F0C800002002B0704710B9084600F083B97047B5
:10F0D80010B9084600F09AB9704703460846114629
:10F0E8000BB900F0E7B90020704710B9084600F0E6
:10F0F80045BD704710B9084600F008BA00207047AF
:10F1080010B40446084611461A46019B14B910BCAF
:10F1180000F01ABA10BC70470346084611460BB9EE
:10F1280000F044BA0020704710B40446084611465F
:10F138001A4614B910BC00F0B1BA002010BC7047D0
:10F1480030B40546084611461A46DDE902341DB9B1
:10F15800029430BC00F02EBB002030BC704710B9C0
:10F16800084600F0DFBB0020704710B9084600F0E1
:10F1780043BD0020704710B9084600F0EEBB0020E0
:10F18800704710B9084600F0EBBB002070470346F3
:10F19800084611460BB900F005BC0020704710B4B2
:10F1A8000446084611461A46019B14B910BC00F0E3
:10F1B800FBBB092010BC704710B9084600F03CBDE5
:10F1C800704710B40446084611461A4614B910BCD4
:10F1D80000F05CBDC8B210BC704700000048704722
:10F1E80003000101064B10B51B6A0446984730B16D
:10F1F8000448054B204498428CBF0020012010BDD4
:10F2080014450108403576C9405DC600F0B5114B7C
:10F2180085B00C4610491F56054601F045F80F4BBE
:10F22800E4B25E6A072D4FF00103CDE902430146BF
:10F238000AD105220023CDE900234FF47A727A43DC
:10F248001846B04705B0F0BD08220020CDE90020DF
:10F258003A46F5E7D73E0108B03E010814450108D3
:10F268001FB5002300930378013B382B00F28580FB
:10F27800DFE803F01D238383832083838383404255
:10F28800444B835356595C5F6265836D206F747974
:10F298007B7E7E80872583838383838383838383A5
:10F2A800838383898B908383899083929600C37824
:10F2B800002B62D0022300935FE08378F8E743785D
:10F2C8008DF8043007238DF805308378003B18BF8C
:10F2D80001235B008DF8063010238DF80730334B7F
:10F2E8001B6801A803F59062CDE9022300F0BCFF7A
:10F2F800009042E04023DEE72023DCE7827890F9A3
:10F30800013042B92A4AD35CD5E7827890F90130B6
:10F318000AB9284AF7E7284AF5E740F6B833CAE7B2
:10F328004FF47A73C7E74FF4FA63C4E741F28833BE
:10F33800C1E741F27073BEE74FF48043BBE71F4853
:10F348004FF47A7101F028FE00F5FA60D0E71C4B03
:10F35800B1E7164B1B6803F59063ACE7134B1B68CA
:10F3680003F28C43A7E71023A5E7104B1B68A2E71D
:10F378000123A0E74FF083430093009805B05DF8A0
:10F3880004FB104BF8E7104B95E740F21123ADF85A
:10F398000030F2E703238EE790F901300B4AB2E719
:10F3A8000B4990F9010000F07FFFA1E7202600201B
:10F3B800E73E0108F73E0108EF3E010818FCFFFF91
:10F3C80000EA06379A99094040F70937D73E0108FD
:10F3D800B03E010837B50B4B02781B680C2101FBC6
:10F3E80002335B7A03EB4304074B1D680369009300
:10F3F800C3684278816805EBC40000F0D5FC03B00F
:10F4080030BD00BF202600201C26002030B587B064
:10F41800027A6423ADF80030012A4FF00003CDE9E9
:10F428000133CDE9033301468DF802308DF81430ED
:10F4380027D0022A2ED012BB006800B34B68F3B164
:10F44800194A1A4C106069461822236001F0C0FD61
:10F45800174B246893E807000C3384E8070093E807
:10F46800070004F10C05032385E80700A4F88C3491
:10F47800012204F28C4104F5906000F086FC07B08C
:10F4880030BD0A4908684360036100F28C4100F509
:10F498009060F2E7054B1B68B3F88024B3F88C142E
:10F4A8000A43A3F88024EAE71C260020202600202F
:10F4B800043C010808B503460A2924D8DFE801F00E
:10F4C80006232323230B161B23212100BDE8084014
:10F4D8000068FFF787BE90F900009978072271B994
:10F4E80000F013FC003818BF012008BD052293F96D
:10F4F80000000021F4E790F900005978EEE70221B6
:10F50800EEE70722F3E70020EFE7000010B50479E3
:10F518001CB1012C0BD0002010BD0A4B01681B68E0
:10F52800012203F5906000F030FC0120F4E7054B60
:10F5380001681B68224603F28C4000F026FC204636
:10F54800EAE700BF20260020F7B50728144D1C461F
:10F55800A8BF072058700E462946174600F0A4FE9B
:10F5680094F90130A070072B13D1322000F09CFDD4
:10F578000C4BDB6D0546984704F10C020834034632
:10F58800019200943A463146284600F092FD03B0B5
:10F59800F0BD054A55F82310D05C00F07DFDE7E783
:10F5A800B03E010814450108D73E01082DE9F04F87
:10F5B800344F90F901607B68D0F804908BB0044612
:10F5C800884698470546002859D1E37C73B92E4AE6
:10F5D8002378126803EB4303990002EB8303D3F803
:10F5E8000490B9F1000F01D152F80190274B484619
:10F5F80013F906B0FB689847A37CD7F818A02289AE
:10F608000993072E28D100230121CDE90223204A9E
:10F618000693CDE90431CDE907330521CDE9002171
:10F628004FF47A7202FB0BF24CF250311846D04775
:10F63800637C13B3174B995D7B6D0D31C9B22846B6
:10F648009847E07C3246494600F040FE88F8006062
:10F6580001200BB0BDE8F08F002101250823CDE97A
:10F668000013CDE90715CDE90511CDE90311029283
:10F67800A1782B465A462846D9E7074BDBE70020F6
:10F68800E7E700BF1445010820260020D73E0108FF
:10F6980085450100F73E0108E73E01082DE9F04FD6
:10F6A8008DB090F90130DFF8F8A0DFF8F890CDE9D7
:10F6B8000A123D4A017812F903B0DAF800203B4BF0
:10F6C8000C2505FB01221B68527A182101FB023325
:10F6D800044693F9021090F9020000F0E0FD344965
:10F6E800064694F9010000F0DFFDA26861688046D3
:10F6F800304600F006FD2178DAF80020D9F80C3001
:10F708006943074650589847D9F81C309C4694F9E5
:10F7180001300025072B4FF47A63CDE90753CDE973
:10F7280005552DD10123CDE903530523CDE9015317
:10F738004FF47A7303FB0BF300933946434646F2C2
:10F74800A81228466746B8472378DAF800200C2123
:10F758004B4394F90110D05800F0DAFDA18994F9CF
:10F768000100FFF753FD0B9B217B1860D9F854303B
:10F77800284698470A9B01201E700DB0BDE8F08FFF
:10F7880001200823CDE90350CDE901032A46CDF82D
:10F7980000B0654643463946A84701200546D3E7E9
:10F7A8002026002014450108D73E01081C26002009
:10F7B800B03E01082DE9F04F8FB0002405468A4677
:10F7C800914698460494ADF81440ADF802400726D7
:10F7D8004FF0010B2B7AA34206D9686804A920448C
:10F7E80000F0F4FB00285DD102238DF8083002A850
:10F7F8006B7A8DF80A30FFF733FDAB7A8DF81D3040
:10F808009DF811308DF81E309DF812308DF81F309C
:10F818009DF810308DF82030EB7A8DF821302B7B55
:10F828008DF822306B7B8DF8233010238DF81C6007
:10F838008DF824303A4E8DF82C000DF102030A930E
:10F84800072332688DF82D30ADF834302B680C92D0
:10F8580006930DF1120204AB0DF1110106A800F098
:10F86800CFFB072805460BD130680C22002100F594
:10F87800906001F0C1FB3368BDF80220A3F8802432
:10F888009DF811308AF800309DF8123089F8003060
:10F898009DF8103088F80030189B28461C700FB06F
:10F8A800BDE8F08F9DF81330BDF81470ADF8027004
:10F8B8002044C4B2F3B917B3194A002011680726C7
:10F8C80002464FF00C0C062B1BD10CFB00FE51F826
:10F8D8000EE0BEF1000F04D00BFA00F23A4397B2E3
:10F8E800012201301028EED1002A3FF473AFADF8A1
:10F8F80002706FE75A1E042A01D9062BDCD00626AF
:10F9080068E747FA00FE1EF0010FEAD00CFB00FE84
:10F9180051F80EE0BEF1000F08BF0626E1E700BF70
:10F928002026002038B505464068FFF75BFC072213
:10F93800841D002195F90000E4B200F0E6F908B949
:10F9480004F0FD0495F901000722002100F0DDF91B
:10F9580008B904F0FB04204638BD002070470000B9
:10F9680010B503780F2B044618D84068FFF73AFC07
:10F9780022780B4902EB42020968831C01EB8200E2
:10F9880051F82220DBB21AB903F0FD0358B210BDBA
:10F99800032B06BF626842600223F7E70020F6E700
:10F9A80020260020022070472DE9F0413A4D0446F8
:10F9B800286896B00E46904600211F460122032370
:10F9C80000F59060CDE90411CDE906118DF80C1011
:10F9D8008DF80D10ADF80E3000F0B9F930B92A687D
:10F9E800B2F8803443F00303A2F880342A68637ABB
:10F9F8008DF8203002F59061CDE90912274A94F973
:10FA0800083012680B921022ADF830200DF10E026A
:10FA18000D9222680E9262680F92D4E90301A27ACD
:10FA28008DF8402001228DF8412011AA82E80300B8
:10FA3800227DE18A8DF8213018468DF84C20FFF799
:10FA4800E5FB08AB15930DF10D0314900093CDF869
:10FA5800048003AB04AA39460EA800F0C1FB044693
:10FA680078B99DF80C10013901F096FA00F15803A5
:10FA78000DEB030010F8483C3370204616B0BDE883
:10FA8800F0810C2801BF2A68B2F8803443F00303E0
:10FA9800A2F88034F1E700BF202600201C260020B1
:10FAA800F8B50679012E054601D80620F8BD0F2EB7
:10FAB8002BD80368187A40F303000722002140B2CC
:10FAC80000F023F92B680446187A40F30310072244
:10FAD800002140B200F019F9A8B1B4FA84F464091D
:10FAE80029680B7A086843F3030243F3031352B2FD
:10FAF8005BB29A42C8BF0124FFF774FB48B9002CD7
:10FB0800D3D10420D2E70124EAE70320CEE7052079
:10FB1800CCE7002CFBD10C4F29683B6806EB46006C
:10FB280003EB80000C2201F053FA3A680C2303FB24
:10FB3800062320465C72B2F880140123B3400B43BD
:10FB4800A2F88034B2E700BF2026002010B4017864
:10FB580001290ED9084B18680C234B43C4180022FE
:10FB6800C250C4E9012200F5906010BC102200F0D8
:10FB7800D5B8002010BC7047202600202DE9F041A0
:10FB880086B050238DF814300379102B074630D1F6
:10FB98000368DD7B6DBB0224A8466426062C14D8B6
:10FBA8003A68535D03932A44517843EA0123039347
:10FBB800927843EA02437343CDE9033863B9684650
:10FBC8008DF80040FFF7C2FF0DE0CDF80C808DF8EE
:10FBD8001480CDF81080F2E703AB01A801938DF8EB
:10FBE8000840FFF75DFF0134E4B2102C05F103056E
:10FBF800D4D106B0BDE8F0811FB502680379116859
:10FC080051B901A88DF80430FFF7A0FF78B900209A
:10FC180040B205B05DF804FB02A802928DF80C30E2
:10FC2800FFF73EFF0628F2D8024B185CF0E70320E6
:10FC3800EEE700BFD03E010870B5114E017832687A
:10FC4800104B0C2505FB01221B68527A182101FB79
:10FC58000233044693F9021090F9020000F01FFBEA
:10FC68002378326861686B43D558A26800F049FA76
:10FC7800054BA289DB6B01462846BDE87040184752
:10FC8800202600201C26002014450108074B9B56FF
:10FC9800C91A431E5842584140008842B8BF084616
:10FCA8000528A8BF0520C0B2704700BFDF3E010885
:10FCB800F0B59A42069D03DB9DF914309A4220DD87
:10FCC8000020F0BD03EB430331F814C005EB8303B8
:10FCD80000264CFA06F7FF0707D51F7A07F00F0E24
:10FCE800724502DBB2EB171F0DDD0136102E03F152
:10FCF8000C03EED10134E4B22301DBB29842E1D81F
:10FD0800DEE70024F8E70120DBE7884204DB9042C5
:10FD1800CCBF0020012070470020704710B514099F
:10FD2800B4EB111F03464FEA11100ED391420CD2C7
:10FD380002B201F00F0133F81240012000FA01F17C
:10FD480024EA010123F8121010BD0020FCE7F0B5E9
:10FD580028B100EB410501270020914200D3F0BDF6
:10FD6800002435F802CB234607FA04F636EA0C06D7
:10FD780008BF013304F1010408BFDBB2102CF3D132
:10FD880018440131C0B2C9B2E7E710B500B149B9AA
:10FD980010BD31F8134020F813400133DCB2A24201
:10FDA800F7D8F5E70023F9E782B030B50488049363
:10FDB8006AB9B3F5616F18D349F6AF2542F21072EC
:10FDC800AB4298BF4FF47A72944238BF1446012C64
:10FDD80038BF01246143BDE83040C3688B428CBF03
:10FDE8005B1A0023C36002B070476422ECE700008E
:10FDF8002DE9F04F91B01546DDF86C8004939DF81D
:10FE0800683009930C46064603F0C2FB684ADFF8DF
:10FE1800A4B10590A8F5F633303BB3FBF2F3534396
:10FE280003F5F63203F5A83303F5C07303931823DB
:10FE380013FB054330320692089300254FF0FF3A32
:10FE4800089BA34207D1002D14BF50464FF0FF3046
:10FE580011B0BDE8F08FBDF97030ADF82C300B99BA
:10FE6800CDF86C804046CDF8288003F021FBB4F82B
:10FE780000906EB9B8F5616F5BD349F6AF2242F2D4
:10FE88001073904598BF4FF47A73994538BF9946D7
:10FE98004B46012B38BF01230793002E52D1B9F1ED
:10FEA800640F48D1A0605F46A1680EA803F022FB4A
:10FEB8000F9B0093DDE90A120E9B0CA803F079FA58
:10FEC800049B0C9A0BB9099B2BB12369BB4202D145
:10FED800394B9A420DD9394BE760984509D9002327
:10FEE800ADF83430069B0D990C93184603F0E0FAF0
:10FEF800A060606800B9E760276126B103F052FB93
:10FF0800E3680344E360D4E903329342059B1D99F7
:10FF18006360079B88BFE2604B43E168994202D265
:10FF28000498A8B9A6B101231D442375EDB218346D
:10FF380086E76423A9E7B9F57A7F0ABF204F214FE6
:10FF4800A060B1E7049B0BB9C4F80CB05F46D0E7DA
:10FF580000209342207506D85B1A9A4505F10105E1
:10FF680028BF9A46EDB2002EE1D1B9F1640F164AC6
:10FF7800ADF8346019D049F6B023B9F57A7F18BFC7
:10FF88001346904584BF039A9B180C931C9B0093BF
:10FF98000CAF97E806001B9B384603F00AFA97E86F
:10FFA800030003F085FA8246C1E74FF46163E8E78E
:10FFB8008051010040771B007F5101002FEC0100A8
:10FFC80080A81201002E930230EC01000378032B65
:10FFD80014D1437803F00F021B098A704B708378A1
:10FFE8008B80C27843EA02238B800379C3F3021221
:08FFF80003F00F03CA700B7047
:020000040801F1
:1000000005207047002070472DE9F3479846437953
:10001000057990F907609146044690F906208A46D2
:1000200083B190F9087075B30F2A12D194F90920A1
:100030000F2E1ED194F90A60072D24D1002F08BF7E
:10004000012720E090F90B7090F9092090F90A60DF
:10005000E9E7A369019394F915300093216994F9B4
:100060001430207BFFF728FE0028E1D105F0FD05C4
:10007000DEE794F91D30B3420FDC94F91C30B34233
:10008000DADA05F0FB0528468AF8002089F80060D6
:1000900088F8007002B0BDE8F0871E46CCE700008B
:1000A000024B03FA00F0B0FBF1F0704740420F0042
:1000B0004FF4FA53B3FBF0F0704730B54FF47A7554
:1000C0000C1F6A4300FB042252001EBF00F1FF34E4
:1000D0001219B2FBF0F2914238BF1146039A116037
:1000E000820048431CBF013040084FF47A71121A55
:1000F00001FB1323002BCABF03F2E73393FBF1F19B
:10010000B3FBF1F1049B196030BD38B540001446D3
:100110000D46F1F77FFC01462846F1F7C9FB214661
:10012000F1F7C6FBF1F7B8FA03F0DAFCF1F794FB4C
:1001300040B238BD2DE9F74F019300231F469C467E
:100140001C01058A5FFA84FE04F0F004A54206D87B
:10015000019B82F800C01F7003B0BDE8F08F0EEB6A
:100160004E054FEA4309AD000024466836F80960A1
:100170002641F60727D5866806EB050A765916B399
:10018000067836B9466926B136F809602641F60781
:1001900019D59AF8086090F901B046F303084FFAB0
:1001A00088F8D8450FDC46F3031676B25E450ADBC5
:1001B0009AF8096006EB4608C66806EBC806367D65
:1001C0004EB90137FFB20134102C05F10C05CCD12A
:1001D0000133DBB2B4E70CF101060EEB040801F8C1
:1001E0000C805FFA86FCEEE72DE9FF470446406885
:1001F000DDE90C671D468A46914603F0D7F923686E
:100200001B1A3B604FF000080123337085F8008013
:10021000636813B12368834224D8CAF80080D4F8F5
:100220001CC0A3699CF800E00393D4E9030101AB6F
:1002300083E80300237D0093DCF80C10237A627AB4
:100240007046FFF7D9FD334638602A46E0694946D3
:10025000FFF770FF2B782BB1C7F80080002004B0A7
:10026000BDE8F0873378002B14BF0B200C20F6E795
:1002700037B590F9002090F90250954204460FD00E
:10028000013A52B295420BD0A368019394F9013020
:1002900000936168E0782B46FFF70EFD0028EFD051
:1002A000104603B030BD8842B8BF08467047000012
:1002B00051F82000054B984205D0054BC31A58420F
:1002C0005841400070470120704700BF90D00300A4
:1002D00020A1070005281FB50ED80C4B53F820307D
:1002E0000093CDE901120A4B01220021022002F005
:1002F00069FE05B05DF804FBCDE90012054B012253
:100300000021022002F05EFEF3E700BF6C3F01080F
:10031000FF3E01081E3F010807B5054BCDE900016E
:1003200001220021022002F04DFE03B05DF804FB23
:100330003A3F010810B5102204460021F13000F0C8
:100340005FFE0021C4F814112046F022BDE81040E1
:1003500000F056BE02460846102100F0A5B92DE96E
:10036000F0430446D0F8140185B00E46154604F259
:10037000011988B3C0F110089045474628BF1746B9
:10038000BAB2484400F028FED4F814313B440F2B95
:10039000C4F814312DD9A8452BD204F1F00304F58B
:1003A000807113F8012F187C8B4282EA00021A70C8
:1003B000F7D104F1F10810224146684600F00CFE26
:1003C00022466946684600F0E9F91022694640462F
:1003D00000F002FE3E44ED1B04F5807804F1F107C5
:1003E000102D09D8AAB23146484600F0F5FDC4F8F0
:1003F000145105B0BDE8F08304F1F003711E13F849
:10040000012F11F8010F434582EA00021A70F6D15C
:1004100010223946684600F0DFFD224669466846EC
:1004200000F0BCF910226946384600F0D5FD1036C0
:10043000103DD5E7F0B589B00C46102200210546E5
:10044000684600F0DDFD22466946684600F0A6F9E0
:100450009DF90030002B6A464FF0000143DA137813
:1004600012F8010F01315B0043EAD0130F2902F8A3
:10047000013CF4D19DF80F305B0083F08703D4F882
:100480001401DBB210288DF80F303BD104F58073D6
:10049000694604F5887013F8016F11F8012B984232
:1004A00082EA06021A70F6D104F1F00304F58071B5
:1004B00013F8012F187C8B4282EA00021A70F7D1E0
:1004C00010220DEB020004F1F10100F085FD22463F
:1004D000294604A800F062F910220021684600F0C5
:1004E0008FFD09B0F0BD137812F8010F01315B00E8
:1004F00043EAD0130F2902F8013CF4D19DF80F30E4
:100500005B00BCE79DF90030002B6A464FF000010C
:1005100037DA137812F8016F01315B0043EAD61322
:100520000F2902F8013CF4D19DF80F305B0083F0F5
:100530008703471CDBB28DF80F30102F04EB00034C
:10054000C0F10F064FF0800288BF002600F58170D1
:1005500083F801210021324620443E4403F072FA20
:10056000C4F8146104F58073694604F5887013F8C3
:10057000016F11F8012B984282EA06021A70F6D137
:1005800092E7137812F8016F01315B0043EAD6134A
:100590000F2902F8013CF4D19DF80F305B00C8E749
:1005A0000A780378534003704A7843785340437085
:1005B0008A78837853408370CA78C3785340C37075
:1005C0000A790379534003714A794379534043715F
:1005D0008A79837953408371CA79C3795340C3714F
:1005E0000A7A037A534003724A7A437A5340437239
:1005F0008A7A837A53408372CA7AC37A5340C37229
:100600000A7B037B534003734A7B437B5340437312
:100610008A7B837B53408373CA7BC37B5340C37302
:10062000704710B50B7814786340037054784B789A
:100630006340437094788B7863408370D478CB7830
:100640006340C37014790B796340037154794B791B
:100650006340437194798B7963408371D479CB790A
:100660006340C371147A0B7A63400372547A4B7AF5
:10067000634043728B7A947A63408372D47ACB7AE4
:100680006340C372147B0B7B63400373547B4B7BCF
:1006900063404373947B8B7B63408373CB7BD27BC0
:1006A0005340C37310BD0000A1F11003DBB2102B47
:1006B0002DE9F04704D8374C24FA03F3DB0705D4BF
:1006C000002382F8F030FF20BDE8F087531E441865
:1006D000A0424ED101F11C039B005FFA83F9C3F3E2
:1006E0000313013B2C4D82F8F03001240B46D61841
:1006F000B3FBF1F001FB103010F0FF0016F804AC72
:1007000016F803EC16F802CC16F8017C36D115F871
:100710000E8015F80CE015F807C015F80A70E0090E
:1007200000EB400084EA080800EBC0006400C0B29F
:10073000E4B24440C246581AC0B212F800808AEAB5
:10074000080A02F803A01044043390F801808EEAEE
:10075000080E86F801E090F802E08CEA0E0C86F8AC
:1007600002C0C078DBB247409945F770BFD800207F
:10077000AAE710F8015B03F8015FA9E71829DAD9A5
:10078000102801BF15F80AA015F80EE015F80CC0E6
:10079000EF5DD0E701010100844101082DE9F04F30
:1007A000A3B092F8F0301D911B920193002B00F042
:1007B000538101461EA8FFF734FF1B9BA74CA84D91
:1007C000A84E10330293002303939DF87C000490FD
:1007D0009DF886000590205C06909DF87B000790B0
:1007E000205C089004989DF881C0205C099014F862
:1007F0000C000A909DF880000B909DF885009DF8F4
:1008000078809DF87DE09DF882A09DF887900C90FF
:100810009DF87A00029B1C9314F80A2014F8093002
:1008200014F8081014F80E700D90205C0E909DF8CE
:100830007F000F90205C10900B98205C11900C981A
:10084000205C12909DF8840013909DF8790014901C
:100850009DF87E001590205C16909DF883001790FF
:10086000205C18901398205C19901498205C1A90C2
:100870000398013003900298DDF804B01030029024
:100880009DF80C00834536D88DF878108DF87A20C5
:1008900009990E9A8DF87C108DF882201199069A8C
:1008A0008DF880108DF87E201999169A8DF8841095
:1008B0008DF886200A99189A8DF87D108DF887207A
:1008C0001299109A8DF87B301B9B8DF881108DF852
:1008D00083201A99089A1D988DF885108DF87F202D
:1008E0001EA903EB0B128DF87970FFF79AFE00201A
:1008F00023B0BDE8F08F15F808B082EA03008BEA58
:10090000000016F80EB080EA0B008DF8780015F89C
:100910000E004B40434016F80A0043408DF87930F2
:1009200081EA070315F80A10594016F809305940B2
:1009300016F808308DF87A107A40534015F80920DF
:1009400053408DF87B30089A069B5340049AAA5C6A
:10095000534016F80C2053408DF87C30DDE9083206
:100960005A4015F80C305340059AB25C53408DF84C
:100970007D30DDE909325A40059BEB5C5340079A14
:10098000B25C53408DF87E30069B0A9A5340049A1D
:10099000B25C5A40079BEB5C5A408DF87F200E9B5F
:1009A000109A53400B9AAA5C53400C9AB25C534085
:1009B0008DF88030DDE910325A400C9BEB5C5340DF
:1009C0000D9AB25C53408DF88130DDE911325A4006
:1009D0000D9BEB5C53400F9AB25C53408DF8823014
:1009E000129A0E9B53400B9AB25C5A400F9BEB5CE1
:1009F0001C995A408DF88320169B189A5340139ADD
:100A0000AA5C5340149AB25C53408DF88430DDE9FF
:100A100018325A40149BEB5C5340159AB25C534019
:100A20008DF88530DDE919325A40159BEB5C534057
:100A3000179AB25C53408DF886301A9A169B534031
:100A4000139AB25C5340179AAA5C1EA853408DF8C3
:100A50008730FFF7A5FDB8E6FF2049E7844101088C
:100A6000843F01088440010808B538B1044A0549AB
:100A70001060D82200F0B0FA002008BD0220FCE788
:100A800024260020B44601080A4B1A6870B50023DA
:100A900002F1180503EB03142E5D864204D11834CD
:100AA00022440A60002070BD01330B2BF2D10320D9
:100AB000F9E700BF242600202DE9F041CCB006461E
:100AC000DDF8488117461C460D4631B3B8F1000FDA
:100AD00023D006A8FFF72EFC204601A9FFF7D4FF7C
:100AE0000446B0B9019906A80131FFF733FC26B1DD
:100AF0001022314606A8FFF732FC3A46294606A8DE
:100B0000FFF72DFC06A902A8FFF794FC029BC8F88A
:100B1000003020464CB0BDE8F0810224F9E7000027
:100B200030B595B013A90446FFF7AEFF002830D1C9
:100B30001B490C2303FB00F2555CA5422BD1139BF0
:100B4000187C1090D87B0F90987B0E90587B0D905E
:100B5000187B0C90D87A0B90987A0A90587A099062
:100B6000187A0890D8790790987906905879059066
:100B700018790490D8780390987802900A445B78AA
:100B80000193936800930022064B1146022002F065
:100B900019FA15B030BD01300B28CBD1F9E700BFF1
:100BA000FC430108844201080B2B10B402D810BC8E
:100BB000FFF782BF032010BC704730B50D4685B0EB
:100BC0001446014668B103AA002000922A46039009
:100BD000FFF772FF18B90398001B18BF012005B07A
:100BE00030BD0220FBE72DE9F0430D46BFB01446AF
:100BF0009946804620B31BB311F00F0122D1F02299
:100C000001A800F0FDF920466946FFF73DFF0446C4
:100C100048B9009801AA10210130FFF745FD2E4682
:100C2000AF1BFFB21EB920463FB0BDE8F08301AA5A
:100C300009EB070108EB0700FFF7B0FD103EEFE7F7
:100C40000224F0E70524EEE7F0B5184E34680246BA
:100C500085B00846002304F1180103EB03154F5D2E
:100C600097421ED10D2A05F1190513D10023CDE9B4
:100C70000033CDE902330C2210216B46FFF7B3FF9E
:100C80000446306810226946284400F0A5F9204641
:100C900005B0F0BD01461022601900F09DF9002456
:100CA000F5E701330B2BD8D10324F0E724260020ED
:100CB00009B1FFF7C9BF022070471FB51446A0B1A4
:100CC0000C2A01D10B2912D10023CDE90033CDE943
:100CD00002330A466B461021FFF785FF18B96946B3
:100CE0002046FFF7B1FF04B010BD0220FBE7032050
:100CF000F9E7F8B51E46DDE907479DF818505BB3E4
:100D000054B34FB3212D29D819462A46204600F066
:100D100063F90122631C691EB018FFF764FFF8B97C
:100D2000E37ADB093B70EBB96319204613F8012C19
:100D300013F8021C120642EA014213F8041C0A438B
:100D400013F8031C012342EA0122291FFFF735FF94
:100D5000003818BF0120F8BD0220FCE70520FAE7A3
:100D60000720F8E70420F6E710B5044628B1044B45
:100D70005B6998472060002010BD0220FCE700BF9F
:100D80001445010808B5014630B1044B0822186823
:100D900000F022F9002008BD0220FCE724260020F4
:100DA00008B530B1044B0822196800F015F900208D
:100DB00008BD0220FCE700BF242600207FB5124EAC
:100DC0000023044602A801930D46FFF7E9FF3368AC
:100DD0005B6901936CB102AA082312F8011B41B9A7
:100DE000013B13F0FF03F8D102A8A04702A8FFF7C8
:100DF000C9FF35B1019B23B901A8A8473368019AFF
:100E00005A61002004B070BD2426002008B50146B8
:100E100038B1054B18680822104400F0DDF80020B6
:100E200008BD0220FCE700BF2426002008B538B129
:100E3000044B19680822114400F0CEF8002008BDC8
:100E40000220FCE724260020034B1B6802280CBF6D
:100E500019615961002070472426002041B1054BDB
:100E60001B6802280CBF1B695B690B600020704780
:100E7000022070472426002030B58FB0002405469C
:100E80000CA80994FFF78CFF9DF8373007939DF865
:100E9000363006939DF8353005939DF83430049331
:100EA0009DF8333003939DF8323002939DF8313032
:100EB00001939DF830300093224621461E4B0220BC
:100EC00002F080F80AA8FFF7B1FF9DF82F300793D2
:100ED0009DF82E3006939DF82D3005939DF82C300B
:100EE00004939DF82B3003939DF82A3002939DF8CC
:100EF000293001939DF82830009322460F4B21465C
:100F0000022002F05FF809A92846FFF7A7FF9DF825
:100F1000243003939DF8253002939DF826300193E9
:100F20009DF8273000932246054B2146022002F00F
:100F300049F80FB030BD00BFE04201081E43010870
:100F40005C43010808B50020FFF7EAFD0120FFF728
:100F5000E7FD0920FFF7E4FD0820FFF7E1FD002091
:100F6000FFF78AFF002008BD10B504460B20FFF7ED
:100F7000D7FD0C20FFF7D4FD0920FFF7D1FD082095
:100F8000FFF7CEFD0A20FFF7CBFD2046FFF774FFE9
:100F9000002010BD014B1860704700BFBC08002046
:100FA0000B4A30B514680B4D43F2390305FB04338B
:100FB0001360091A6FF00042B3FBF2F2C2EBC27287
:100FC00001319B1A93FBF1F201FB1233184430BD3F
:100FD000BC0800206D4EC64101380A44914200D140
:100FE000704711F8013B00F8013FF7E710440A444D
:100FF000914200D1704711F8013B00F8013DF7E73D
:1010000002F020BD30B530B10A4D01444FF0FF333E
:10101000814201D1D84330BD10F8012B5340082242
:1010200043F30004013A2C4092B284EA5303002AAD
:10103000F6D1EDE72083B8ED01207047054B4FF462
:1010400000529A62044B1B6813B15B6803B11847E6
:10105000704700BF0004004828270020054B4FF4CC
:1010600080529A62044B1B6813B1DB6803B11847C6
:10107000704700BF00040048282700200120704767
:101080000120704701F048B901F036B910B501F000
:1010900019FE0E21044640F61F1001F02DF92046DE
:1010A000012101F0F9FDBDE8104001F0D7BA0000C0
:1010B00070B50C4E01EB40030D46B3654FF6FF7162
:1010C000002304461A46084601F05EFB96F85600D7
:1010D000002101F0E1FD29462046BDE8704001F005
:1010E00095BA00BF4427002010B5044601F0AAFEBF
:1010F00001281CD101F0AEFE34B11248214602F0A5
:1011000017FB104802F0DAFA0F4C104B00214FF495
:101110008052A1659A6194F8560001F0BDFD637894
:101120006BB16FF07F40BDE8104001F053BA00236F
:1011300040F262211A46084601F026FBDCE7A0686F
:101140008001F0E72C2700204427002000040048FD
:10115000002001F0BFB9000008B501F0C7F804385D
:10116000C0B2032896BF024B0020185C08BD00BF28
:101170001045010808B501F0BAFD033008BD01F0C3
:1011800049B901F009B908B501F000FD00B208BD88
:1011900038B50D46144601F05DFB284601F092FD7E
:1011A0000E21054640F61F1001F0A6F82846012141
:1011B000074D01F071FD01F051FA4FF47A7161436E
:1011C000284602F0B5FA2846BDE8384002F076BA63
:1011D000A027002001F03EBB08B5084B002193F882
:1011E000560001F059FD00234FF4C0711A4608461D
:1011F00001F0CAFABDE8084001F024BA44270020F3
:1012000010B5044601F01EFE01281CD101F022FE9B
:1012100034B11248214602F08BFA104802F04EFA1F
:101220000F4C104B00214FF48052A1659A6194F845
:10123000560001F031FD63786BB16FF07F40BDE87F
:10124000104001F07DB9002340F262211A460846A1
:1012500001F09AFADCE7A0688001F0E72C27002073
:10126000442700200004004808B54FF0040001F0B6
:1012700017F9BDE808400220F1F738BC08B5002393
:101280001A461946184601F07FFABDE8084001F0F9
:101290006DB900001D4B73B51D4D186000241D482D
:1012A0006C70C5E90144AC6501F098FAAC8101F0BD
:1012B00003FA2146204601F04BFC2146042201207E
:1012C00001F0FCFA144E154D4FF6FF7123462246ED
:1012D000084601F059FAFFF7C7FF2246104B009469
:1012E0004FF0FF31304602F03DF90E4B009422469C
:1012F0004FF0FF31284602F035F9304602F090F900
:10130000284602B0BDE8704002F08AB928270020C4
:1013100044270020DD220108A02700202C270020E0
:101320003D1001085D1001080128084805D1084B4F
:10133000C17719700E3001F0A7BB437D012B03D19B
:10134000034B81751970F5E7704700BF44270020F3
:10135000C00800200D4B10B50446187358730120C7
:1013600000F016F85CB134214FF4E86000F0C4FFDF
:101370004421BDE8104040F2417000F0BDBF14218F
:101380004FF4E86000F0B8FF2421F2E74427002082
:1013900038B5114C0546207001F061FD052D04D8CB
:1013A000DFE805F0090B03171709032001F070FAB5
:1013B0000023637338BD0020F8E7012001F068FACC
:1013C000207B637B8342F5D06073BDE83840FFF734
:1013D000C1BF0220EAE700BF442700202DE9F04307
:1013E0001E4687B000230546CDE901330C4617465B
:1013F00001F027FD032D61D8DFE815F07B00C30065
:101400000E010400A27C082A04D94FF0FF3007B077
:10141000BDE8F083A16801A801F0DCFE2168002985
:10142000F3D042F210729142E37C864D51D80322F0
:10143000AA7385F83820E96385F844304FF0020834
:101440006368A17DDB002B820423AB74A37CDB00EB
:10145000EB7402294FF000032B75637D02D0227DCF
:10146000022A42D103F10F02D2B2012A01D9012B83
:10147000CBD1754B754A196803944FF0010903A845
:101480008DF8149001F0DAFC0028BED1287685F89A
:1014900017906875FFF75CFE4046FFF779FF6C48D0
:1014A00001F086FA6B4801F0EFFA01A800F084FF22
:1014B000208A00F055FFA08900F09AFF384601F01D
:1014C00001FC604C84F8560001F0C0FC666000200E
:1014D0009DE74FF00008E963890885F80E8085F8DC
:1014E000388085F844302964AAE7EB7529766A7557
:1014F000D0E72368002B88D0A27C082A85D8514DDC
:10150000A16801A801F066FE002385F83830226842
:10151000EA63E27C85F84420A269AB732A646268BE
:10152000A17DD2002A820422AA74A27C2B75D2004B
:101530000229637DEA7402D0227D022A1DD103F1C3
:101540000F02D2B2012A02D9012B7FF45EAF3E4BCB
:101550003E4A196803944FF0010803A88DF81480DF
:1015600001F06CFC00287FF450AF287685F81780D6
:101570006875FFF7EDFD00208FE7EB7529766A753A
:10158000F7E7304D012185F83810227885F8502092
:10159000637885F85130A37885F85230E3788B4230
:1015A00002D0022B03D03BB985F8533004E00B3A4C
:1015B000012A29D885F853104FF0010885F80E80CC
:1015C000A388AB83A379AB77E37985F82030237ABE
:1015D00085F82130FFF7BCFD4046FFF7D9FE1C48D7
:1015E00001F0E6F91B4801F04FFA95F85130062B4F
:1015F00040F689000AD100F08FFE00F0FB0140F6B2
:10160000890000F079FE59E70023CDE700F084FE61
:1016100040F00401C9B2F2E72368013BB3F57A7FD9
:10162000BFF4F3AE0320FFF7B3FE0648022380F8B1
:10163000383023688364162380F84C30383001F04A
:10164000B7F93BE74427002028270020A0270020E7
:101650007C270020522700202DE9F041002686B08B
:101660001F461446CDE9016680460D4601F0E9FBB0
:10167000B442764C16BF0123334637466370B8F147
:10168000000F06D0B8F1010F7CD0002006B0BDE8F5
:10169000F081AB68002B00F0D680EB68002B00F0E7
:1016A000D280AA7F082A00F2CE80296901A801F021
:1016B00091FD2868003818BF012000F0D9FF84F898
:1016C0003880AB68E36395F8203084F8443068686C
:1016D00001F05AFB84F80E8084F84500EB68DB00CB
:1016E0002382EB7FA374AB7FDB00E37495F821309A
:1016F000237595F82230002B3ED12A7D95F82410D1
:10170000A275022995F8232001D0022B36D102F1CF
:101710000F03DBB2012B02D9012A40F09480002391
:101720008DF814304A4B4B4A1968049503A801F010
:1017300085FB002840F0878001232076E3756075E3
:10174000FFF706FD0020FFF723FE434801F030F9C4
:10175000424801F099F901A800F02EFEA88B00F094
:10176000FFFD288B00F044FE4FF4FA53AA687B4338
:10177000B3FBF2F3A36088E7FF22BFE7E2752176AF
:101780006375DDE72B8E002B5DD095F83230A86AAB
:10179000012B0CBF95F814804FF0FF08003818BFDC
:1017A000012000F065FFF8B200F06EFF012184F81F
:1017B000381095F82C2084F8502095F82D3084F8B6
:1017C000513095F82E3084F8523095F82F308B42F6
:1017D00002D0022B03D03BB984F8533004E00B3A1B
:1017E000012A28D884F853102B8EA38395F8323021
:1017F000A377AB8E23840126A67384F81F80FFF79E
:10180000A7FC3046FFF7C4FD134801F0D1F8134898
:1018100001F03AF994F82130B34240F236700CD11D
:1018200000F07AFD00F0FB0140F2367000F064FD3C
:101830004FF6FF739EE70023CEE700F06DFD40F00A
:101840000401C9B2F0E74FF0FF301FE74427002042
:10185000282700202C2700207C270020522700204A
:101860002DE9F04F85B082460E9DBDF840B09DF841
:1018700044709DF84890019288461E4601F0E1FAB6
:10188000BAF1010F524C54D0BAF1040F00F091801C
:10189000BAF1000F3AD10B22304684F8442084F884
:1018A00038A0E56301F070FA019B23644FEACB0393
:1018B000B9F1000F238241F60403638214BFF223BF
:1018C0000123E37587F001070123237684F845009F
:1018D00084F80EA084F814A06775FFF739FC504611
:1018E000FFF756FD04F1380001F062F804F10E0034
:1018F00001F0CAF8374A1068516802AB03C302A866
:1019000000F05AFD40F2FF1000F02AFD404601F0C1
:10191000D9F90E2184F8560040F61F1000F0ECFCB7
:1019200094F8560001F092FA169B636005B0BDE88A
:10193000F08F294984F838A0EAB2895D84F85020F4
:1019400076BB0B3D012D8CBF00250125053A012AF0
:1019500004D8BBF10C0F38BF4FF00C0B1F4B9DF898
:101960003C201B7884F85350E37701259DF85430D0
:1019700084F8511084F8522084F82130A573A4F81B
:101980001CB0A77784F82090FFF7E2FB2846FFF70A
:10199000FFFC134801F00CF8124801F075F8B5E7A8
:1019A000012E04D1A5F10C035D425D41CEE7002577
:1019B000CCE75046FFF7ECFC022384F8383004F102
:1019C00038001623A56484F84C3000F0F1FF9DE741
:1019D000442700201C3C0108DE440108C008002008
:1019E0007C270020522700202DE9F04F87B0DFF838
:1019F000B4B29DF864A09DF84C90029314469DF8F3
:101A000054309DF85020BDF84880039205468BF86D
:101A100001A0BDF8446001930F4601F012FABAF13B
:101A2000000F18BF4FF00008DFF87CA2039AB9F14D
:101A3000000F08BFFF22012D8AF8002000F0C880A7
:101A4000052D48D0002D40F0C080284600F010FE43
:101A50000B2238468BF844208BF83850CBF83C40AA
:101A600001F092F9019B8BF8450041F60402002B2E
:101A7000ABF812209AF800208BF8162014BFF2223F
:101A800001228BF81720F600012289F001098BF85A
:101A900018208BF80E50ABF810608BF814508BF8B0
:101AA0001590FFF755FB2846FFF772FC0BF1380045
:101AB00000F07EFF0BF10E0000F0E6FF7B490868A6
:101AC000496804AA03C204A800F076FC40F2FF10A3
:101AD00000F046FC71E0012000F0CAFD09224FF041
:101AE00000098BF8442038464FF44872CBF8402068
:101AF0008BF83890CBF83C4001F046F94FF4805217
:101B0000ABF812209AF800208BF845008BF81620CD
:101B100028460122F6008BF817208BF80E90ABF8C0
:101B20001060ABF814908BF81890FFF731FC0BF1B4
:101B3000380000F03DFF0BF10E0000F0A5FF5B49FF
:101B40008868C96804AA03C204A800F035FC40F202
:101B5000FF1000F005FC40F6B80000F0DDFB00F0DF
:101B6000EF0140F6B80000F0C7FB042140F6B900D1
:101B700000F0C2FB40F69B0000F0CEFB00F0E3015A
:101B800041F0080140F69B0000F0B6FB40F2D16046
:101B900000F0C2FB40F01801C9B240F2D16000F081
:101BA000ABFB40F2AC6000F0B7FB00F08F0141F0FE
:101BB000500140F2AC6000F09FFB4FF4FA5202FB80
:101BC00008F2B2FBF4F2CBF8082007B0BDE8F08FC2
:101BD000002000F04DFD36498BF83850E2B2C95D67
:101BE0008BF85020002F4DD10B3C012C8CBF0024D2
:101BF0000124053A012A02D80C2E38BF0C26029B7C
